:020000040800F2
:1000000000500020D53301087134010899CA000856
:1000100071340108713401087134010800000000D6
:100020000000000000000000000000007134010822
:10003000713401080000000071340108D76B00081A
:1000400071340108713401087134010871340108F8
:100050007134010871340108E76E0008F16E000880
:10006000EF6E0008ED6E0008EB6E000809590008FD
:10007000F9580008E9580008D9580008C95800087C
:10008000B5580008A15800087134010871340108FE
:10009000713401087134010871340108E96E0008F7
:1000A00071340108D9D3000871340108C9D300089C
:1000B000B9D30008A9D3000899D30008475D000808
:1000C0004D5D00083D5D0008435D00087134010886
:1000D00071340108156C0008096C000871340108BE
:1000E000E56E000871340108713401080000000059
:1000F0000000000000000000000000000000000000
:0C01000000000000000000005FF808F1A3
:100110002DE9F04FB34B95B01B780690012B07D11A
:10012000B149B24A0968C9691180B1490988518049
:10013000B04D2A78002A00F01185072B40F02A8262
:1001400006F0F0FC0890AC4B1A68099312F4806F2B
:1001500005D0AA48836813B100F150019847A84B15
:100160001B68190705933ED5A64EA749B46824F02D
:10017000004012F0D7FE0A22A44BB3F9043093FBDF
:10018000F2F3002800F00982A14A1288520740F1D8
:1001900004826A889B1A9BB218B210F1B30FBCBFDD
:1001A00003F5B47318B2B328C8BFA0F5B473994A65
:1001B000C8BF18B22B7A1278002B0CBF4FF0FF3358
:1001C000012317070FD5944A434312681BB2107ED0
:1001D00043431E2093FBF0F012F0B2FC0146204690
:1001E00012F0F8FBB0608D4B8D4E1B68B6F90640DF
:1001F0005A890A96944280F2D2814FF07E53EB6086
:10020000884B4FF0000A1F8B95F9083095F8059040
:10021000002B14BF01234FF0FF3395F80480794E73
:1002200007930A9B33F91AB0ABEB07000028B8BF5D
:100230004042B0F5FA7FA8BF4FF4FA70BAF1020F4E
:1002400000F0C0814045CCBFA0EB0800002012F0B8
:1002500077FCBB4546F82A00C0F2C2810AF1010AC8
:10026000BAF1030FDDD1099B1E6816F4805800F027
:10027000BE81B4F5FA6F2346A8BF4FF4FA63B3F515
:100280007A7FB8BF4FF47A73A3F57A732A7C22B1D0
:100290006A7C5343642293FBF2F34FF0640E93FBAA
:1002A000FEF2614802F1010C30F9121030F91C0025
:1002B0006FF0630C0CFB0233401A584390FBFEF0C6
:1002C000084400B212F03CFCDFF838918246C9F8CD
:1002D0000C00B8F1000F1DD01D2011F09DF8C8B121
:1002E000524BDB78B3B95249504612F073FB12F00F
:1002F00057FE4FF47A7300B2000390FBF3F3C7F597
:10030000FA6000B2584340F30F30384412F018FC42
:10031000C9F80C003E4B1F8879063BD53B4BB3F91F
:1003200004000A2390FBF3F02B8BC01A00B212F0EA
:1003300007FC404912F058FC3F49054612F04CFBBF
:1003400010F0ABFC8346284610F0A7FC2D4D8146EB
:100350002B6859461846099312F046FCD5F804A0BC
:1003600007905146484612F03FFC079A0146104656
:1003700012F030FB59462860504612F035FC099BBC
:1003800082461946484612F02FFC0146504612F0AC
:1003900023FB6860059B174D13F0140F1AD017F458
:1003A000027F17D01B4BDFF85C901A7812F0100216
:1003B00000F03281AB7EE869002B0CBF01234FF0C7
:1003C000FF33584312F0BCFBD9F8041012F004FBC1
:1003D000C9F80400194BDFF84C901A780793002AEB
:1003E00036D02DE07A170020901F002098150020AD
:1003F0008A1C0020380C00207C170020FC220020E2
:100400007017002008130020000070411C2A0020F3
:10041000661300200C15002074170020982F002070
:100420003C130020801700209C2F00208013002008
:1004300000007A4435FA8E3CDB0FC93F00000020F3
:10044000B9F81A30A342A1BF00239E4A6B6493609F
:1004500095F84A40002C30D0BA072ED09A4B9B49D1
:100460001F6A384612F068FD002840F021813846A6
:1004700015F0ACF9E96C12F0B7FB15F02FF9B0F5F7
:10048000617FA8BF4FF4617012F05AFB904912F0DF
:10049000ABFB10F002FC0746204612F051FB394638
:1004A00012F0A2FB15F01AF900B212F049FB854CCC
:1004B0000146E06812F090FAE06095F85070002F65
:1004C0005AD0844B0420D3F8EC4044F620639C427D
:1004D000A8BF1C46B4F57A7FB8BF4FF47A74A4B2B3
:1004E000A5F8524010F098FF08B9F30044D54FF436
:1004F0007A73B4FBF3F4642393FBF4F4DFF8E8A11C
:10050000142CA8BF1424DAF80030B8F1000F00F062
:10051000D1805E8E76086B496A6DD1F80C80531CD1
:100520006B65404605EB420B059312F039FD059BC8
:10053000ABF858009C42DCBF00236B656B6D05EB8C
:100540004303B3F9580012F0FBFA0146404612F09B
:1005500041FA12F025FD00B20028B8BF4042B04277
:1005600040F3AB80DAF80030988E12F0E9FA5A497D
:1005700012F03AFB079B586099F81E30002B00F0F0
:10058000D481022B00F0B280032B00F0A281534BE8
:100590005888B0E000230893D5E56B8023E6B4F5D6
:1005A000FA6F187ABFBFA31A5843C2F5FA6290FBDC
:1005B000F2F0C0F1640012F0C3FA494912F014FBE2
:1005C000E8601DE64845D8BF0020079BC8BFA0EBE8
:1005D0000900584312F0B4FABB45B060BFF643AE11
:1005E00056F82A1001F1004146F82A1036E63D4B34
:1005F0005A8B94420EDBB4F5FA6F2346A8BF4FF432
:10060000FA634FF47A719B1A4B43C2F5FA62B3FB5B
:10061000F2F33BE61346F4E7E979B5F92030A8791F
:1006200061B3E11A0029B8BF4942814210DD6A6214
:1006300001229C4285F82820C8BF404212F080FA6F
:100640000146D9F80C0012F0C7F9C9F80C00C1E650
:1006500095F8281019B1296BE96285F82820E86916
:100660001844B0F5FA6FA8BF4FF4FA60B0F57A7F7E
:10067000B8BF4FF47A7012F063FAE6E7E21A82EA42
:10068000E27EAEEBE27E864507DD022192FBF1F2CF
:100690006A63012285F83820DFE795F82820002AD0
:1006A000DDD02A6B85F83810EA6285F82810D6E785
:1006B0000020F9E6B3F932602DE74FF07E53079A38
:1006C000536059E708130020DC2900208FC2753CD5
:1006D000D06D393A340000206F12833A7C2100201B
:1006E0000AD7233C8017002074170020B5F8520069
:1006F00000F57A7080B299F81F400234E4B2002FFE
:1007000000F0FC80002800F0F9808C4B00261B686C
:100710008B4FB0FBF3F000B2A5F8800012F010FA96
:1007200001464FF07E5012F013FB8046DFF818921E
:1007300007F1100AA642C0F2D480824B1B78092B25
:1007400011D1814B814E186814F0C8FF804B308066
:10075000D3F8EC004FF47A7390FBF3F012F0F0F959
:1007600012F01EFC7080B5F98030002B40F3DF8062
:1007700000273E46DFF80C82DFF8CCA1A8F1100973
:10078000A742C0F2C18095F850300024002B18BF5A
:100790000226704BDFF8F091D3F80080694B1B788C
:1007A000099308F105030A93B44240F3EF80099BD3
:1007B000694C092B07D1654EB4F88030E06BB380EB
:1007C00012F0EEFBF080654B93F82160002E60D0B4
:1007D0001E2010F021FE00285BD0614B1B885F06B5
:1007E00057D494F8BC30B34214D084F8BC6030467F
:1007F00012F0A6F95B4912F0F7F95B49064612F0D0
:10080000EBF810F04AFA594B9860304610F045FA70
:10081000C4F8C000079BEE6BD3F8089030464946F9
:1008200012F0E2F9D5F84480D5F8C0708246394616
:10083000404612F0D9F90146504612F0CBF84C4927
:10084000824612F079FB08B9DFF824A149495046E5
:1008500012F07CFB08B9DFF81CA149464046C5F8F8
:100860003CA012F0C1F939468046304612F0BCF97E
:100870000146404612F0B0F83D49064612F05CFBD6
:1008800000B93B4E3B49304612F060FB00B9394E8F
:100890006E64002384F85030374B1B78002B40F0F7
:1008A0005081364EB378002B00F04B81344C2378C6
:1008B000013B0A2B00F21C81DFE813F00E01C0019E
:1008C000F8012C021A011A0146025A028805A505F0
:1008D000B60599F82000C0EB401300EB8300C00080
:1008E00008E75AF8261059F8260012F073F8414626
:1008F00012F07AF947F8260001361BE7B5F8803088
:10090000013BA5F880302EE758F8270059F827104A
:1009100012F062F8022F3E46B8BF022648F82700C0
:100920004AF82700F6B201372AE7A5F8803095F893
:100930005030002BB0D0002625E700BF581700200C
:10094000BC0C00207A170020081300209815002006
:1009500034000020982F0020380C00208017002041
:100960006613002035FA8E3CDB0FC93F00000020E3
:1009700000C0F94400C0F9C4501A0020702F0020B4
:10098000FE150020CC0C00200AD7233C022C15BFFA
:1009900098F8000098F8010098F802B098F809B0AB
:1009A00012F0CEF8494612F01FF94FF08041074689
:1009B00012F0D6FA60B14FF08041384612F00AF8D2
:1009C000A44912F011F90146384612F005F807461D
:1009D000A3000593A04BA14953F8240012F004F999
:1009E00020F000439E4A0593059B42F824000C32F8
:1009F000824642F82430BBF1000F20D0584612F056
:100A00009FF8494612F0F0F883465146504612F0DE
:100A1000EBF8059912F0E8F8594612F0E5F8594656
:100A20000B904FF07E5011F0D5FF0B9A0146104607
:100A300011F0D2FF0146504612F0D6F8824689499D
:100A4000384612F0D1F8514612F0CEF80A9B07460C
:100A500013F8010B0A9300B312F072F8494612F032
:100A6000C3F8059912F0C0F87F49824612F078FA6F
:100A700068BB0021504612F055FA50BB51464FF06A
:100A80007E5011F0A7FF01464FF07E5012F060F942
:100A90000146384612F0A8F80746099B0C2B05D1F1
:100AA000384612F07DFA714B23F81400704938462D
:100AB00012F042FA00B96E4F6E49384612F046FA0B
:100AC00000B96C4F6C4BA200D75001346CE649461C
:100AD000DAE74FF07E51D7E7684B1B78DD0707D583
:100AE00080200DF07FFD08B10EF028F907F01CFD05
:100AF000F37833B3614B1D7815F0010509D1604BD4
:100B0000DFF8A0911F785F4BD3F80080BD42C0F2A0
:100B1000AA845D4B5D4D1B68D5F8F8209A4240F2DF
:100B2000B5842378012B0CD1584C94F8F72042B9A6
:100B3000B378032B00F0A28407F0F6FC012384F8BD
:100B4000F730534B1B78072B05D105F0EBFF089BC3
:100B5000C01A464B988000224C4B1A704C4F3B7881
:100B6000072B40F0A38405F0DDFF0890494C636833
:100B700020469847A246002849D00026B4F8B45031
:100B800084F85560DFF82081002D40F03385626ADB
:100B9000B4F93C3094F856109B1A2363A26AB4F956
:100BA0003E3004F130009B1A6363E26AB4F94030CE
:100BB0009B1AA36309F08EF9374B1B78002B40F08A
:100BC000D7841D4604F12C0656F8040F11F0B8FF27
:100BD000DAF8201012F008F805F59C720146DAF8F0
:100BE00034310AEB0200984705F5D4720146DAF871
:100BF000A4310AEB02009847DAF8B8300146D6F87B
:100C0000F800984724356C2D48F8040FDCD1204CAF
:100C10002278072A05D105F085FF089BC01A134BDF
:100C200018801A4A92F8FD301546002B00F0B8855E
:100C3000013B82F8FD3015B0BDE8F08F0022174B64
:100C40001A60174B1A60104A12685A600323237007
:100C50004EE700BFD7A36841081300206F12033B83
:100C6000DC0C002000004843A4707D3F9815002054
:100C700000C0F94400C0F9C4740C00200413002023
:100C8000A0150020541A0020C4130020380C0020A6
:100C90007A170020FC220020341B00206C2F00203B
:100CA0004C17002054190020802500200FF086FCEE
:100CB000954D964B1A686B6864339342BFF418AF36
:100CC00040200FF061FC00287FF412AFDFF8E082D3
:100CD0004027C246DFF8DC922B6818F8030068B1A1
:100CE0000FF0ACFCD9F80030013F03F1FF33C9F835
:100CF00000302B6803F101032B60EDD12B681AF84B
:100D00000330002B7FF4F4AE2B604FF0FF336B60A9
:100D100004239CE70FF052FC7D4A5021A2F10C0302
:100D200001932923029200934920A2F10A03163A63
:100D300007F026FB00287FF4DBAE4FF0FF32724B4A
:100D400018605A60072382E70FF038FC0523002162
:100D50000093704B02910191A3F10802532007F018
:100D60000FFB00287FF4C4AE674B186008236EE7C2
:100D70000FF024FC684B694D186814F0AFFC8046F6
:100D8000D5F8C40014F0AAFC814640200FF0FCFB0B
:100D9000294600287FF4ACAE5B4D614F2B68787814
:100DA0004C2B01F29883DFE813F04D0053006100F3
:100DB00068006C0070007600840088008D0092004E
:100DC00097009E00A30007011101160122012701CF
:100DD0002C013101390141014901510159016101E0
:100DE000690171017E01870190019901A201AB01A6
:100DF000B401BD01C601CC01D501DC01E201E8016D
:100E0000EE01F401FB01020209020F0215021C02AD
:100E1000830289028F0295029B029F02A302A8020D
:100E2000AD02B202B802BE02CB02D002D502DA0293
:100E3000DF02E402EA02EF02F402F902FE02030317
:100E400008030C03374A384938480FF0B0FC09E072
:100E5000374B384A0193384B384900933848394B5F
:100E60000FF0A5FC2B6801332B6041E6364B374A67
:100E7000374938480FF09BFCF4E7374A2A4937488E
:100E8000E3E7374A28493748DFE7374B3749B3F9B3
:100E900000203748D9E70FF0C9FC32883249424375
:100EA000B1F90010034692FBF1F23248D2B2324956
:100EB000E0E732882D493148C7E7314B2B499A8901
:100EC0003048C2E72E4B2949DA892F48BDE74FF059
:100ED0007E522E492E48B8E71FFA89F31FFA88F28E
:100EE0002C492D48C6E72D4B2D499A8A2D48ACE751
:100EF0002D4B1B68D80404D591F8C8202B482849ED
:100F0000A3E70F232B60ADE74C170020C41300208C
:100F1000FE7E0108DC80010818160020380C002035
:100F2000241C0020F9960108BB9D010805970108C3
:100F30004497010819970108509701082497010860
:100F400032970108139701085A970108639701081F
:100F50006F970108759701080C000020839701081E
:100F60003B1F0020969701087E2F002051B30108F7
:100F7000A1970108B2970108AC970108BD97010835
:100F800004160020C5970108D197010818AE010882
:100F9000DD970108B4980108E89701084015002082
:100FA000D0A90108F497010800160020FB9701085A
:100FB000987E01086C2F00208D498E488B784A78E6
:100FC000097800918C490FF0F2FB4BE78B4B8C4971
:100FD0001A888C4839E7864B9B79012B7FF442AF06
:100FE000B1F9CC30B1F9CE208748884942E7884B27
:100FF00088491A68884828E7884B86499A7888483B
:1010000023E7884B83491A7887481EE70C2303FBA4
:101010000011864891F8D0207E4916E70C2303FB87
:101020000011834891F8D2207A490EE70C2303FB84
:101030000011804891F8D120764906E70C2303FB84
:1010400000117D4891F8D9207249FEE60C2303FB7C
:1010500000117A4891F8D3206E49F6E60C2303FB81
:101060000011774891F8D4206A49EEE60C2303FB7F
:101070000011744891F8D8206649E6E60C2303FB7A
:1010800000117148B1F8DA206249DEE60C2303FB57
:10109000001191F8D63091F8D52091F8D7106B480F
:1010A00000916B498FE76B4B6B4819684B780A7856
:1010B00089780091664986E7664B684819680B791C
:1010C000CA784979009162497DE7624B64481968A2
:1010D000CB798A79097A00915D4974E75D4B614863
:1010E00019688B7A4A7AC97A009159496BE7594B4A
:1010F0005D4819684B7B0A7B897B0091544962E704
:10110000544B5A4819680B7CCA7B497C0091504962
:1011100059E7504B56481968CB7C8A7C097D009171
:101120004B4950E74B4B534819688B7D4A7DC97D2D
:101130000091474947E7474B36491B684E481A7E9E
:1011400083E6444B4D4819680B7FCA7E497F009166
:101150003F4938E73F4B2F491B68494893F8262001
:1011600073E63C4B2B491B6846481A8C6DE6394B9D
:1011700028491B684448DA8B67E6364B25491B68CB
:1011800042485A8C61E6334B22491B6840489A8C8E
:101190005BE6304B1F491B683E4893F8272054E616
:1011A0002C4B1C491B683C4893F82C204DE6294BDE
:1011B00018491B68394893F82D2046E6254B1549F8
:1011C0001B6837485A8E40E6224B12491B68354847
:1011D0009A8E3AE61F4B0F491B68334893F8362026
:1011E00033E61C4B0B491B68304893F837202CE63C
:1011F0006E1300200F9801080698010816160020AB
:10120000D0A901081F98010827980108B49801087F
:101210008025002051B3010835980108E8220020FC
:101220003E980108892200204E9801086098010824
:1012300068980108709801087C980108889801084E
:101240009098010899980108A2980108BA98010895
:10125000B198010874170020C0980108C8980108C7
:10126000D1980108D8980108DF980108E69801088C
:10127000EE980108F6980108FF980108F89801080F
:101280000699010818990108259901083099010863
:101290003F990108529901085F9901086D99010869
:1012A0007E99010895990108A7990108C19901083B
:1012B000804B81491B6881481A8FC6E57D4B7E496A
:1012C0001B687F485A8FC0E57A4B7B491B687D4875
:1012D0001A8DBAE5774B78491B687B485A8DB4E57F
:1012E0000A797A487449B0E54A7979487249ACE597
:1012F000784B7149DA787848A7E5764B6E491A79C8
:101300007648A2E5734B6C495A7975489DE5714A58
:101310007449D38974485289ACE56E4A7149138A7D
:1013200072489289A6E5724B188811F009FC714940
:1013300011F05AFC11F034FE5F4902466E4884E514
:101340006B4B5D49DA786D487FE56D4B5A495A79A8
:101350006C487AE56C4B5849DA786C4875E591F839
:10136000F4206B48544970E56A4B53499A7F6A48A8
:101370006BE5684B504993F82020684865E5654B5C
:101380004D495A8C664860E5624B4B491A7A65486C
:101390005BE5654B48491A79644856E5624B464916
:1013A0009A78634851E5604B43491A8861484CE597
:1013B0005D4B41495A89604847E5BA783E495F48E4
:1013C00043E55F4B3C491A685E483EE51A2010F041
:1013D00023F8A0B15C4B1B888BB95C4B10A91B6830
:1013E0000E201093069B119306F01CFD584B1A68B3
:1013F000584B1A600A232370069806F061FD06F028
:10140000DDFCFFF775BB544B1B78002BF4D01A2082
:1014100010F002F80028EFD1504B93F8F730002B72
:10142000EAD109232370EAE74D4B1A684D4B5B68FC
:10143000C833934211D2B378032B0BD14A4D28689D
:101440000DF06DFC00232B60484B1B78022B01D163
:101450000DF050FE0123FFF7FABB0FF0CFF8002884
:10146000E9D1FFF745BB414659F8250011F050FD81
:10147000002801F03C800135FFF748BB80200DF0CB
:10148000B1F800287FF45DABFFF756BB2378012B42
:101490003FF457AB95F8F730002B3FF452AB07F011
:1014A00025F8002385F8F730FFF74BBB002308939E
:1014B000FFF75CBB7417002051B30108D7990108EE
:1014C000E5990108EF990108FC9901080DA70108A9
:1014D0000D9A0108E82200201A9A0108239A0108AF
:1014E000359A0108B4980108459A0108539A0108F1
:1014F000361B00200000C842659A0108709A010856
:10150000E21400207D9A0108601B00208B9A0108DC
:10151000989A010880170020AE9A0108BF9A010826
:10152000D99A0108F39A010804160020059B0108C6
:10153000169B0108299B0108389B0108499B01085B
:10154000C01D0020549B0108F8150020F415002050
:10155000F8140020F4140020AC170020380C0020F0
:10156000C41300204C170020782F002055170020AE
:10157000834E04F12C0944460AF59C7897F800B094
:1015800059F8040FBBF1170F02BF05EB0A039B8F3D
:10159000338011F0D5FADAF8201011F025FBBBF1F9
:1015A000080F014604D1059014F098F80599308091
:1015B000DAF8343140469847DAF8A431014608F1A8
:1015C000700098473B788346032B02D114F086F8CD
:1015D0003080DAF8B8305946D9F8F8009847023523
:1015E000062D44F8040F08F1240806F10206C5D1BF
:1015F000FFF70DBB634BD8F800205B780796099383
:101600004FF47A73B3FBF2F3C3EB431203EB8203A1
:10161000DB009BB205933B7804F124070A93584BF7
:10162000B3F90690059B5B080B93059B9D4201BF98
:101630000023BB64C4F888303B60534BF318B3F904
:101640003C00BB6C0344BB6411F07AFAD4F88820E8
:1016500002F10108B8F1010FC4F8888008D1002315
:10166000012DE067A067C4F8803060D1002033E02E
:10167000D4F878A00D9251460C9011F0ABF9834646
:10168000404611F05DFA0146584611F061FB5146A3
:1016900011F0A2F90C9B01468246E067184611F052
:1016A00099F9594611F0A0FAD4F8801011F094F984
:1016B000012D8346C4F88400C4F878A0C4F88000E3
:1016C0000D9A34D1B8F1010FD0DD104611F038FA7F
:1016D0000146584611F03CFB14F0C0FA0A9B8046C4
:1016E000032B05D113F0FAFF01230FFA80F90793BA
:1016F000099BABB1184611F023FA414611F012FCD8
:1017000070B1079B13B11E4BA3F806901F4808F059
:10171000D1FB00221E4B5A609A60DA60FFF777BA5D
:101720000B9ABB6C1344059A93FBF2F33B600236B1
:10173000062E07F1040704F114047FF476AF079B2B
:1017400013B10F4BA3F80690012D11D10022114BBC
:101750001B689A621A63DA620F4B93F8FC3023B16C
:101760000E4B1B8823F4006313B901200DF042FDDA
:10177000054AB2F8B430013BA2F8B430C9E700BF63
:1017800098150020E8220020FC220020B023002031
:1017900080250020901F0020380C0020A41300207A
:1017A000AE4B5B79002B00F02E84AD4B1B78013BD8
:1017B000DBB285F8FD302378072B40F0278405F055
:1017C000B1F90B90A74B4FF07E501B680893EB6864
:1017D0000E93D5F8003119460A9311F0FBF8A24B8D
:1017E000196811F001FA4FF07E510C9011F0A4FB32
:1017F00010B94FF07E530C934FF0000800259B4B1F
:101800009B4C07939B4B0993DFF8C892294659F8E4
:1018100028304FEA88060593974B53F828703846CE
:1018200011F076FBE8B909F1C80959F82890059834
:10183000494611F0CFF8824620F00041384611F0B9
:1018400071FB58B12946504611F08AFB002800F080
:10185000E1834946384611F0BFF80590874B059A59
:10186000F250874BB3F8009019F0030F3AD0B8F15B
:10187000020F37D0089B93F82EB0584611F060F94C
:10188000804BF15811F0B0F98246CBF1000011F015
:1018900057F907460146504611F044FB40B95846F7
:1018A00011F04AF95146074611F046FB00B9574678
:1018B000754B33F91800099BB3F90030C01A11F0C9
:1018C0003FF9724911F090F90146384611F082F85B
:1018D00019F0010F0D9000F0D1836D4B196811F0D4
:1018E00083F905906B4B05983344D3F804A0514617
:1018F00011F070F894F810310746002B00F0858045
:10190000069AD4F81431D31A634A126893427CDDE4
:10191000089B93F84830022B02D1012005F053FABE
:10192000B8F1020F40F05D845C49504611F018FB9D
:10193000002840F075845A49504611F0F3FA002807
:1019400040F06E84574B3846D3F8009009F1004BB5
:10195000594611F0E7FA002840F0658449463846B8
:1019600011F0EAFA00B94F46079B069A1D60D4F8B9
:101970001431D31A4C4A1268934223DC4FF07E5143
:101980000A9811F0CFFA00283FD0484BDFF804B195
:10199000D3F80090DBF80400494620F0004011F035
:1019A000C1FA90B3DBF80810484621F0004111F06D
:1019B000D7FA50B3DBF80C10484621F0004111F083
:1019C000CFFA10B33A4B186810F0020019D0394B17
:1019D0002D4839491A68B1F90CE0B0F90030A3EB91
:1019E0000E03002BB8BF5B4293420EDAB0F902300F
:1019F000B1F90E105B1A002BB8BF5B429A4204DDAE
:101A0000002084F8100105F0DEF92C4B0E98F158F7
:101A100011F0EAF8394611F0E7F8DFF8BC90B8F1B8
:101A2000020F014646F8090006D1254A254B1068E9
:101A30001B689847C9F80800079B1B680D93224B49
:101A40005968224B186811F0CFF80C9911F0CCF8B6
:101A50001F4BF15811F0C8F840E000BFE822002009
:101A60008922002074170020E0280020281500207B
:101A7000380C0020421B0020D42800203C0D002000
:101A800066130020DC0C00201C2A0020CDCCCC3DAD
:101A9000BC28002080250020E828002000C0F84451
:101AA00000C0F8C400290020E4280020F02800200D
:101AB00070170020EC280020361B00209028002002
:101AC000B429002010290020000000208C220020D2
:101AD0009C280020740C00201C150020394611F0B1
:101AE00083F80D9910F078FFA54B0F90D3F800B054
:101AF0000BF10049494611F015FA38B90F9A5946C9
:101B00001046914611F018FA00B9D946B8F1020F03
:101B100040F08C8394F81831012B02D0192B40F03F
:101B200085834FF00103974938460F9311F018FA57
:101B30000F9B00B90346DBB23BB10D9B29F000407F
:101B400023F0004111F0EEF910B1079BC3F80090AB
:101B5000B8F1020F00F093808B4A8C4B51461B6802
:101B6000B05898478A4A8B4B01461B68B058984733
:101B7000089B814693F83730002B00F06183864B39
:101B80001B88002B40F05C83844BF158844B186811
:101B900011F02AF84FF07E51824611F0CDF908B9C4
:101BA0004FF07E5A7F4B5046196811F01DF80146E0
:101BB000059811F019F8494610F00CFF7A4B814650
:101BC000F15810F007FF794B196811F0C1F8764B06
:101BD000824646F80390089B93F84830002B44D087
:101BE000734B1B78DA0740D54FF07E510A9811F0FD
:101BF000ADF9F8B194F81031E3B96E4B2AF000401A
:101C0000196811F0ADF9A8B16B4B27F000401968C5
:101C100011F0A6F970B1694BF058694B20F0004003
:101C2000196811F07FF928B1012384F81031069B5F
:101C3000C4F81431069AD4F81431D31A614A1268E0
:101C4000934212DA5C4B27F00040196811F06AF9F0
:101C500040B95A4BF0585A4B20F00040196811F027
:101C60007FF910B1002384F81031574B0E98F158CA
:101C700010F0BAFF514610F0B7FF544B985194F84A
:101C80002431534F23B9079BBD511D604F4BF55075
:101C9000079B08F1010804330793099BB8F1030F70
:101CA00003F1020309937FF4AFAD4A4E3278072A5D
:101CB00005D104F037FF0B9BC01A474B588033788F
:101CC000012B40F0BF8204F02DFF4449D4F82831A5
:101CD000414A0968C31A93805B1A0590D380C4F8FF
:101CE00028013F4B3F4E1B6893F82CA03E4B1B68CE
:101CF00013F4805F00F004832D4BB4F82E911B7811
:101D00004846DB0758BF394BF6685CBF1B8BA4F80D
:101D10002C3110F015FF80460146304611F00CF9C9
:101D2000002800F09882324BD4F834111868C4F8B7
:101D30003811C4F83C11C4F8300110F04BFEFF23F9
:101D4000C4F8400184F84431304611F04FF931466F
:101D5000A4F82C01404610F03DFEC4F84801D4F828
:101D60004C512946D4F8480110F0F2FF4FF07E5153
:101D7000054611F0E1F800283CD14FF07E5539E0DE
:101D80000429002000009642142900200829002080
:101D9000642900200C29002066130020E80C002094
:101DA000B8280020B4280020540D00208C220020E8
:101DB00004130020F8280020F4280020740C0020D0
:101DC000FC280020E8280020A82800203415002046
:101DD0001C1500207A1700209815002058170020A5
:101DE00074170020081300207C17002080170020A3
:101DF000181600200021284611F0A8F800B9002587
:101E0000C4F84851864CDFF86CB22168386810F08D
:101E1000E3FDDBF8001010F0DFFD824910F0E4FE76
:101E2000814B8046D3F8009009F10046314611F00D
:101E300079F8002840F082824946404611F07CF84B
:101E400000B9C8466168786810F0C6FDDBF8041078
:101E500010F0C2FD734910F0C7FE834601463046BC
:101E600011F07EF830B9594648464E4611F064F8F4
:101E700000B95E46A168B86810F0AEFD694910F07F
:101E8000B3FE6A4B81461F6807F10044214611F0FA
:101E900049F830B9394648464C4611F04DF800B97A
:101EA0003C46634B5B780BB904F10044BAF1000F78
:101EB00025D0604B5A7912B35F4A1778FFB1187872
:101EC00010F03AFE8146384610F03AFE0146484688
:101ED00010F08AFE594B0746188810F02DFE014677
:101EE000384610F035FF5649074611F025F800B97D
:101EF000534F4FF07E51384611F028F808B94FF093
:101F00007E574FF0000A4F4BD3461B78DFF868919D
:101F100006930023069A9342C0F2308251465846F7
:101F200010F058FD484C4FF07E51C4F800010646B1
:101F300011F016F8002800F0618231464FF07E5013
:101F400010F006FF0025074610AE069BAB4200F3DB
:101F50004C820FF067FA18B14FF07C53C4F8483147
:101F600094F9440110F0ECFDD4F840318246079317
:101F7000D4F83C31D4F830010893344B0025DB7899
:101F8000D4F848B10B9311F00BF88046D4F838011F
:101F900011F006F82E4B81461E68304611F000F80D
:101FA00007462C4B1B6803F0100203F480530D937B
:101FB000294B0C92B3F90630284A0993284B147820
:101FC0005B8B04F001040A93069B9D42C0F03A82A9
:101FD0002CB9244B244A0699A14200F373821A4C6F
:101FE00094F8A021002A40F07382204B1B78072B25
:101FF00005D104F097FD059BC01A1D4BD880012325
:102000002370FEF718BE0123FFF7D3BB00230B9309
:10201000FFF7D8BB3946484610F0DCFC1DE400BF92
:10202000281500206F12833A90220020942200206D
:10203000781700206E130020841C0020B4150020A7
:10204000713DAA3FA0150020380C0020801300200D
:10205000541A00207C1700203C1300200413002099
:1020600080170020A4150020541900207A170020A2
:102070009815002034150020980D0020D4F8B09059
:10208000D4F8B4704946384610F060FF00B94F46A6
:10209000AB4BB3F90000B3F902300028B8BF40429F
:1020A000002BB8BF5B429842B8BF184610F048FDFD
:1020B000A44910F099FDA44B82461B78002B55D003
:1020C000A24B2946D3F800B0584610F049FF00282B
:1020D00000F085809E4B2946D3F80090484610F0CA
:1020E0003FFF00287BD007F100409A4910F07CFDAB
:1020F000594610F02DFE4FF07E5110F06DFC514608
:102100000746484610F066FC494610F021FE4FF0A5
:102110007E51814610F010FF08B94FF07E592946D4
:10212000484610F013FF00B9A9463946484610F05A
:102130005BFD4FF07E51074610F0FEFE08B94FF0F0
:102140007E572946384610F001FF00B92F46824BD2
:102150000D98196810F048FD0146384610F044FD0E
:102160000146059810F038FCFFF7BBBB7B4B7C4960
:10217000D3F80090484610F0D5FE60B349464FF0C2
:102180007E5010F027FC774910F02EFD5146834613
:10219000754810F01FFC0146584610F025FD4946D1
:1021A00010F01AFC694B196810F01EFD8146294693
:1021B000484610F0C1FE90B94946664810F0C8FD87
:1021C00007F100470146384610F00EFD4FF07E51F2
:1021D00010F002FCADE75D4BD3F80090E7E728462E
:1021E000A7E7624B1B6899077FF5BEAB099BB3F964
:1021F0000000534B33F91830C01A10F0A1FC5C4BAF
:1022000007465049186810F0EFFC0146384610F0B8
:10221000EBFC5146059010F0DDFB0746FFF7A4BB31
:102220002F46FFF7A1BB5F46FFF79EBB4FF00103B0
:102230004FF07E51D4F800010F9310F087FE77E441
:102240002946B5E4072B03D104F06CFC059048E562
:102250000023059345E5B4F8500110F071FC804669
:102260000146304610F072FEF0B1D4F85411D4F8A3
:10227000C400C4F83011C4F83C11C4F8380110F09F
:10228000A9FB0123C4F8400184F84431304610F022
:10229000ADFE4146A4F82C01304610F09BFBC4F87B
:1022A0004801D4F858515CE5B4F82C314B4513D8AB
:1022B000304BD4F834111868C4F83811C4F8300120
:1022C000C4F83C1110F086FBFF23C4F8400184F8E9
:1022D0004431C4F8485142E5D4F85411D4F8C4004C
:1022E000C4F83011C4F83801C4F83C1110F072FB86
:1022F0000123C4F8400184F84431C4F84851D0E7C0
:102300001D4B588B10F01CFC0146F06810F062FB6E
:10231000184BC4F848011968D4F8C400C4F8301147
:10232000C4F83801C4F83C1110F054FB0123D4F870
:102330005C51C4F8400184F8443112E5B04681E5AF
:102340001C2A0020CDCCCC3DC8280020C428002069
:10235000CC2800200000C842C0280020D02800203F
:10236000AE47813F610BB63B00003443701700203D
:10237000BC2800201816002080170020D9F804106F
:102380004046089310F030FCD9F80810079030460A
:1023900010F02AFC079A0146104610F01DFBD9F8F0
:1023A0000C100790204610F01FFC079A01461046BB
:1023B00010F012FB394610F017FC5946079010F048
:1023C000CFFD079A089B70B91146504610F0B4FD36
:1023D000079A089B00B9924610A941F8232009F1F9
:1023E0001009013396E59346F6E756F8250039467D
:1023F00010F0FAFB46F825000135A6E50FF012F8BB
:1024000038B94FF07C51284610F0AAFD00283FF45F
:10241000A7AD4FF07C51304610F0E6FB0646014672
:10242000284610F07FFD50B931464FF07E5010F035
:10243000D1FA2946064610F07FFD00B92E46C4F8B1
:1024400048618DE52F4A2B019958584610F0CCFB76
:1024500010AB53F825100E90504610F0C5FB0E9BA4
:102460000146184610F0B8FA079910F0BDFB08991C
:1024700010F0B2FA0B9BFBB110F092FDB84203DBF7
:102480004845A8BF484600E0384610F059FB0C9A72
:10249000034662B15CB10D9A4AB90E900EF0C2FFCC
:1024A0000E9B20B9099A0A998A42B8BF3346164A48
:1024B00042F82530013587E510F072FD4045DFDA3E
:1024C0004046E2E752F8241043F82410013482E534
:1024D0000DF084F989E50EF091F800283EF408AB80
:1024E0000A4B1A680A4B1A600A23FEF7B0BB094B65
:1024F000094A1B6803F59C530833C2F8F830FEF70D
:1025000010BB00BF980D0020A4150020F814002077
:10251000F4140020C4130020380C00202DE9F04FE3
:10252000B34A91B013780192002B00F0B280B14B06
:10253000186800286BD004F0DCFCAF4FAF4D386852
:1025400004F0B9FB002862D0386804F0B1FB092818
:10255000AB4C01D03F2851D14FF0000AD046A94ED4
:10256000D4F8009006F1F00BB9F1000F05D04A46FF
:102570003168284615F0B1FB18B9B246B8F1000F22
:102580002FD008365E45EFD3B8F1000F11D0D8F840
:102590000060DAF800E02368F05C1EF80310814266
:1025A00007D15A1CF9B97D2B1DD820202260E85490
:1025B000A95423680BB1D04509D093480EF06AFDA9
:1025C000D04513D991480EF065FD4FF000092368FE
:1025D0009945B4D215F809000EF04AFD09F1010938
:1025E000F5E7B046CDE7E8542260D4E758F8080B89
:1025F0000EF050FD09200EF03BFDE1E72368002BB3
:1026000041F0C981042805D17C4807F02EF811B0AB
:10261000BDE8F08F0C2841F0E1817D480EF03AFDD5
:102620007A480EF037FD8AE701220B4601F0C5B962
:10263000591E685C2028F7D002B123600022714E39
:10264000EA5406F1F0083168284607F00FFA30B96D
:1026500008364645F7D36F480EF01CFD03E04645AB
:10266000F9D273689847002301F0ABB97F2B3FF68E
:1026700066AFA0F12002D2B25E2A3FF660AF13B976
:1026800020283FF45CAF5A1C2260E8540EF0F0FCA6
:1026900055E79846604F614D3A7802F0010200928A
:1026A00055F80A3C002B41F01C8108F10108B8F1F3
:1026B000030F05F1CC05F3D1A9E7012B05D14D2876
:1026C0000CBF0223002301F022B9022B56D10023B4
:1026D0003C2805F8023C4CD03E2849D015F802ECC5
:1026E000BEF1060F41F0FE8015F8014C002C41F0C0
:1026F000D7804FF001094A4B08AE0FCB86E80F0098
:1027000015F8053C15F803AC2B440D93BAF1440FB2
:102710000FFA8AF30C95ADF83830ADF83A408DF8E1
:102720003C90ADF8283001F0AB8000F20C81BAF19A
:10273000050F00F04B8200F2C480BAF1020F00F0E6
:102740008E8100F2A780CA4500F07E813146504656
:1027500001F06AF9002840F07581BAF1740F00F0B9
:10276000C182BAF1770F00F0FA826FF00109C7E277
:10277000012305F8013C032301F0C9B8032B0BD159
:102780000023C0289FBF05F8063C05F8050C05F896
:10279000040C042301F0BBB8042B09D115F8043C48
:1027A00005F8030C5E4005F8046C052301F0AFB892
:1027B000052B93D115F8061C15F8053C15F8042CCB
:1027C0008B420CD94B1C05F8063CCC23424005F843
:1027D000042C144A03FB08230B4498727EE78242C0
:1027E00002D1062301F093B8002301F090B800BF96
:1027F000501A00206419002068190020CC1900200C
:102800004C1A0020F4940108299C01082E9C010810
:10281000339C01083E9C0108041300201A26002066
:10282000FC80010810260020009B002B41F05A80FC
:10283000232824D10123019955F80A2C0B708B4BC6
:102840008B491A608B4B8C481A609A609DF8002067
:1028500059605A7340221A73884A191D1160884AB8
:10286000D278003218BF012283F850200EF090FD7C
:1028700084480EF00FFC4FF480500CF0A1FD824B09
:102880009B7CB3427FF42AAF804B814A1A60814B14
:10289000DC6023E7BAF1030F00F01681BAF1040FF0
:1028A0007FF454AF002404227B4930460EF0B8F880
:1028B000002130460EF0D2F8089B5A1C08921C707A
:1028C000CAE0BAF1240F00F0BF811FD8BAF1200F7F
:1028D0007FF43CAFDFF8D8A1704B9AF80120D91CE7
:1028E0001A709AF8002008915A709AF80220BAF8E3
:1028F00008109A7030460EF0B1F8089B9AF805203F
:10290000591C08911A709AF8062083E0BAF1280F32
:1029100000F0CC81BAF1380F7FF418AF05225F4B7D
:102920004FF001095A700A2200249A705C4A83F819
:1029300000901178DC701971517892785971D91D15
:1029400008919A71C8E0BAF1810F00F0818130D806
:10295000BAF1540F00F0BF8108D8BAF1520F7FF4DA
:10296000F5AE4E4B5A1C08921C70B5E0BAF16E0FD2
:1029700000F03981BAF1800F7FF4E8AE00210A2619
:10298000484B494C1B780B3BDBB299425ADA228800
:102990000898FF2AA8BFFF2200F1010ECDF820E021
:1029A00006700898013100F1010ECDF820E00270A8
:1029B000EBE7BAF1A00F00F0378130D8BAF1820FFF
:1029C0007FF4C4AE394B30461A78344BDFF8F0A0B0
:1029D000591C1A70364B089119890EF03FF8354B87
:1029E000089A1B88511CFF2BA8BFFF230891137066
:1029F000DAF80810304681F3100189B20EF02EF893
:102A0000DAF80010304601F30F0189B20EF026F813
:102A1000294B1A78089B591C08911A705CE0BAF18E
:102A2000B80F00F01381BAF1FE0F7FF48FAE0024CF
:102A3000DFF8909039F81410304601340EF00EF89B
:102A4000042CF7D1002407E0144BDA1C089224224E
:102A50001C7083F801A09A704FF001093CE0042239
:102A6000164930460DF0DCFF36E000BF6819002043
:102A7000FF6C0008140E00205E9C01086419002001
:102A8000241C00202E9C0108A2250020F04F0020CD
:102A9000EFBEADDE00ED00E0291C00201631002065
:102AA000000D0020A015002014190020841C002017
:102AB0006E130020B415002069130020649C0108E7
:102AC000BC150020981500200222B44B5A70DA1C65
:102AD00083F800A008929C70ADF82A90B9F1000F1D
:102AE00066D0089B55F80A0C0993AC4B0893036811
:102AF0001B6A03B19847089B099EF61A00230793A7
:102B000024238DF818304D238DF81930BDF92A3063
:102B1000FF2E3246A8BFFF22013300F0B4869DF895
:102B20002C30002B14BF3C233E23FE2ECCBF4FF095
:102B300007094FF005098DF81A30BDF828308DF8D7
:102B40001B208DF81C304A46C8BF331206A955F821
:102B50000A0CC4BF8DF81E308DF81D6004F0B1F86A
:102B600006AB994400230DF11B02914540F08E867F
:102B7000002E8DF817300EDD3246089955F80A0CF4
:102B800004F09FF8089B9DF817201E449E4240F0D9
:102B900082868DF8172055F80A0C01220DF11701D5
:102BA00004F08FF855F80A0C03685B6A03B1984784
:102BB000002305F8023C002C3FF477AD55F80A0CD1
:102BC0000CF0A2F855F80A0CA0476EE50B227449E8
:102BD00030460DF025FF0822724930460DF020FFE7
:102BE000072271493DE7714B6C4A1B88DFF8F4A15D
:102BF000FF2BA8BFFF23511C0891DAF808101370AF
:102C000081F3100189B230460DF028FF684B304641
:102C100019880DF023FFDAF8001001F30F0189B2D3
:102C200030460DF01BFF57E7624B304619680DF038
:102C300001FF614B304619680DF0FCFE5F4B1968CF
:102C400030460DF0F7FE47E75D4BF8E75D4BF6E7E2
:102C50004FF00A0A4FF6FF7B5B4B5C4A1B780B3B3D
:102C60005FFA83F94C45BFF6EDAE1168936859459C
:102C7000A8BF59460898029321EAE171431C0893C2
:102C800089B280F800A0304603920DF0E7FE029B67
:102C900030460AFB03F15945A8BF594621EAE171C4
:102CA00089B20DF0DBFE0134039ADBE70A223B4BCD
:102CB000DFF82CA19A70BAF800101A1D83F8009062
:102CC00083F801E083F80390304608920DF0C6FEC9
:102CD000BAF80210A4E7314A134603F8024B0893EE
:102CE0005470F9E60C9B0D9A9A420FBF01465A1C8C
:102CF0000C921978364A30460FF0B0F84FF00109BF
:102D000019F1020F40F0EA820D990C9BBAF1290FDC
:102D1000A1EB030468D0BAF1390F2AD0BAF1210F20
:102D20007BD15A1C0C921A462A4C12F8021B10A88E
:102D30000C9261705A782270DA1C40F8102D9B7842
:102D4000A3700DF05DFE0C9B20815A1C0C921A465C
:102D500012F8021B61710C925B78A37154E00C9B1A
:102D60000D9A9A421DBF5A1C0C92197801461A4AB4
:102D7000C1E75A1C0C921A780A2A40F0CC859A1C9A
:102D80000C925978154A1170D91C0C919978517090
:102D9000191D0C91DB78937036E000BF16310020CE
:102DA000639701085A97010850970108B41500204D
:102DB00064130020E8F7FF1FECF7FF1FF0F7FF1F79
:102DC000C01D0020D01D0020A0150020E01800200C
:102DD000151E01086E130020E11B0108000D0020E4
:102DE000040D0020BC1500205A1C10AC44F8102D16
:102DF0001B7820460A2B0AD10DF002FEBC4E308013
:102E000020460DF0FDFD70804FF0010966E20DF0E7
:102E1000F7FD20460DF0F4FDF6E7BAF1610F00F082
:102E2000B58300F23081BAF1370F00F0CC8470D84E
:102E3000BAF12B0F00F0E88320D8BAF1230F00F08D
:102E4000658206D8BAF10B0F00F005854FF0FF3907
:102E500044E2BAF1250F00F0C683BAF1270FF5D18D
:102E60000CA80DF0CDFDA34C60650CA80DF0C8FDBD
:102E7000A0650CA80DF0C4FDE065C5E7BAF1310FFF
:102E800000F0C5841ED8BAF12D0F00F0D083BAF13E
:102E90002F0FDBD1984C04F140060CA80DF0B0FDCB
:102EA0000C9BA4F880005A1C0C921A4612F8021BC4
:102EB000043484F87E100C925B7884F87F30A6424C
:102EC000EBD1A1E7BAF1330F00F06A84BAF1350F04
:102ED000BCD15A1C0C921A780E2AB7D8991C0C91A6
:102EE0005C78032CB2D806215143844842185471AF
:102EF000DC1C0C949C784454191D0C91D9785170A9
:102F0000197991705979D170D91D0C919B791371F0
:102F10007AE7BAF14C0F00F0E08334D8BAF13E0FF3
:102F200000F0E98104D8BAF13C0F3FF46DAF8DE7B2
:102F3000BAF1410F00F03B84BAF1430F86D10CA8DF
:102F40000DF069FD00236E4C0CA823600DF042FDCE
:102F5000236818430C9B20605A1C0C921A78694B0A
:102F60000CA81A720DF04CFD624C60650CA80DF0B7
:102F700047FDA0650CA80DF043FDE0650CA80DF021
:102F80003FFD0CA846E7BAF15B0F00F06A8221D83A
:102F9000BAF14E0F00F0E083BAF1510F7FF456AF53
:102FA000594A1278012A3FF62FAF5A1C0C921A4642
:102FB000564C12F8020BA070D81C0C92091A5A78C1
:102FC00001290C909E7840F306830CA80DF018FDA3
:102FD000208019E7BAF15D0F00F08182BAF15F0F2E
:102FE0007FF434AF0CA80DF00BFD0CA80DF008FD1C
:102FF0000CA80DF005FD0CA80DF00DFD0C9B444C2C
:10300000591C0C911946226811F8020B82F82C0009
:103010000C9159780CA882F83610D91C0C919B7829
:1030200082F837300DF0F7FC0CA80DF0F4FC0CA87A
:103030000DF0F1FC0CA826680DF0E2FC70870CA8DE
:1030400026680DF0DDFC0C9B0D9A3087D21A012A00
:1030500008DD591C0C9122681B780CA882F82E30D0
:103060000DF0D9FC0C9A0D9B9B1A032B09DD0CA8C3
:1030700026680DF0C5FC70860CA826680DF0C0FC13
:10308000B086206869E0BAF1D40F3FF4BDAE00F21B
:103090008B80BAF1CC0F00F0518161D8BAF1B90F31
:1030A00000F0AB8238D8BAF1B70F7FF4CFAE5A1C1C
:1030B0000C921A4612F8029B0C92DA1C58780C9269
:1030C0009978B9F1000F40F0F08001283FF69CAEEE
:1030D00001293FF699AE81423FF496AE4E220D4B48
:1030E00002FB013102FB003012F092F98CE600BFC6
:1030F000040D0020140E0020841100207C1E0020EE
:10310000C01D002080170020FE150020702F002019
:1031100074170020422B0020BAF1C80F3FF474AEA0
:10312000BAF1CA0F7FF492AEBC4B1868034600F1A7
:103130001E040C9A0333511C0C91114611F8026BBA
:1031400003F8036C0C91517803F8021CD11C0C910C
:10315000927803F8012CA342EBD10CF087F953E6E7
:10316000BAF1D00F00F0238211D8BAF1CD0F00F0E0
:103170002982BAF1CE0F7FF469AE3B78DA073FF5CA
:1031800043AEA74A137843F0040313703CE6BAF148
:10319000D20F73D0BAF1D30F7FF458AE0CA80DF054
:1031A0002FFCA04B18802FE6BAF1DD0F00F0428310
:1031B00032D8BAF1DA0F00F01B8114D8BAF1D60F69
:1031C0004BD0BAF1D90F7FF441AE0CA80DF018FC2A
:1031D000954C20800CA80DF013FC60800CA80DF01D
:1031E0000FFCA08010E6BAF1DB0F00F03581BAF1D8
:1031F000DC0F7FF42BAE5A1C0C921A4612F8020B0D
:103200008A490C9208708A4A59789170DA1C0C929B
:103210009A78884B9A70F7E5BAF1EF0F61D00FD822
:10322000BAF1DE0F00F0D680BAF1E00F7FF40EAEF7
:103230000CA80DF0E5FB00EB800040007D4BB1E7F2
:10324000BAF1F20F3FF4E0ADBAF1FA0F7FF4FEAD40
:103250003B78DB073FF5FAADAFE10024764EDFF8AF
:10326000F09133789C42BFF6CFAD0CA80DF0C8FBAF
:103270000FF062FC49F824000134F2E75A1C0C926A
:103280001878060609D43B78DC073FF5BDAD032866
:1032900028BF002009F038FCB6E500F07F000328C5
:1032A00028BF002005F03CFFAEE5B9F1010F7FF427
:1032B000ABAD01283FF6A8AD01293FF6A5AD81428F
:1032C0003FF4A2AD0C235D4A584303FB01210B6878
:1032D000841883504B6863608B68A3600024FFF7F9
:1032E000FBBB0CA80DF08CFB514CE0810CA80DF041
:1032F00087FBA08188E55A1C0C921A46504912F8A7
:10330000020B88700C925B784B707DE55A1C0C9216
:10331000197813293FF69AAD9A1C0C920C260022BC
:103320005C78DFF830E106FB02E090F808C0A445C5
:1033300000F0FC820132252AF5D187E5092C7FF7C0
:1033400085AD5A1C0C921A463E4E12F8021B346888
:1033500021700C9200225B78601DA370022A14BFBA
:103360004FF0640E4FF0FF0E0C9B0132591C0C9174
:1033700019787145A8BF7146032A00F8011BEDD1E9
:103380009A1C0C925A7810A8642AA8BF6422227250
:10339000DA1C0C929A78E2701A1D40F8102DDB7836
:1033A00023710DF02DFB0D9B0C9A6081991A002959
:1033B00004DD501C0C90316812784A720C9A9B1AEA
:1033C000002B04DD511C0C91336812785A700EF0FA
:1033D00073F819E50CA80DF013FB1B4CA0810CA889
:1033E0000DF00EFBE0810CA80DF00AFB20820BE52E
:1033F00019465A1C0C9211F8020B144A0C91597878
:103400001070517010A8D91C40F8101D9B78937053
:103410000DF0F6FA044BD880F6E400BF74170020D4
:103420000C1500203A0C0020902F0020E8220020EC
:10343000361B0020601B0020A0150020080D002076
:103440002C0D0020982F0020041600203C0C00209A
:1034500054190020008F0108B04B4E22B049186863
:1034600042E65A1C0C921A46AE4C12F8021BAE4EA3
:103470000C92A1705978AD4A0DF140091170DA1C17
:103480000C929A7832711A1D49F8102DDB78484653
:10349000042BA8BF0423B3700DF0B2FA0C9A0D9B55
:1034A00030809B1A012B03DD48460DF0A9FA70818C
:1034B0000C9B0D9A9A4206D05A1C0C921B78003332
:1034C00018BF0123E37109F0E1FB0C9B0D9A9A42AE
:1034D0003FF49AAC5A1C0C921B78F37094E45A1C7B
:1034E00010AC44F8102D1B788C4EDFF83892204633
:1034F00089F80530D6F800A00DF082FAAAF820006D
:103500002046D6F800A00DF07BFA0C9A0D9BAAF885
:103510001E009B1A072B17DD20460DF071FAA9F843
:103520000A0020460DF06CFAA9F80C002046D6F8E7
:1035300000A00DF065FAAAF822002046D6F800A0F7
:103540000DF05EFAAAF824000C9A0D9B9B1A032B2F
:1035500009DD20460DF054FAA9F80E0020460DF0C2
:103560004FFAA9F810000C9B0D9AD21A002A05DD1B
:10357000591C0C9132681B7882F8263009F086FBC2
:103580000AF0BAFE30680CF041F83DE45A1C0C9287
:103590001A46674912F8020B0C92C8705978654AAE
:1035A0005171DA1C0C929A78634BDA702CE43B78F8
:1035B000D8073FF529AC09F0B9FD09F0BBFA09F0CD
:1035C000F7FB21E43B78D9073FF51EAC4FF4C872F6
:1035D0005A4B1A8018E45A4BB3F90030534393FB0B
:1035E000F6F3238010E40023564C0CA823600DF062
:1035F000F1F923681843206006E40023524C0CA81C
:1036000023600DF0E7F9F6E70CA80DF004FA0C9B27
:103610000D9AD21A002A7FF7F7AB5A1C0C921B782E
:103620004A4A003318BF01235370FFF7EDBB5A1C01
:1036300010AC44F8102D1B78454E204633720DF027
:10364000DFF9B08320460DF0DBF9308320460DF022
:10365000D7F90C9B70835A1C0C921B78F3740D9B4A
:103660009B1A032B07DD20460DF0CAF9B0842046D3
:103670000DF0C6F9F0840C9B0D9AD21A032A0DDDC9
:103680005A1C0C921A4612F8021B2046B1770C9273
:103690005B7886F820300DF0B3F970840C9B0D9A9E
:1036A000D21A052A0CDD5A1C0C921B782046F372A4
:1036B0000DF090F90C9BF0605A1C0C921B7833743F
:1036C0000C9B0D9AD21A002A7FF79EAB5A1C0C92C3
:1036D0001B7886F82130FFF797BB5A1C0C921A46CC
:1036E0001C4C12F8021B10AE46F8102D21715B78AD
:1036F000304663710DF084F90C9B20805A1C0C92AB
:103700001B783046A3710DF07BF90C9B60805A1C2E
:103710000C921B78E371FFF777BB00BF7417002092
:10372000A4940108E8220020041600208922002029
:10373000361B0020E2140020601B002040190020EE
:103740007E2F0020C01D0020D01D002078170020F3
:1037500080170020482A00205A1C0C921C78112C3B
:103760003FF674AB9A1C10A840F8102D5B78A34E5E
:1037700006F814300DF044F940F6CA039842A8BF89
:10378000184640F2EE239842B8BF18461923A0F21B
:10379000EE2090FBF3F006EB44046070FFF734BBBF
:1037A0005A1C0C921A78964B5A75FFF72DBB0023C2
:1037B00093490C9A501C0C9012785A540133082BE0
:1037C000F7D1FFF721BB4FF00709B4FBF9F9C9EBBB
:1037D000C903E41A7FF43AABDFF844A25FFA89F92F
:1037E0000AF1080BE3B299453FF40EAB0C9B5A1C4F
:1037F0000C9293F900309AF902209A4200F0B180BD
:103800009AF90A209A427FF421AB5E46AAE05A1C3C
:103810000C921E781F2E3FF619AB052C7FF416ABC9
:103820000CA80DF0D7F8774B43F826000CF02AFDD2
:10383000FFF7EABA5A1C0C921A4612F8020B0C92C5
:10384000DA1C59780C929A7804F0C6F900287FF4B3
:10385000DBAAFFF7FBBA002111226B4814F009FA2A
:10386000102C4FF0000328BF10246749A342BFF477
:10387000CBAA0C9A501C0C9012785A540133F5E7DD
:10388000624CFFF729B92123FFF74FB912F8011B4A
:103890004B40FFF76AB913F8011B4A40FFF776B9AE
:1038A000012C1BD1102200210CA814F0E2F915F80C
:1038B000053C0C952B440D9315F8033C6E2BADF88D
:1038C00038300BD10CA80DF0A6F80CA80DF098F824
:1038D0000CA80DF095F80CA80DF092F80024FFF755
:1038E00067B94B4C55F80A0C03F0E5F900283EF493
:1038F000DCAE55F80A0C03F0DBF915F8023C06467D
:10390000002B7EF4DAAE24287EF48EAF012305F876
:10391000023CFEF7E3BE0CA80DF07DF80CA80DF0FC
:103920007AF80CA80DF077F8FFF76EBA394A0078EC
:1039300002F82100D81C0C90987802EB81011A1D26
:1039400048700C92DA7800208A705A1D0C921B790C
:10395000CB700DF027FD304B80F001001870FFF7A1
:1039600053BA5646B3700CA80DF04AF80C9B308041
:103970005A1C0C921A4612F8021B01340C92F17078
:103980005A783271DA1C0C929A78B2711A1D0C9224
:10399000DB78737126E70C283EF43FAE0A2801D08D
:1039A0000D2820D10DF0FBFB2321284614F087F9C8
:1039B00008B1401B206000222368002B7EF438AE43
:1039C00002B1236080220021284614F052F9019BA5
:1039D0001B78002B7EF424AEFEF719BE7F287EF400
:1039E00048AEFEF7ACBD7F287EF440AE0022013B1E
:1039F0002360EA540948FEF714BE00BF5D22002090
:103A000080170020841100203B1F002059CA0008A5
:103A10000400FA05DC1D0020000000205A9C01086B
:103A2000A2250020000000002DE9F0435A2885B0AF
:103A300005460C4600F0C08400F2C180362800F034
:103A400021845CD82C2800F0988310D8222800F01C
:103A5000728304D80A2800F0F482002068E3262844
:103A600000F013832A28F8D1754B19781AE330280F
:103A700000F01C8419D82E28EFD1724D05F14006B4
:103A8000B5F8801020460CF0E9FF236895F88220F5
:103A9000591C21601A70236895F883200435591C3D
:103AA000B54221601A70EBD1C5E2322800F0A48340
:103AB0003428D2D1644B03F15A0122685879551C3D
:103AC0002560107022681878551C256010702268D7
:103AD0005878551C2560107022689878551C256010
:103AE00010702268D878551C2560107022681879EB
:103AF0000633551C8B4225601070DED19BE24228B4
:103B000000F07D8312D83B2800F00D8303D83A28BB
:103B1000A3D100215CE13D2800F0C28240289CD165
:103B200008224A4920460CF07BFF84E24D2800F031
:103B3000F1811ED8462800F008844B288DD1444DD1
:103B40000B682A79591C21601A7023686A79591CFC
:103B500021601A70298820460CF080FF2368AA791A
:103B6000591C21601A70698820460CF077FFEA79A9
:103B7000D4E24F2800F0F88350287FF46EAF01257F
:103B80000B68344E5A1C0A601D700B68B2785919C4
:103B900021601A700CF04AFE338858432E4BB3F95B
:103BA000003090FBF3F023685A19226018700CF073
:103BB0003DFE23685A1922601870318834E16F285D
:103BC00000F0758200F23481662800F0008200F275
:103BD00003815E2800F0218444D85C287FF43DAF47
:103BE0001E4E0B6872791E4D591C21601A702B688D
:103BF0002046198C0CF032FF2B682046D98B0CF034
:103C00002DFF718920460CF029FFB18920460CF068
:103C100025FF2B682046598C0CF020FF2B6820468E
:103C2000998C0CF01BFFF18920460CF017FF318AAC
:103C300020460CF013FF2B6893F826206EE200BF9D
:103C400078170020841100207C1E0020801700209F
:103C5000482A0020702F00207E2F0020E82200201C
:103C600074170020602800F0288465287FF4F5AEE2
:103C700000264FF6FF78B84FDFF82C930096019698
:103C800002960396F1574B1C0BD048FA06F3D8075F
:103C900007D5B9F800303341DA0702D502A80DF094
:103CA0005CF901360B2EEDD100260FF2A429D9E9DB
:103CB00000893246404649460EF0DAF9002100F00C
:103CC000010050EA010307D0F0B20DF0A5FB18B1D6
:103CD000314602A80DF041F90136252EE9D1002721
:103CE0003E469E4BDFF8C4821B78DB0742BF029B37
:103CF00043F001030293394640460DF03AF948B1CA
:103D0000394602A80DF035F918B1314668460DF074
:103D100024F901360137252FEDD1914B2046B3F818
:103D200050100CF09BFE8F4B204619888E4F89B2A5
:103D30000CF094FE8D4B204619684A01C1F34003F4
:103D400002F020021343C1F3800243EA4203C1F3AD
:103D5000C00243EA8203C1F3401243EAC20301F006
:103D6000100119430CF07AFE0422694620460CF03B
:103D700057FE23683A78591C21601A707C4B204604
:103D800019886429A8BF64210CF068FE962D40F0C4
:103D9000198123685A1C226003221A7023687A78DA
:103DA000591C21601A700822193E96FBF2F2236812
:103DB00082F30402591C216020461A7001A90CF0FC
:103DC0002FFE23685A1C226010221A70694B198832
:103DD00020460CF02FFE2EE1692800F08D8016D8C9
:103DE00068287FF43AAE0025634E644F032D06D851
:103DF000182303FB05635B7C002B40F0308100211E
:103E0000204601350CF02AFE082DEFD113E16C2875
:103E100000F02B816D287FF420AE594B20461968A5
:103E20000CF008FE574B198820460CF017FE02E1F3
:103E30007E2800F0B2823DD8752800F0B98020D8E5
:103E400070287FF40AAE00214F48036801EB41025D
:103E50009D5C236801315E1C26601D7003680A2981
:103E600013445D78236803F1010626601D70036822
:103E700013449A78236803F1010525601A70E4D190
:103E8000D9E07C2800F07E827D287FF4E6AD3F4BB0
:103E900022681978501C2060117022685978501CD3
:103EA000206011709A782368591C21601A70384B71
:103EB000D988B9E7852800F05C8110D87F2800F008
:103EC000008283287FF4C9AD324D2046A9890CF0C9
:103ED000C5FDE98920460CF0C1FD298AA4E7962892
:103EE0003FF4C6AEF0287FF4B8AD2B4D2046E989EB
:103EF0000CF0B4FDA98997E70025284E284F3378A8
:103F00009D4280F2988037F8151020460CF0A6FDEF
:103F10000135F4E70025214F224E3B789D4280F287
:103F20008A80236816F81510581C06EB450220609D
:103F300019705178204601EB810101EB810101F2FA
:103F4000EE2189B20CF08AFD0135E6E7AFF300807F
:103F500090E33FF4080000003C81010804130020B6
:103F600034000020861C0020241C00207017002034
:103F70008A1C0020A41300206C190020A415002026
:103F8000680C002034100020741700203C0C002026
:103F9000902F002004160020361B00207C210020DA
:103FA0003C1300205D220020661300200831002011
:103FB000A54A12F8013F002B3DD02168481C206023
:103FC0000B70F6E7002120460CF048FDEBE69F4E13
:103FD000B28AB2F5006F30D8B2F5806F2FD8B2F543
:103FE000007F2CBF0227012700257319996B2046FB
:103FF00091FBF7F1043589B20CF030FD0C2DF4D1B2
:104000000125934E934F396A56F825000EF0A0FE15
:1040100011F064FB013581B220460CF01FFD042D28
:10402000F1D100258C4E36F82510204601350CF0D4
:1040300015FD032DF7D101207AE00827D4E70427E6
:10404000D2E786480EF00CF8002384498342F2DA66
:1040500022685D5C561C266001331570F6E757F840
:1040600025000EF0C3FF81B2CAE67D4D20462988A7
:104070000CF0F4FC698820460CF0F0FCB5F9041053
:104080000A2391FBF3F189B2CEE6764D20462988CA
:104090000CF0E4FCA98820460CF0E0FC2989C3E67A
:1040A000714B99782268501C2060117035E06F4D7B
:1040B0002B681A780B68591C21601A702B689A7843
:1040C0002368591C21601A7000232A681A44517908
:1040D00022680133501C032B20601170F5D12B682E
:1040E00020461A7A2368591C21601A702B68DA78E6
:1040F0002368591C21601A702B681A792368591C8F
:1041000021601A702B6859890CF0A8FC2B685A7A28
:104110002368591C21601A702B685A782368591C2F
:1041200021601A7087E701200B685A1C0A6018701A
:1041300005B0BDE8F0834E4D05F1500628780DF02E
:104140007AFE2368027A591C21601A7023686A7803
:10415000591C21601A702368AA78591C21601A70B2
:104160002368EA780435591CAE4221601A70E5D103
:1041700061E7404BB3F9001082E73F4D0B682A7AA4
:10418000591C21601A70A98B20460CF067FC298B02
:1041900020460CF063FC698B20460CF05FFC236822
:1041A000EA7C591C21601A70A98C20460CF056FC40
:1041B000E98C20460CF052FC2368AA7F591C216030
:1041C0001A70236895F82020591C21601A70698C98
:1041D00020460CF043FC2368EA7A591C21601A70CF
:1041E000E96820460CF026FC23682A7C591C2160D3
:1041F0001A7095F8212091E71F4B5A7D8EE71F4BCF
:1042000020461A780B68174D591C21601A701C4BF8
:1042100019680CF00FFC184B20461A7A2368591CB9
:1042200021601A7029880CF019FCA98820460CF02E
:1042300015FC298920460CF011FC002120460CF0C9
:104240000DFC0021F0E500BF0B81010840150020A6
:1042500080250020FC220020881500203B1F002024
:104260001C2A0020680E00202C0D0020982F002012
:10427000DC1D0020601B0020801700207817002024
:10428000C01D0020A34DA44E05F1100795F9023082
:1042900096F906209A4200F01F8196F90E209A4264
:1042A00000F01A810835AF42F0D1C4E600259B4EDC
:1042B00056F82510204601350CF0BCFB202DF7D117
:1042C000B9E6964D002306272846002107FB03F692
:1042D000226802F1010EC4F800E01370226802F1B6
:1042E000010EC4F800E011708A192A4492F8C0E067
:1042F0002268013102F1010C0629C4F800C082F8DD
:1043000000E0E5D10133062BDFD1002221684D1CEE
:1043100025600B7021684D1C25600A70811891F88A
:10432000E450216801324E1C0B2A26600D70EDD13D
:1043300023685A1C226007221A7023685A1C2260C4
:1043400000221A7090F8F020E8E600250B6820465D
:104350005A1C0A601D7029460CF06CFB2946204649
:104360000CF068FB294633E500250B685A1C0A60EF
:104370001D700B685A1C0A601D700B685A1C0A607D
:104380001D70EBE7664D204629880CF067FB6988B5
:1043900020460CF063FBA98846E5624B1A780B684F
:1043A000591C21601A70604B9A782368591C21604F
:1043B0001A705E4B9A78B1E65A4E0B68F27812B3D7
:1043C0005A1C0A6008221A700B685A1C0A600122E3
:1043D0001A70574D23682A79591C21601A70236876
:1043E000AA78591C21601A70298820460CF036FBE7
:1043F000698920460CF032FB2368F279591C216050
:104400001A70EA788AE6B278591C21601A70494B12
:104410001A782368591C2160DAE70026002120461B
:104420000CF01CFB002120460CF018FB002120465C
:104430000CF014FB2368404D5A1C22601E702B6840
:10444000204693F82C202368591C21601A702B6891
:1044500093F836202368591C21601A702B6893F852
:1044600037202368591C21601A7023685A1C226067
:104470001E7023685A1C22601E7023685A1C22601A
:104480001E702B68598F0CF0E9FA2B682046198FA3
:104490000CF0E4FA2B68204693F82E202368591C70
:1044A00021601A7023685A1C22601E702B68598E76
:1044B0000CF0D4FA2B68998EB6E41B4BDA780B68B3
:1044C000591C21601A701D4B5A792368591C2160B0
:1044D0001A70164BDA7821E622682046511C2160BA
:1044E000137029880CF0BAFA2368EA78591C216005
:1044F0001A7023682A79591C21601A702368AA79D6
:10450000591C21601A7023686A79591C21601A703D
:10451000C8E600BFA22500209025002084110020BD
:10452000902F0020E8220020361B0020601B002076
:10453000041600208922002074170020E2140020B5
:104540002DE9F04F00F59C43A44A20331360A44B9F
:104550008BB01D788046002D65D1A24EA24F344607
:1045600096F824309D42C0F2BF8042F201014FF420
:104570007A799E4AB8FBF9F912680A4001929C4A7E
:1045800006D09C49097811709B4908789B490870AE
:1045900017781FB1994A177887F001070F22032077
:1045A00084F82520904A94F826A0918CD28C00247F
:1045B0000392BAFBF0F202EB4202AAEB0202D2B281
:1045C0008F4D0492DFF84CB209F596720291A5F175
:1045D0002806059206909C42C0F2AE80814D894E1D
:1045E00095F82530884C0F2B0CBF01220022874BF9
:1045F0001A7040F023811B200CF00EFF002840F0C1
:104600001D813368E268A3609B1AC82B05D901237A
:10461000042084F821300AF0CBFE95F826300133CF
:1046200085F8263005E07A4A1268904201D9013DAA
:104630001D706E4B1A68029312F4805F05D0002043
:104640000CF0EAFE08B904F05FFA674A537D019264
:10465000E3B1704A013B32F91300634BDB7D1BB1C0
:10466000C0F53B60083000B2A0F57A70B0F57A7FF3
:10467000A8BF4FF47A7020EAE0700EF061FA664944
:104680000EF0B2FA0EF0B2FC644B1880644B5E4C34
:10469000984503D9A3780BB90123A370A378DFF859
:1046A00094B1002B00F026811B200CF0B5FE94F88D
:1046B00021709BF80050012F05F00109824608BFC8
:1046C0000025504EDFF8708118BF05F0020594F800
:1046D0002030052B00F20A81DFE813F0D0002F0113
:1046E0003A01590164017A014E48072DD4BFE95DB2
:1046F000E9B243689847032D1ADCC8B14A4B33F836
:10470000252003EB8501831A4FF47A7058434B88B8
:104710009B1A90FBF3F040F6CA0300F57A709842BA
:10472000A8BF184640F2EE239842B8BF184680B2A0
:1047300024F81500013513E74FEA440EB7B136F9F6
:104740001400029A80B2904202D3039A904220D978
:10475000364A52F8240081450AD23BF80E00019AED
:10476000E2B92BF814000635013434E73846E8E79F
:10477000E0B2079309F030FC032C079BEFDC012229
:1047800096F825C002FA04FE2CEA0E0E86F825E003
:10479000E5E7059A254941F82420E0E7049A96F8D0
:1047A000B8E025F81200BEF1000F06D1BAF1020FF1
:1047B000D7D94FF0010286F8B820B5F800E0688834
:1047C0001B4A7044B5F804E0704400B222F81400AB
:1047D000069A90FBF2F080B2C3E700BF8821002068
:1047E00088220020840E0020801700207C170020E3
:1047F00005130020582100203C0400203D04002027
:10480000AC0E0020C4130020801300200D150020E2
:10481000842200203C130020AAF1823F6413002070
:10482000404B4C007C210020AA220020F40E0020E6
:104830003E0F002004130020482A002001236E4A66
:10484000042013706D4A6E4F13700AF0B9FD33687F
:10485000A268E3609B1A626895F82460934284BF63
:10486000002384F821300024B442BFF6D6AEE0B273
:1048700009F0B2FB27F814000134F5E7B9F1000F95
:104880002BD00CF0DDFD012806D164213268B8F888
:10489000023001FB03232361BAF1000F0BD098F81B
:1048A000063043B10BF074FC032384F820304FF43E
:1048B0007A73E3610BE7012F18D0336822699A42BB
:1048C00007D20BF065FC032384F8203040F6B833A0
:1048D000EFE7012384F82030F9E64FF48060BAF165
:1048E000000F27D00AF056FD0023236115B128469A
:1048F0000AF080FC0CF0A4FD06460CF093FD414D3F
:10490000002800F087809BF80030D80740F18280B3
:10491000019B588C0EF014F93B4B0146D8680EF001
:1049200015FB002800F00F810122384B83F8D220BC
:10493000012381E00AF01EFDD6E7012F01D10523F6
:10494000C8E798F80730012BBBD00BF021FCBEE67E
:10495000012F04BF052384F82030B9F1000F0AD0DD
:104960000325019BB3F91820254B1A805A809A80A1
:10497000B8F80020DA80336862699A4202D3B9F14C
:10498000000F35D147F23053E3610323A2E7022041
:104990000AF016FD04F0B8F83268E3691344A36125
:1049A000042397E7012F0ED13368A2699A429DD262
:1049B000174B187818B90CF02FFD002896D102205B
:1049C0000AF0F6FCBBE73268E3691344A3618DE7A4
:1049D00064213268B8F802304FF4806001FB032391
:1049E0002361002384F82030E3700AF0C3FC6EE6F4
:1049F000012F3FF46CAE79E73C0400203D04002019
:104A00003C1300205C0D002008130020840E0020C1
:104A10000000002000226D4B83F8D220002E87D1A9
:104A200000226B4B1A605A609A606A4B1B6893F8BD
:104A30002D30002B7FF47CAF2B709BF80030D90712
:104A400024D5029B1B68DA0620D5634A1278D70664
:104A50001CD4DD041AD40CF0E5FCB8B95F4B5B4DF7
:104A60001B78002B00F08A805D4B9B78002E74D160
:104A7000002B00F085805B4B1A685B4B1B689B1A10
:104A8000002B7DDA04F040F885F8D3600022019B0A
:104A900056495D8B9F8B134631F912009B08A84243
:104AA000C4BF63F07F03DBB20132B842B8BF43F04A
:104AB0004003042AF0D1454D95F8D4209A4266D19E
:104AC0004B4AB5F9D6001268D1694A4A91FBF2F215
:104AD00002F5FF427F32904206DC4FF47A7291FB7E
:104AE000F2F10144A5F8D6103C4A85F8D430177885
:104AF000002F40F0828138460CF08EFC00284CD00C
:104B000085F8D97004F000F99BF80030DA077FD4FB
:104B100095F8D80000287BD1B5F9D630322B77DD57
:104B2000012295F8D43085F8D820572B40F0A38186
:104B3000314805F0BFF9314B1B685B0768D50A2285
:104B40002F4B1A8064E0002E7FF4F2AE1F4B93F8D7
:104B5000D230002B7FF4ECAE62E73BB14FF47A71B8
:104B6000204A126801FB03231F4A136095F8D330D3
:104B7000002B8BD00AF024FB002305E0002EF5D19A
:104B800010200AF037FB012385F8D3307EE700229E
:104B9000A5F8D62085F8D820A6E71A4B18609BF810
:104BA0000030D807B4D5184B1B788BB3E3787BBBA8
:104BB00095F8D9300133DBB2032B85F8D93027D9EA
:104BC000074B5B7813B303F09FFF9DE7840E002033
:104BD00028150020741700200C150020000000206C
:104BE0002C0D0020C4130020481900203C13002085
:104BF000901F002018FCFFFFB0230020701700203A
:104C00003E1900204C19002005130020002EDAD098
:104C1000029B1B685E0728D595F8DC309BB19BF89A
:104C20000030D8070FD5BC4BB3F90620019B5B8B36
:104C30009A4208DD00200CF0EFFB20B9322385F802
:104C4000DC00A5F8DE3011200CF0E6FB002800F0B7
:104C50008D8195F8E0302BB995F8DA3013B932230D
:104C6000A5F8DE30012385F8E0300023AB4D08AE17
:104C7000089305F150077360294615F8010C0CF0F4
:104C8000A5FB30B115F8021C242902D830460CF0DF
:104C900064F90435AF42EFD1A14B96E8030083E8F5
:104CA0000300A04B1E78002E00F0708101200CF054
:104CB000B3FB9D4E9D4D18B9E378002B00F068833F
:104CC00033689A0740F164832C8814F0010440F0A3
:104CD000648301200AF05EFB02200CF09DFB00289B
:104CE00000F05D83002C00F05A8301200AF042FBA3
:104CF0002B889B0702D402200AF04CFB2988012054
:104D000011F0030118BF012102F082F824200CF0F9
:104D100083FB38B99BF800305F0744BF23F00403DE
:104D20008BF80030336813F00A0F2BD005200CF0FD
:104D300073FB002800F037832B885C070AD404201B
:104D40000AF028FB0A227A4BB3F9043093FBF2F302
:104D5000784A138006200CF05FFB002800F02783C0
:104D60002B88580602D440200AF014FB07200CF0D0
:104D700053FB38B10A226E4BB3F9043093FBF2F3C4
:104D80006D4A13800C200CF047FB002800F01383C1
:104D90004FF480700AF0FEFA684B1B78082B01D0A4
:104DA0000E2B02D140200AF0E5FA029B1B68590540
:104DB0000FD5634B1B79002B40F002839BF800302A
:104DC000DA0740F103833C2009F00CFC002840F096
:104DD000028301225B4B1A7003F0B0FE33685B075D
:104DE00008D503200CF018FB002840F0FA820820B8
:104DF0000AF0C0FA0BB0BDE8F08F5F2B20D1B5F9F7
:104E0000D630B3F5FA7FFFF603AF95F8D830002B14
:104E10007FF4FEAE012385F8D8309BF8003013F004
:104E2000010602D003F070FEF2E60F200AF0E2F96C
:104E3000B5F8D63085F8D860FA3BA5F8D630E7E665
:104E40006F2B7FF461AEB5F9D630B3F5FA7FFFF67C
:104E5000DFAE95F8D830002B7FF4DAAE012285F86A
:104E6000D8209BF80020D10702D403F04DFFCFE6F5
:104E7000354A1360CCE6029909684F0716D55A2BBC
:104E800014D195F8DA3023B185F8DA0085F8DB2003
:104E9000BEE695F8DC3083F0010385F8DC301BB109
:104EA0000B200AF0A7F9B3E60C20FAE75D2B00F01F
:104EB000AD825B2B00F0B1825E2B40F0B08203200C
:104EC000A5E2A72B05D1214A137843F00403137000
:104ED0009EE60022BB2B089218D10223ADF82230A7
:104EE0001B4BBDF820109A890A449A81BDF8221004
:104EF000DA890A44DA8108F00FF9B5F8D630FA3BBE
:104F0000A5F8D630002385F8D83081E6B72B21D11B
:104F10004FF6FE73E2E700BF3C130020DE1D0020C9
:104F2000FC140020501A0020701700206613002087
:104F30001C2A00203A0C0020500C0020781700207A
:104F4000C0250020880C00204C1900200C150020E2
:104F5000361B0020BE2B03D10223ADF82030BFE763
:104F6000BD2B7FF455AE4FF6FE73F6E795F8DA30B9
:104F7000002B3FF47AAE9BF8003013F0010302BF20
:104F800085F8DA30012385F8DB306EE64FF00C0A45
:104F90004FF00109BF4DC04F05F15A08294615F8D9
:104FA000010C0CF013FAE0B12979AB780AFB01701F
:104FB000BA4A013B03EB43031344D0F8E82095F8C9
:104FC00003E093420DD0C0F8E83097F8143109FAA5
:104FD00001F123EA010180F8E4E0C0F8EC6087F811
:104FE000141106354545D9D14FF00009AC4BDFF817
:104FF000C0821E68AB4BA8F1E4051B680393AA4B63
:105000001B780493D8F80430002B69D01F78002F48
:1050100066D0D8F8082003998A1A002A0CDB01F51B
:10502000FA72C8F80820012202FA09F195F8142151
:1050300022EA010285F81421049A002A50D098F837
:10504000002059780432D2B2002940F04F819749AC
:1050500031F91210019A128B02F1C80081422ADD47
:1050600093F802A095F8142142FA09F2D10737D437
:10507000BAF1000FCCBF022001200AF063F97A1EBA
:10508000162A40D8DFE812F034004C0056006600C3
:105090007D0084009F00BA00D600E200EE003F00D1
:1050A0006600730084009F00BA009300AE00CA003F
:1050B000FA0016012401C83A914203DA9978C1F145
:1050C000000ACFE7012303FA09F295F8143123EA25
:1050D000020385F81431039B03F5FA73C8F808300E
:1050E00009F10109B9F1040F08F10C088AD1DDE5D5
:1050F000317801205144FA29A8BFFA2121EAE1714F
:1051000031700CF0C5F9D5F818010AF0AFF9012398
:1051100095F8142103FA09F3134385F81431DFE7F6
:10512000B178022051446429A8BF642121EAE171C9
:10513000B170E6E731798A44BAF1640FA8BF4FF045
:10514000640A2AEAEA7A86F804A00CF0B5F9514616
:105150000320D6E7B1790D2051446429A8BF64210A
:1051600021EAE171B1710CF093F90D2FCBD0717977
:105170000E2051446429A8BF642121EAE1717171B4
:10518000BFE7F1790520514481F30801F171B8E7D7
:10519000D5F818210F20D1785144C829A8BFC821BB
:1051A00021EAE171D1700CF073F90F2FABD0D5F873
:1051B0001821122011785144C829A8BFC82121EA1A
:1051C000E17111709DE7D5F8182110201179514433
:1051D000C829A8BFC82121EAE17111710CF058F962
:1051E000102F90D0D5F81821132051785144C82998
:1051F000A8BFC82121EAE171517082E7D5F81821D2
:10520000112051795144C829A8BFC82121EAE17170
:1052100051710CF03DF9112F3FF475AFD5F81821FD
:10522000142091785144C829A8BFC82121EAE1710E
:10523000917066E7D5F81821092091795144C82961
:10524000A8BFC82121EAE17191715AE7D5F8182168
:105250000A20D1795144C829A8BFC82121EAE171A7
:10526000D1714EE7D5F818210B20117A5144C82985
:10527000A8BFC82121EAE171117242E771781520B7
:105280005144B1F5967FA8BF4FF4967121EAE171C0
:10529000717036E77D1E0020840E002047810108D2
:1052A000982F0020C4130020051300203C13002079
:1052B000680F0020D5F81821162092F837105144B5
:1052C000FE29A8BFFE2121EAE17182F8371018E714
:1052D000D5F81821172092F8361051446429A8BF38
:1052E000642121EAE17182F836100AE701297FF48E
:1052F0000EAF524931F9121040F633029142A8BF65
:1053000011469A784FF49663B1F5617FB8BF4FF4B8
:10531000617193FBF2F3A1F561710C2F91FBF3F333
:105320001ED0182F7FF4F3AED9B2C8290B46A8BF00
:10533000C823D5F81821D8B292F817E070453FF489
:10534000E6AEA3EB0E034FF0080E93FBFEF3013322
:10535000DBB2D075384605930CF09AF8059B10E047
:105360005FFA83FA364B5A7852453FF4D0AE504636
:1053700003F0D6FE514638460CF08AF80AF10103D4
:10538000DBB2002B3FF4C3AE184609F0DBFFBEE6EC
:10539000012009F0EFFF01249EE400249CE4022098
:1053A00009F0E8FFAAE4042009F0E4FFD2E4402079
:1053B00009F0E0FFDAE44FF4807009F0DBFFEBE482
:1053C00014200CF029F800287FF4FDAC02F000FB5B
:1053D00009F090FEFDE409F0B1FC3C2009F0CCF8A6
:1053E000F4E42C8814F008047FF404AD082009F0DC
:1053F000D1FF144B1A68144B1A60104BDA88134B08
:105400001A80134B1C60134B1C60F3E4012001381D
:10541000C0B207F079FBFFF7FBBB0220F7E7562B82
:1054200001D107F079FE95F8D430972B7FF449AD80
:105430004FF4C872084BFFF784BB00BF3C13002039
:10544000241C0020680C0020640C0020580C002054
:105450005C0C0020540C002040190020022310B5E1
:105460000168047B0A68A3401A420AD00024054A56
:1054700040681470026822F001021204120C0260EB
:105480004B6010BD1E13002024234343F0B5A14CF4
:10549000A14AE118E3585B689E8AB6B2F5B215F0EE
:1054A000010F4ED01D8825F400652D042D0C1D80A4
:1054B0001D88ADB245F480651D80002515708D7E78
:1054C000002D31D0557815B9C97DFF292CD1012186
:1054D0005170242101FB0041097E022901BF198876
:1054E00089B241F400611980242101FB0041897DCA
:1054F00041F001011982242101FB0041097E92F94A
:10550000005001318D420ED10021517092782AB1A4
:105510009A8822F440721204120C9A80242303FB0E
:10552000004000234375F0BD242101FB00418D7D27
:1055300005F0FE051D82C97DFF29DCD0FF21117019
:10554000D9E7AF0744D5BFF35F8F0D7EEDB2012DD4
:1055500018D1897EB1B15178A1B1198821F4806147
:105560000904090C1980BFF35F8F198B1988957096
:1055700089B241F400711980998889B241F480613F
:105580009980B8E7198BBFF35F8F242101FB00419D
:105590000D7E022D0FD1897E69B1517859B11988DC
:1055A00021F480610904090C1980998821F4806133
:1055B0000904090CE4E7242101FB00410D7E032DC1
:1055C000DAD1897E0029D7D051780029D4D0ECE7F0
:1055D0006F075CD5012595708D7E002D3FD05578E5
:1055E000002D3CD00D7E92F90060022D0F6A1D88BF
:1055F00021D925F480652D042D0C1D80B3F810E011
:10560000F5B25FFA8EFE07F806E01E88B6B246F4E1
:1056100000761E800E6AA91C1170198A0135C9B264
:105620006DB27155998889B241F480619980198869
:10563000C905FCD45FE7ADB245F400751D80B3F831
:1056400010E0F5B25FFA8EFE07F806E00F6A198ADD
:105650006E1C76B2C9B20335B9551570E7E75178BB
:1056600021B9242101FB0041497E41B1198889B249
:1056700041F400711980117801311170D7E7198850
:1056800089B241F48071198001215170CFE715F082
:10569000400521D092F900C0B3F810E00F6A5FFA1C
:1056A0008CF65FFA8EFE751C07F80CE06DB20F7E6B
:1056B000E91C8F42157005D1998821F48061090495
:1056C000090C9980242101FB0041097E8D427FF461
:1056D00012AF023616700EE737067FF50CAF92F95F
:1056E00000707E1C0AD0CE697D1CF65D6DB21E82F4
:1056F000097E1570A9427FF4FEAE56E71570CD7D88
:105700001D828D7E002D7FF450AF097E00297FF42D
:10571000F2AE4AE7DC0B0020A00F002010B5084BCA
:1057200007281B68C8BF14381844007D0C4601F0D8
:10573000F7FA20B12146BDE8104001F03ABB10BD98
:10574000D80B002070B50446C56C8668AB8986B05E
:1057500023F400531B041B0CAB818379617913F094
:10576000020F14BF4FF40052002213F0040F14BFB5
:105770004FF48060002011F0010F14BF04230023B8
:105780008907298A48BF43F0080389B221F44051B0
:1057900011432982AA8922F4B05222F00C02120489
:1057A000120C02431343AB81AA8A01A822F440726F
:1057B0001204120CAA8209F011F8294A039B0499D9
:1057C000954218BF19461922AB894A4313F4004F7A
:1057D00014BF7100B100B2FBF1F16426B1FBF6F326
:1057E000AA891801120406FB13132ED5DA003232EF
:1057F000B2FBF6F202F0070242EA00039BB22B81F1
:10580000A379DB070BD5E36C154A934225D0A2F5AB
:105810007442934203D101200121FFF77FFFA37956
:10582000E26C13F0080F938A0BBF23F008039BB2BE
:105830001B0443F0080308BF1B0C938293899BB29F
:1058400043F40053938106B070BD1B013233B3FBA8
:10585000F6F303F00F030343D0E70020DCE700BFBB
:1058600000380140072838B5D8BF04460B4BC8BFE5
:10587000A0F114041B6805462344187D01F050FA7A
:1058800058B127220134C4718271122101F06AFAE1
:105890002846BDE83840002140E738BDD80B00203D
:1058A0000348D0F8B0300BB1A8301847704700BF9C
:1058B000780300200348D0F894300BB18C3018479F
:1058C000704700BF780300200248836F0BB170302F
:1058D00018477047780300200248C36D0BB154305D
:1058E00018477047780300200248036C0BB138302A
:1058F00018477047780300200248436A0BB11C30F8
:1059000018477047780300200248836803B118479E
:10591000704700BF780300202DE9F04FB0F1FF3F42
:1059200087B0804600F0F880242000FB08F0844B0C
:105930001E581F189946002E00F0EE8014301844AF
:1059400010220021746812F094F9BD6808F1010377
:10595000FF68DBB215B11522EB71AA7117B11622DF
:10596000FB71BA71B07B08F017FCA388284623F4BA
:1059700040731B041B0CA38001F016FA384601F09B
:1059800013FA1621284601F0EDF91621384601F0E8
:10599000E9F94FF0080A4FF0640B25B12B68AA888B
:1059A0009B681A4204D1BBF1000F40F0B88015B1DA
:1059B0002B68AA885A610A2001F0F8F8284601F0FD
:1059C000F3F90A2001F0F2F8BAF1010AE5D117B1B2
:1059D0003B68BA885A610A2001F0E8F815B12B68D3
:1059E000AA885A610A2001F0E1F8284601F0DCF9A2
:1059F0000A2001F0DBF8384601F0D6F928461F21CD
:105A000001F0B0F91F21384601F0ACF94D4B4E4F73
:105A10009C4203F5DE331A6901A80BBF42F4001261
:105A200042F480021A611A610BBF1A691A6922F4E2
:105A3000001222F480021A61A388444A23F44073BE
:105A40001B041B0CA380242303FB089898F8103038
:105A5000002B08BF1746238807EB47079BB243F08C
:105A600001032380A58808F0B9FE039B384825F080
:105A70003F05B3FBF0F02D042D0C0543ADB2A5801E
:105A800021884FF4967221F001010904090CB3FB3F
:105A9000F7F321804FF47A7142439BB2002B92FBC3
:105AA000F1F208BF0123013292B243F40043228491
:105AB000A383238800259BB243F00103238023881E
:105AC00001A823F4816323F002031B041B0C43F49D
:105AD000806323804FF480432381238823F0800355
:105AE0001B041B0C23800124337C8DF805508DF89A
:105AF00004308DF806508DF8074008F06BFBF37BFF
:105B00009DF807208DF804308DF805508DF806506B
:105B10005AB101A808F05EFB07B0BDE8F08F0A207B
:105B200001F044F80BF1FF3B37E75A09094903F04C
:105B30001F0304FA03F3203241F82230ECE700BFE0
:105B4000DC0B00200054004000350C00801A0600D9
:105B500040420F0000E100E0F8B52425214F069CEB
:105B600005FB00756E680EB34900C9B2A975EA75E8
:105B7000012100226A76A9762B7669752A75B38889
:105B80002C629905EC611ED43388DA0516D44FF4E3
:105B9000805433889B050CD5013CFAD1124A1388F6
:105BA00001339BB21380FFF7B7FE00E03446204676
:105BB000F8BD33889BB243F480733380B3889BB2C3
:105BC00043F44073B38024234FF4805403FB0077E5
:105BD0007B7D13B1013CFBD1E0E73C7D84F0010407
:105BE000E5E700BFDC0B0020861C00202423434394
:105BF00073B5244E0546F218F3585C68A38A9BB22D
:105C00000193019B13F4706F1CBF01231375019B5B
:105C100013F4E06F1DD0238BA38823F480631B044F
:105C20001B0CA380019B9B0513D42388980510D4DB
:105C30002388D9051AD52388DA05FCD423889BB29A
:105C400043F40073238023889B05FCD42846FFF788
:105C500063FEA38A23F470631B041B0CA38224231A
:105C600003FB056500236B7502B070BD23889BB2F2
:105C700043F400732380A38823F440731B041B0C9C
:105C8000A380E6E7DC0B002030B4451C03D00228DB
:105C900001DC30BC60E7002030BC704773B5441CA9
:105CA0008DF807302AD0022828DC2423214E03FB5C
:105CB00000635D6815B34900C9B29975DA750021B2
:105CC00001220DF107045A7699761A765A751975DC
:105CD000DC611C62AB8899051DD42B88DA0515D4CC
:105CE0004FF480542B889B050BD5013CFAD1124A06
:105CF000138801339BB21380FFF70EFE002002B021
:105D000070BD2B889BB243F480732B80AB889BB211
:105D100043F44073AB8024234FF4805403FB0066AC
:105D2000737D13B1013CFBD1E1E7307D80F00100D0
:105D3000E5E700BFDC0B0020861C00200120FFF7F8
:105D4000A3BB012052E70020FFF79EBB00204DE7D8
:105D50002DE9F04F85B0814601F03AFECD4B1D781C
:105D6000002D40F0B583CC4F3B685A0540F1B0831D
:105D7000CA4BCB4E1B68002B00F05A81C94C3268CD
:105D80002368D31A7C2B40F253814FF024082379E7
:105D9000DFF848A3013322602371AAF1340B404697
:105DA00001F0FCFD5AF8040F0CF0CAFE0090BBF89D
:105DB00014000CF0C5FE009A014610460CF0C8FF16
:105DC000B9490CF011FF0DF0EBF808F1010800B231
:105DD0005FFA88F808F0C6FEB8F1270FDFD130204F
:105DE00001F0DCFDB4F9080008F0BCFE01F0CEFDC6
:105DF00023799B0734D141F2883322689A421CD917
:105E00004FF06408DFF8D8A2102001F0C7FDDAF8DF
:105E1000000090FBF8F000B208F0A4FE212001F091
:105E2000BDFDDAF8003093FBF8F008FB10300028D5
:105E3000B8BF404200B208F095FE142001F0AEFD5C
:105E40009A4BB3F904000A2390FBF3F008F08AFEA2
:105E50001C2001F0A3FD002008F084FE01F096FD57
:105E60002379580740F0BD80022001F097FD904B48
:105E7000DFF870A2986A6423323090FBF3F000B22E
:105E800008F070FE032001F089FD8A4B1B7813F0A7
:105E9000010F00F087810BF0D3FA874B87498046CA
:105EA000D8680CF0A1FE0DF0A1F880B2B8F1000F97
:105EB00004D13B6813F0100F18BF002000B208F0A7
:105EC00051FE9AF80530002B59D07D4B93F800B065
:105ED000BBF1000F53D04FF064087A4A06201188B6
:105EE000019308FB01B14FEA4B08B1FBF8F1B4F89C
:105EF0000C8000924FEA08181FFA88F848EA012837
:105F00001FFA88F8C1F3032148EA010801F046FDB1
:105F10000FFA88F008F026FEA189009A013189B2B3
:105F200091FBFBF0B2F80080674A0BFB101B517A23
:105F3000A4F80CB00129019B40F03A81392001F00E
:105F40002DFD0FFA88F008F00DFE282001F026FD47
:105F50000A23DFF89481D8F8000090FBF3F000B238
:105F600008F000FE042001F019FDBAF80830002BFB
:105F700000F0478103F0E8F800B208F0F3FD03A950
:105F8000524808F0C5FD132001F008FDBDF90C00D2
:105F900008F0E8FD1B2001F001FDBDF90E0008F03E
:105FA000E1FD232001F0FAFC4E2008F0DBFD03A9FF
:105FB000464808F0ADFD122001F0F0FCBDF90C00E0
:105FC00008F0D0FD1A2001F0E9FCBDF90E0008F040
:105FD000C9FD222001F0E2FC452008F0C3FD01F0DC
:105FE000D5FC2379282B23D1002317202371346873
:105FF00001F0D4FC4EF660204FF03C08B4FBF0F307
:10600000B3FBF8F008FB1030000200B208F0AAFD64
:10601000182001F0C3FC4FF47A70B4FBF0F4B4FB29
:10602000F8F008FB104000B208F09CFD01F0AEFC57
:10603000274B1B78002B00F09E801A4C254A2369C1
:10604000A9EB0303934240F282800023A3752376D9
:106050001C4B1B88DAB21B0A84F8322084F83330D8
:1060600084F8282084F829303268236CD21A164B21
:10607000D97A4FF47A734B439A4237D33368236407
:10608000154B1B78013B012B9FBF1023A3750223E7
:1060900023762BE0501A00207C170020A813002044
:1060A000C41300202C10002000007A441C2A002079
:1060B000C81500200413002008130020CDCC4C3E4E
:1060C000841C0020B4150020C02500208096980074
:1060D000B61300203F0D0300691300207415002043
:1060E000680C00206E130020BC1500200A21874B8D
:1060F000C4F810901A689B6892FBF1F293FBF1F3DD
:10610000642184F834301B1284F83530804B84F8D5
:1061100030201B68121293FBF1F303F5FA739BB264
:1061200084F82E301B0A84F82F30A36884F83120BD
:1061300003F1300284F8362003F5EA4293FBF1F3D1
:1061400030321212783384F8372084F8383094F8DB
:1061500044B0BBF1000F00F04D83E36C5BB194F8E9
:106160004430002B7BD040F6B732636DA9EB0303BC
:10617000934200F2A48033680093664B1B78002B97
:1061800000F00B81644B1A689846002A00F00581E4
:10619000624B1B78013B012B00F2FF80DFF89091EE
:1061A0005F4CDCE00523BAF80800B0FBF3F085E6AD
:1061B0006E2000FB08F04FF01508527B90FBF8F0C2
:1061C00022B193F8008080B290FBF8F01FFA80FBB8
:1061D0003A2001F0E3FB6423BBFBF3F80FFA88F0ED
:1061E000009308F0BFFC3B2001F0D8FB009B03FBB1
:1061F00018B04FF00A0880B2053090FBF8F000B2FA
:10620000A1E6D8F8080080F31000B5E698F8003051
:1062100023B1C4F8489088F800B09EE7A36CA9EBBE
:106220000303B3F57A6F98D30123DAF8000088F8F6
:10623000003000F03DFD8046DAF8000000F038FD47
:1062400018F07F0F89D18E2887D194F84430002B25
:1062500083D1344BE3642D2384F850307DE7012251
:1062600084F85830304B84F844201B689B781E3BE0
:1062700093422E4B1ED918680221043008F0FCFB13
:1062800094F85020DFF8A4E0013AD2B284F850200C
:1062900094F8581094F85930DAB94A1C013384F84C
:1062A000582084F85930DEF8000000F007FDC4F8EB
:1062B000549060E70221186800F0F4FCE0E794F8DD
:1062C0005030002BDCD1E36484F8443008F006FC45
:1062D000D6E7E06C013310F801CB84F859300CEBB1
:1062E000010284F85820E0646146DCE7D8F8000039
:1062F00000F0DEFC83B27E2B32681BD1002384F8D1
:106300005A3084F85B3089F8013028E0BC15002051
:10631000680C0020B8130020E0220020C0130020E9
:106320002C10002040100020D0250020BC2500208B
:106330002000002099F8011089B994F85A20002A09
:1063400040F0D3801B2B40F0C680D8F8000000F04E
:10635000B2FC002840F0EB80012384F85B30D8F8D1
:10636000000000F0A8FC0028C0D1C14C94F86930AE
:106370000BB184F86900DFF824B3DFF82483DFF879
:10638000249394F85B3043B13368009A9B1A012B35
:1063900040F2DC80002384F85B30B64B1B78002B86
:1063A00000F09680B44B1B68002B00F09180B04C3D
:1063B0003668236FF31A632B40F28A800A27DFF8CE
:1063C000E882412008F015FBB8F9020090FBF7F0D5
:1063D00080B208F005FBB8F9000090FBF7F080B23E
:1063E00008F0FEFAB8F9040090FBF7F080B208F06C
:1063F000F7FA08F0CEFA94F87430D80745D49F4BDA
:106400001B88D90513D4DA0600F1EA819F0600F152
:10641000E981580600F1E881190700F1E781DA0700
:1064200000F1E68113F0020F0CBF01250325944B08
:106430001F78944B07F00107DB780BB147F0020798
:10644000532008F0D6FA904B188800EB800000EB40
:106450008000800080B208F0C3FA002008F0C0FA83
:10646000FE208A4B1B88584340F2FF3390FBF3F029
:10647000C0B208F097FA002008F094FA47EA8500C5
:10648000C0B208F08FFA08F084FA94F874309BB91F
:106490004F2008F0AEFA08F095FA08F093FA08F0E9
:1064A00091FA012008F07EFA794B187800F001008B
:1064B00008F078FA08F06DFA0A2194F8743026672B
:1064C0000133DBB2B3FBF1F201FB123384F8743019
:1064D00005B0BDE8F08F0D2B29D1012184F85C3087
:1064E00084F85A10A4F8662039E77D2B03D10123E4
:1064F00084F8683033E794F868E0BEF1000F04D008
:1065000080F02000C3B284F86810511CC9B2224444
:10651000092984F85A1082F85C300AD1B4F8662050
:10652000C2F1FF02934202D1012384F869300123B2
:10653000E9E608293FF613AFB4F86600034403EB1D
:10654000132303F0FF03A4F8663008E794F86A30D9
:106550003BF8130018B984F86A004FF4036094F80C
:106560006A30B0F5826F03F1010384F86A3000F0FD
:10657000E0805BD8B0F5007F00F0B5800ED8B0F5B4
:10658000807F00F0BB80B0F5887F7FF4FAAED8F84A
:1065900000305A077FF5F5AEA1689CE0B0F5047FA6
:1065A00000F08480B0F5806F7FF4EBAE94F86B3030
:1065B00042F210710133DBB2032B88BF012384F850
:1065C0006B3094F86B305943324B1B88002B40F0F2
:1065D000AE8001312A4B1B78DB07284B48BF0431C2
:1065E0001B88D80748BF0A319A0748BF14311806DC
:1065F00048BF2831DA0548BF2831580748BF643101
:106600001A0748BFC831980548BF01F5C8719A06F6
:1066100048BF01F57A71D80648BF01F5FA615A06FC
:1066200048BF01F57A614FF4806054E0B0F5E26F45
:106630007AD00ED8B0F5C06F68D0B0F5E06F7FF4B7
:10664000A0AE154A916B64234B43918A93FBF1F101
:1066500041E0B0F5046F61D0B0F5116F00F0B1808A
:10666000B0F5E46F7FF48DAE0B4A116CEBE700BF21
:106670002C100020CC130020B82500206613002029
:106680000413002080130020B415002064130020A0
:106690000C150020A4130020401500209081010853
:1066A00070170020C02500201C2A00205C4B5B795D
:1066B000002B3FF466AE5B4B197800293FF461AEC6
:1066C00099F80D30584A63B1138893FBF1F30A210E
:1066D0004FF40470594308F0A5F9002384F85B30A7
:1066E0004FE61388F3E74E4B9B79002B3FF449AEFE
:1066F0004E4B19680A2391FBF3F1ECE7D8F8003010
:1067000059077FF53EAE4A4B1968E4E7444B9B7945
:10671000002B3FF436AE454B9968DCE70A21454B28
:10672000B3F904305943D6E7434AD16B8BE70231C2
:1067300050E7D8F8001011F0200A7FF422AE3A6832
:10674000130605D5514608F06DF984F85BA018E6EC
:1067500099F80C30002B3FF414AE94F86C30032BF6
:106760002DD8DFE803F002181F26344A126810788B
:1067700092F803E09179090401EB0E21014401EB49
:1067800003610133DBB2042B08BF00234FF48260A6
:1067900084F86C309FE7294A1268507892F804E038
:1067A000D179E8E7254A1268907892F805E0117AE5
:1067B000E1E7234A1268507992F806E0F0E70021F9
:1067C000DDE7174B5B79002B3FF4DBAD154B1978F8
:1067D00000293FF4D6AD144B1A880A23534335E7FA
:1067E0000D2524E6092522E6042520E608251EE6D7
:1067F00002251CE6DFF84CA0DAF8000000F05BFA96
:10680000C0B201287FF6A9AC0228DFF83C803FF433
:10681000FDAC08F053F9012388F800309DE400BF77
:106820006E130020841C0020B4150020BC1500202D
:10683000680C00201C2A002040150020741700203E
:10684000982F0020BC2500202000002010B5046BEC
:106850000346C168406944B11A6C8C1A013A08BFFA
:106860000A46005D1A64C0B210BD1A6A805C01322B
:106870008A4228BF2246C0B21A6210BD436B13B1D0
:1068800090F850007047836A406A1B1A584258417A
:106890007047416A836A0269994238BF8918CB1AE6
:1068A000416B21B149680B44511E8B4202D2501EEC
:1068B000C01A704700207047036B4BB1026C5B68D5
:1068C0009342A3EB02032EBF1846C068C01870475E
:1068D000C269036A9A422FBFD01AC0688018C01AD2
:1068E00070471A238372192303700023037513233F
:1068F000C37212234370222343757047232303700E
:106900002423437000238370C37070472D2343708A
:106910002E23C3702F23437170472DE9F0410127C7
:106920000B4DDFF830802C686A6914400CB9BDE863
:10693000F081B4FA84F3C3F11F0358F8230007FA77
:1069400003F60368984724EA06046E61EEE700BF89
:1069500000040140A41000204171FEF7F3BE8160E5
:10696000FEF7F0BE00232A22036042702B22C27081
:10697000012243604271C37170472DE9F04706461A
:1069800089464FF000474FF00008038A8589ADB271
:106990001D400DB9BDE8F087B5FA85F327FA03F27B
:1069A000D2431B3B91B231821540042BF1D8DFE872
:1069B00003F02925211A0300D9F8244084B1013CB1
:1069C000A4B2C9F82480D9F820A0BAF1000FE0D011
:1069D000DAF80030504621469847DAF804A0F4E788
:1069E000B48DA4B2EFE7D9F80000B18E036889B284
:1069F0009847CEE7D9F80400318FF7E7D9F80800B7
:106A0000B18FF3E7D9F80C00B6F84010EEE71FB5E8
:106A10000023ADF80A30ADF806308DF80C30084B85
:106A200001391B68ADF80810B3FBF2F204A9013A72
:106A300021F80C2D07F019FC05B05DF804FB00BF30
:106A4000740300200B4B800A98420FD004D8B0F595
:106A5000801F09D0FE207047074B984208D0493369
:106A60009842F7D1002070470120704702207047FC
:106A7000032070470100100002001000F8B5046800
:106A800005462046FFF7DEFF032841D86B794FEA21
:106A9000930E39B975460227A689AF40B6B226EAE9
:106AA0000706A6810A2505FB00E51D4E46F82510C0
:106AB000043546F82520324631B199080223A589CC
:106AC0008B402B439BB2A3812823434303F1200136
:106AD0001144EFF31286502585F3128804251033F4
:106AE00013441F6817B10F6019680431013D03F1A9
:106AF0000403F6D10D60F3B283F31188282303FB5E
:106B00000020036A2BB1A3899BB243F00103A38148
:106B1000F8BDA38923F001031B041B0CF7E700BF9A
:106B20003C1800201D4B70B55B681D4AC3F3080379
:106B30009BB9EFF3128383B91A4910688C6800BFC0
:106B400013689842F9D14FF47A72174B596C02FBD3
:106B500001F31B1BB3FBF1F31CE0EFF312841023D2
:106B600083F312880F4D1049AE682B6813F4803FF1
:106B70001EBF01230B64AE681568086CE2B282F395
:106B800011884FF47A72496C284402FB01F39B1B75
:106B9000B3FBF1F302FB003070BD00BF00ED00E07D
:106BA000C413002010E000E0A410002038B5044613
:106BB000FFF7B8FF0546FFF7B5FF401BA042FAD329
:106BC00038BD10B5044604B910BD4FF47A70FFF714
:106BD000EDFF013CF7E7EFF31283102282F31288F6
:106BE0000649DBB20A6801320A600021044A1164D6
:106BF000044A126883F31188704700BFC413002051
:106C0000A410002010E000E0014B586804F0FABA2C
:106C100074280020014B186804F0F4BA742800208E
:106C200070B5EFF31282502383F31288436BD2B214
:106C3000196811F0010F08D15E68DEB9446A816AF3
:106C40008C4205D1012380F8503082F3118870BD49
:106C5000856998BF04690D448CBF611A611ADD60B3
:106C60008CBF596059604FF000018CBF846286620E
:106C700080F85010196841F001011960E5E7436A96
:106C80008269D154436A02690133934228BF0023C9
:106C90004362436B03B1C3E7C26CD36843F0800324
:106CA000D360704703689B69184703685B6918479E
:106CB0000368DB68184703685B68184703681B684C
:106CC000184703682DE9F041DB6904460E46174674
:106CD00093B90D467B1B3344002B01DCBDE8F081EA
:106CE000236820469B6898470028F9D015F8011BB7
:106CF0002046FFF7E3FFEDE7BDE8F0411847E0E786
:106D0000064B03EB8000826C32B193881268D16825
:106D10000B4218BF1B041361704700BFA410002072
:106D200038B50409013C022C00F00F0214D80B4DB9
:106D300035F8141041FA02F313F001000DD00120D0
:106D40009040013808400CF0C1F92C44A379034469
:106D5000034800EBC30038BD002038BDB2810108F4
:106D6000901C002037B50D460446C8B103680D4A93
:106D700003F14043A3F5843302EB9323587A07F0E1
:106D80000BFAA38801A9ADF80430206805F00303CD
:106D900005F07C058DF806308DF8075007F07FFD73
:106DA00003B030BDB281010810B1036882881A6156
:106DB000704738B1002914BF002110218388026870
:106DC0008B4013617047104B0146B3F8542032B921
:106DD000986D93F85C300BB981F00101E9E75A6FC7
:106DE00082B158B1B3F87800084A196E92FBF0F2FC
:106DF00092B20A80012283F8712070471A6E1080C7
:106E000083F87100704700BFA410002020A1070084
:106E1000012310B4084A834092F87A4002EB8002C2
:106E20002340906C21B1191C18BF012110BCC0E790
:106E3000B3FA83F14909F9E7A410002038B50D46EB
:106E4000012104460846FFF7E3FF00210846FFF74B
:106E5000DFFF04B938BD0120FFF752FF0020FFF724
:106E60004FFF0120FFF7AFFF2846FFF7AAFE0120E2
:106E7000FFF746FF0020FFF743FF0020FFF7A3FFC7
:106E8000013C2846FFF79DFEE4B2E2E738B50D4627
:106E90000130C4B205B938BD05203221FFF7CEFF5D
:106EA0004FF4FA70FFF78DFE1CB1FA212046FFF770
:106EB000C5FF4FF47A70FFF784FE013DEAE708B59D
:106EC0000A21FFF7E3FF034A034B1A60034A044B0E
:106ED000DA6008BDEFBEADDEF04F00200400FA0519
:106EE00000ED00E019E518E517E516E515E514E5F0
:106EF00013E510B5427A044632B1036800F10A0185
:106F0000406898470023637210BD2DE9F34105697D
:106F100006460F46002D3BD1D0F80080C8F3090388
:106F200073B300234FF40050D6F80080019307F0AC
:106F3000A5FC042821D12B4C4FF40050236943F0C9
:106F400001032361BBB2A8F8003007F097FC0428C6
:106F50003CD108F102030193019B3F0C1F804FF4C9
:106F6000005007F08BFC2369042823F001034FEA4B
:106F7000C3434FEAD34323612FD06FF0010507E0ED
:106F80004FF4302007F07AFC042805D04FF0FF358D
:106F9000284602B0BDE8F081124C4FF4302023693E
:106FA00043F002032361C4F81480236943F04003D3
:106FB000236107F063FC2369042823F002034FEAEE
:106FC000C3434FEAD3432361ABD0DFE7236923F008
:106FD0000103DB04DB0C2361CFE733680433336048
:106FE000D6E700BF00200240F8B504460D46002752
:106FF0008E18B54201D12069F8BDE368591CE160E3
:1070000015F8012B234404291A72F2D1A1682046F5
:10701000FFF77BFFE7602061EBE770B50D460646A2
:1070200044880021C4F30B042246284610F021FEB8
:1070300033690A4A934209D3094A934206D2224647
:107040002846BDE8704019460EF0E2B923B121464A
:107050002846BDE87040184770BD00BF00BC01085D
:10706000A6BC0108064B07498B4202D300231846F1
:1070700070471A88C2F30B029042F8D01433F3E73A
:10708000B8B8010800BC0108024A136823EA0000EE
:1070900010607047C01D0020F8B5174D2B78A32B4A
:1070A00028D16B78BE2B25D1022229464FF6FF70DE
:1070B00009F03DFF114FAC1C22884AB1A618BE4210
:1070C00018D2052A16D9214609F031FF3446F3E7D4
:1070D0002146022209F02BFF0222A11809F027FF06
:1070E0000634074B641B1C8041F60F53C31A5842E9
:1070F0005841F8BD0020F8BD00F801080000020862
:10710000881C002070B50646B6FBF2F4084615460A
:1071100014B12046FFF7F6FF05FB1464024B1B5D1C
:1071200000F8013B70BD00BF699C01081523837105
:107130004FF41673038140F2D9330122438140F2A8
:10714000C5330270838102220023C2704371037130
:1071500043708370704730B5134A58B113885B0889
:10716000012B98BF48F2050313800B6803F5C33366
:10717000A0330B60138813F0010306D10B4C04F10C
:10718000F40592F878118B4200DB30BD54F82310DF
:10719000490441BF92F8EC1002EB8101D1F8840060
:1071A00045F823000133ECE7801100208411002012
:1071B0002DE9F047264B274CB8B11A78F02A28DD84
:1071C0007F2293F901001A7094F87A21904201DA33
:1071D000002802DA9A7852429A709A7802445A70D9
:1071E0000A6802F582421A320A60002211461878B3
:1071F000194D94F8786193F9017093F902E0C0F1A8
:10720000FF08A0F17F0C05F1F409B24204D3BDE8F8
:10721000F0870F321A70E3E755F8223094009B0490
:1072200010D5CBB2DB1B83EAE37AAAEBE37ABAF19F
:10723000010F09DC53B1734514BF434663464C4408
:10724000E37001310132E0E70823F8E70346F6E78F
:10725000220000208011002084110020F0B5264A71
:10726000A0B192F87C31DBB1013BDBB282F87C311A
:107270002D23D2F880014343642093FBF0F31F4891
:10728000053390FBF3F308681844086000210C46AE
:107290001B4D05F1F40692F87831994203DBF0BDFD
:1072A00092F87B31E0E755F821008F00C0F303230B
:1072B000062B1AD192F88431DB0718D592F87C316D
:1072C00092F87BC103EB040E9EFBFCF30CFB13E373
:1072D000012BCCBF0023012333B1C0F3834002EB69
:1072E0008000D0F88400B85101340131D3E7E34382
:1072F00003F00103F0E700BF8011002040420F00BF
:10730000841100202DE9F0410F46464C48B394F813
:1073100085310E68002B4AD0D4F88851D4F88C31CE
:1073200025F0004523F00048414628460BF00EFEAC
:1073300000B9454628460BF033FEA0F119032D2075
:10734000584340F2DB1390FBF3F0374B053093FBCF
:10735000F0F094F89831064483F001033E6084F81D
:10736000983194F8983103B3D4F888512F492846BE
:107370000BF0F6FD08BB28462D490BF0D3FD002885
:1073800014BF08250025D4F88C61284930460BF03D
:10739000E7FDA0B145F0010500222649264F01F185
:1073A000F40694F878319A4212DBBDE8F08106F5D4
:1073B000433606F5A0760E60D3E70425E3E71C49C3
:1073C00030460BF0AFFD0028E6D045F00205E3E7BC
:1073D00051F822304FEA820ED80318D594F999C19A
:1073E000C3F3031003F00F03634512DD94F99AC150
:1073F0006345ACBF0223002394F99BC160450ADBBF
:1074000043F004031D421CBF3B684EF806300132B6
:10741000C7E70123F0E794F99CC16045D8BF43F06A
:107420000803EFE78011002040420F000000C84130
:107430000000C8C184110020D0810108022803D0B7
:10744000431E584258417047054B1B7913B1142015
:1074500009F0E2BF034B93F8840100F0010070478C
:10746000C0250020801100202DE9F04FC34D8BB0C6
:1074700095F89D310646E3B195F89E31CBB90F20C2
:1074800009F0CAFFBE4CB8B195F8F33013B195F8C6
:107490009F318BB9E37863B10023BA49BA4A0968CE
:1074A00042F823100133202BFAD108F05BFF0023B0
:1074B000E3700BB0BDE8F08F002301229946E27023
:1074C000B248B34CB34FDFF8DCE250F823104FEA78
:1074D000830C711A01EB0408B84507D902FA03F8C6
:1074E000714549EA080988BF4CF800600133072B51
:1074F000EBD1B9F1000FDCD095F88431A64C13F034
:107500000103039317BFB5F9C231039BA3F57A7248
:1075100064231EBF53434FF47A7293FBF2F3C5F812
:10752000803195F8F430B5F8E42105EB4303B3F965
:10753000BC7195F8EB300026203304EB83030193F4
:1075400043F69823534340F2FF3293FBF2F303F5E3
:10755000A573079395F8E830A7F57A72203304EB0A
:107560008303029395F8E930C5F8E071203304EB0A
:10757000830BB5F8E631049406934FF4B473534388
:107580004FF47A7293FBF2F3099395F878319B00EC
:107590000893089BB34217D1002401277B4D7F4EEF
:1075A00007FA04F313EA090F05EB840156F82430B7
:1075B00014BF0120002001349847072CF0D10BB0F4
:1075C000BDE8F04F08F0CEBE7348019B56F800802E
:1075D0000199C8F303201A88C9789B78042800F21F
:1075E000E380DFE810F005006800AF00BD00E500B3
:1075F000C8F3834A0AF111000AF1200300F00F00DA
:107600000AF10F0A20300AF00F0A04EB800E0AF18B
:10761000200A34F8200004EB830104EB8A0C18F4F0
:10762000805F34F8232005908B789EF8020034F8B0
:107630002A50C9789CF802A09EF803E09CF803C089
:107640001BD040F2DB5847454FF4FA7818DCA7F519
:107650007A70521BA3EB0A03A1EB0C014243434394
:10766000414392FBF8F293FBF8F391FBF8F12A44C3
:107670005344614492B2DBB2C9B24FF4B47052E0E9
:10768000059DA7F2DC5CAD1AC01AAEEB010E0CFB37
:1076900005F50CFB00F00CFB0EFC95FBF8F590FBE0
:1076A000F8F09CFBF8FC2A4403448C4492B2DBB211
:1076B0005FFA8CF1E1E70020394D4FEA800C35F894
:1076C00020E0BEF1000F1CD12E48C8F3855E0CEB04
:1076D0000005002095F83A504EFA00FC1CF0010F0E
:1076E00017D00623254A03FB0525284490F8C4300B
:1076F000049A203302EB830132F823208B78C97877
:107700000AE0069D1EEA050FDED101300628D3D11E
:1077100002E001300628DFD14FF4B47018F4805F26
:1077200001D0099D28444FF4B475024492FBF5F052
:1077300005FB102214483252024632449370D17035
:10774000043626E7039B33B1BBF800209BF80230D8
:107750009BF80310E0E7029B02991A889B78CEE71A
:1077600001F0F2FC96225043642290FBF2F000F507
:10777000A5700023FF211A46D0E700BF801100202A
:1077800022000020C481010878120020201300206C
:107790003F4B4C003E4B4C008411002014820108EA
:1077A000FC8101089F86010000283FF466AFB3E723
:1077B0000798DEE7154B60B16422B3F8E401424359
:1077C00040F2FF3092FBF0F2322A04DD012283F80E
:1077D000E8210F4A09E0142A93F8E82182F0010217
:1077E00083F8E821CCBF0B4A0B4A086802440A60C0
:1077F00093F8E8214AB993F8EB300849203301EBBC
:1078000083014FF4806008F023BD70478011002091
:1078100040420F0020A1070048E801008411002029
:10782000144B78B193F8E9214AB1012A93F8EA217F
:107830000AD082F0010283F8EA210F4A09E001220E
:1078400083F8EA210D4A04E082F0010283F8EA217C
:107850000B4A086802440A6093F8EA214AB993F88F
:10786000EB300849203301EB83014FF4407008F0FE
:10787000EFBC70478011002048E8010040420F0033
:1078800020A10700841100202E4B68B393F8EB2150
:10789000013202F00F0283F8EB2102BB83F8EC21E6
:1078A00093F8F3212AB193F8E92112B1022283F867
:1078B000EC2193F803222AB193F8EC2142F0040260
:1078C00083F8EC2193F88421D00708D4B3F824225C
:1078D0002AB193F8EC2142F0010283F8EC210A6806
:1078E00002F5C332A0320A6093F8EC2122B393F878
:1078F000EB118B081A41D20723D5012B01F00101AE
:107900000BD002D3022B13D070470F4BA3F11802F8
:1079100000290CBF1946114606E00C4B03F1080282
:10792000002914BF194611464FF4003008F090BCEE
:10793000074B03F11802EBE793F89F310BB10549B0
:10794000F2E7704780110020DC810108C481010842
:10795000D4810108D08101085E2810B50A4C09D1F4
:10796000D4F828325D2098473E20D4F82832BDE86C
:10797000104018475D28D4F82832F8D19847D4F839
:1079800028323D20F3E700BF80110020024B5E202B
:10799000D3F82832184700BF8011002070B5054683
:1079A000054C5E20D4F828329847D4F8283228466F
:1079B000BDE87040184700BF80110020038813F015
:1079C000400004D013F4057F14BF0120002070474D
:1079D0002DE9F743774CD4F82C82B8F1000F33D05F
:1079E0004046FFF7EBFF744E814658B1D4F8283279
:1079F000B34229D0D4F8303233B3704A1360C4F89C
:107A0000286221E094F83402FFF718FDD4F82832F8
:107A100005469A1B53425341834215D0674F0028B5
:107A20007CD0674B98F902005B794A46B3FA83F33E
:107A30005B0901930223042100934FF4165307F0CE
:107A400093F938600028DAD194F83502FFF7F6FC94
:107A500094F83632054683421DD0002867D0594B32
:107A60001B68C3B1564A93F9020092790323002A96
:107A70000CBF00220822009301924FF4964300228B
:107A8000082107F071F9504B186020B107F026F873
:107A9000012384F8363294F83702FFF7CFFC94F8CC
:107AA00038320546834224D0002848D0D4F83C120E
:107AB000F9B1434A91F9020093795279002B14BF2E
:107AC00008230023002A08BF43F001030193032386
:107AD0000022009320214FF4614307F045F93B4B0E
:107AE000186030B1012384F8403284F83832D4F879
:107AF0004432D4F8485265B32846FFF75FFF40B3DD
:107B000094F84C32002B49D1D4F83032002B45D0B8
:107B10002F4A1360012384F84C323FE03868002874
:107B200092D007F0FCF83D60C4F828528CE7264E4E
:107B3000306807F0F4F8356084F83652ABE7234E2E
:107B4000306807F0ECF8356084F8405284F8385219
:107B5000CFE794F84D02FFF771FC94F84C320646DB
:107B600083421BD0E8B1CDB1AB791A4A002B08BFD4
:107B7000022302EB8303124A95F902005279DB6E6D
:107B8000003218BF0122019202221021009200222D
:107B900007F0EAF80E4B18600028BBD103B0BDE82F
:107BA000F0830B4D286807F0BAF82E6084F84C6219
:107BB000F4E700BF8011002089E10008E4220020E2
:107BC000C0250020D0250020BC250020E022002078
:107BD000B8250020C48101080F2A10B51CD805283B
:107BE0000AD8052918D806240C4B04FB00300144A0
:107BF00081F8C420012010BD062806D10A290BD81F
:107C00000648014481F8E820F4E7072804D119B9AF
:107C1000024B83F8F420EDE7002010BD8011002016
:107C200030B5214C85B094E82C009A42207E1F4943
:107C30001F4A637E1EDB91F82010127825612075A3
:107C40006175A275E375532008F0F8FC206908F00F
:107C50008EFD207D08F08BFD637D01A80193A37D3F
:107C60000293E37D039308F0F3FC002301202360DB
:107C700005B030BD91F820101278019504F110057F
:107C80008DF808008DF809108DF80A202946082281
:107C900001A88DF80B300FF0C3FF0028E8D001AB2E
:107CA00003CB20616161CEE7F41400208013002033
:107CB000051300202DE9F74F3B4C0025D4F81C801C
:107CC00004F12801464608F1300746F8040B04F198
:107CD000340B04F1400A04F14C0204F19409685891
:107CE000019200910BF05CF946F8040B55F80B007B
:107CF0000BF056F9B06055F80A000BF051F92B4B18
:107D00007061E81840680DF0E9FC019A27F8020B51
:107D10005019806B0099B88055F8090004350C2D76
:107D2000F884DCD10025224F08F1280657F82500F9
:107D30000BF036F90135042D26F8020BF6D100259B
:107D4000B4F8A43094F8AC70A8F83C30B4F8A6307D
:107D5000DFF86490A8F83E30B4F8A83008F1440683
:107D6000A8F84030B4F8AA30A8F84230BD4212DB7F
:107D7000B4F8C230A8F84E30D4F8CC30A8F850305F
:107D8000D4F8F830C8F854300A4B1B88A8F85E3095
:107D900003B0BDE8F08F59F825000BF001F901356B
:107DA00026F8020BE2E700BFF41400208025002033
:107DB0000813002064130020A4150020164B174957
:107DC0001A68B1F9001001321A60D3F800210132AB
:107DD000C3F80021B3F80421013292B28A42A3F819
:107DE00004210ADB0021B3F80621A3F804110132B3
:107DF000A3F80621A3F808117047B3F80821084931
:107E00000132B1F9001092B28A42A3F80821A4BF4E
:107E10000022A3F808217047F41400207E2F0020D0
:107E2000802F002038B5244B054693F80A310C46C4
:107E3000093B012B3FD8452008F000FC284608F0FC
:107E4000FDFB0E2D0ED003D83DB10D2D0FD038BD4A
:107E50001E2D07D0FF2D29D038BD2068BDE8384041
:107E600008F085BC206808F082FC6068F6E7637A59
:107E7000207AA3B180F0800008F0E0FB6468E0B2F3
:107E800008F0DCFBC4F3072008F0D8FBC4F307407C
:107E900008F0D4FB200EBDE8384008F0CFBB08F056
:107EA000CDFB2068BDE8384008F070BC034808F0FE
:107EB000B3FB0020EFE738BDF41400208E9C0108CE
:107EC0002DE9F04F624C89B0B4F804310646002B1E
:107ED00040F0C6805F4B1B880BB9FFF7A1FE304610
:107EE000FFF7E8FEE56949202E4608F0A7FBD4F825
:107EF000000108F03CFC56F8040B08F038FC304652
:107F000006F078FB05F1100006F074FB10264FF028
:107F1000010805F11C07D4F80C2108FA06F31342F6
:107F200002D0386808F032FC0136132E07F104073E
:107F3000F1D1032105F1280008F02CFCB4F81C3124
:107F4000B5F92E00C01A08F012FCD4F80C31DE048A
:107F500008D5B4F82201B5F84E30C01AC0F30D00B0
:107F600008F005FCD4F80C31980403D5B5F850009E
:107F700008F0FDFBD4F80C31590504D5032105F1B7
:107F8000580008F007FCD4F80C311A0502D5686DCA
:107F900008F0FCFBD4F80C311B0403D5B5F85E00E7
:107FA00008F0E5FB032105F1300008F0F3FBD4F8FD
:107FB0000C31DF0204D5032105F1360008F0EAFB9D
:107FC000D4F80C319E0204D5042105F13C0008F0E0
:107FD000E1FB0126B5F944000AF0B2FDD4F8241102
:107FE0000AF0F8FC0BF002F808F0C1FB94F8AC8042
:107FF00005F14607B04522DCD4F80C31980505D5CB
:10800000B5F95600A0F2DC5008F0C0FBE26922622C
:1080100062621149114B521A521153430322013328
:1080200093FBF2F202EB42029B1A602202FB031363
:10803000E361012384F8483209B0BDE8F08F37F9D5
:10804000020BB5F944300136C01A08F09FFBD1E7A6
:10805000F4140020702F00201C160020ABAAAAAA3E
:10806000D4F84C32D4F850229A4207D008A941F8EB
:10807000203D0020C4F85032FFF7D4FEBE49042250
:10808000A1F513700FF0CCFD58B1D4F8543208A903
:108090000193A3681E2041F8203DC4F85432FFF735
:1080A000C1FEB4F80851002DC6D1B44B1B88002B7B
:1080B000C2D0FFF7B5FD3046FFF7FCFD5020E76961
:1080C000D4F8208008F0BAFA626AE36910681B6885
:1080D000226A034410683E1DA3EB400008F056FBE3
:1080E0002B4608F1040056F8232050F82310521AAA
:1080F0004DF823200133032BF5D10025684606F007
:1081000079FA07F1100008F1100150F8253051F804
:1081100025209B1A4DF825300135032DF5D16846F1
:1081200008F096FA10264FF0010B07F11C0A08F12F
:108130001C09D4F80C310BFA06F21A4206D0DAF810
:108140000000D9F80030C01A08F020FB0136132EC9
:108150000AF1040A09F10409EBD1002307F1280010
:1081600008F1280130F9022B31F9026B921B4DF80E
:1081700023200133042BF5D100265DF82530B6000D
:10818000F6B22BB103F108020F2A77D846F00106A8
:1081900015F1FF35F1D20025304608F04FFAEB46D5
:1081A000A9460DF1100A06F00303022B78D0032B29
:1081B00000F08A80012B07D1B9F1000F66D19946F2
:1081C000DBF800502D01EDB20BF1040BDA454FEA5C
:1081D0009606E8D1B9F1000F02D0284608F02EFA31
:1081E000D4F80C3113F4805506D00125B7F84E2091
:1081F000B8F84E10521A009299040AD508AA02EB58
:108200008501B8F85000B7F850200135121A41F82E
:10821000202C5A0513D50DEB850207F1580108F102
:108220005806043A07F15E0E31F9020B36F902CB1B
:108230008E45A0EB0C0042F8040FF5D103351E0566
:1082400009D508AA02EB8501D8F854007A6D0135EA
:10825000121A41F8202C18044AD508AB03EB85020A
:10826000B8F85E10B7F85E3001355B1A42F8203C72
:10827000012D68D1009808F089FA3BE08033FF2B8C
:1082800094BF46F0020646F0030681E7DBF80000E3
:108290004FF0000900F00F00284308F0CFF993E7F2
:1082A000B9F1000F04D19BF8000008F0C7F98BE783
:1082B000DBF80000C0F30310284308F0BFF9DBF837
:1082C00000502D01EDB27FE7B9F1000F04D19BF80A
:1082D000010008F0B3F9E6E7DBF80000C0F3033073
:1082E000284308F0ABF9DBF80000C0F30710E4E71F
:1082F000002DBDD10321302001F0BCFDD4F80C319C
:10830000D90203D50321362001F0B4FDD4F80C3195
:108310009A0203D504213C2001F0ACFD94F8AC1086
:10832000442001F0A7FDD4F80C319B0506D5B7F920
:108330005600B8F95630C01A08F028FA236AE269E4
:108340006362226265E600206B1E5DF82320400018
:10835000C0B20AB140F0010013F1FF33F5D208F0CA
:108360006DF900265DF8260008B108F00FFA013615
:10837000AE42F7DBBEE700BF48170020702F002099
:108380002DE9F74F9B1A164600930D9A0E9B002974
:1083900014BF062504259B1A01934E4B0746D3F8BC
:1083A0005C228A460132984626D1D3F85842A5422B
:1083B00040F28E80484A52F824B0584609F050FEE8
:1083C0000B3008F0E1F8814618B1012003B0BDE898
:1083D000F08F5A46032C94BF394651463F4808F067
:1083E00013FA3F4988F860920A68101AD8F85C229C
:1083F00008600132C8F85C22DFF8E490DFF8E8B0EA
:10840000D8F85C420C9B9C421BDB13D1012008F086
:10841000BBF878B932490A200A68013A0A6008F0C4
:108420000DF9D8F858220132C8F858224FF0FF321F
:10843000C8F85C22D8F85802854294BF0020012079
:10844000C4E70D9B53B1019B04FB03F20D9B995CA8
:1084500001228A40D8F80C110A4228D0009BD8F893
:1084600058225C43371942BB305909F0F9FD00F13D
:10847000050A504608F088F80028A6D1D9F800006F
:1084800098F86022A0EB0A00C9F80000C2B12C20C5
:1084900008F0D4F8D8F85822B2B9305908F0BCF82E
:1084A00097F904104B1C02D0584608F0ADF9D8F8E3
:1084B0005C220132C8F85C22A2E74FF0030AD8E739
:1084C000012288F86022E5E7174439790548ECE78E
:1084D00000207BE7F414002070820108999C0108B9
:1084E0006C2F002051B30108A89C010810B50C4C5A
:1084F00094F80A210B2A0BD8012340F6030193407C
:1085000019400CD113F4C06F02D0FF20FFF78AFC92
:10851000044B1B68C4F85C320B2384F80A3110BD8D
:10852000F4140020C41300202DE9F04F7D4B87B0D8
:108530009A787D4C032A1CBF03229A709B78032BE8
:1085400024D1802006F0B2FD0646F8B1802106F065
:10855000A3FD7579754B84F8610253F8253096F9BF
:108560000200B3F5613F0CBF0222002201920222F9
:1085700080210092002206F0F7FB0C3D6C4B032D8E
:1085800018606C4A08D840231370A0B9002384F8FF
:108590000A3107B0BDE8F08F4FF4FA71D4F86432B5
:1085A00003EB4303B3FBF1F31BB1402BA8BF402304
:1085B000EAE70123E8E7142200215F480FF059FBA6
:1085C00000205E4B574903F160022262D4F88022FA
:1085D0000F8803925A4A17F1FF379679527906F1BC
:1085E000FF3518BF01276E426E41E361121A03F195
:1085F000C00394F8AC5018BF0122636294F886E27D
:10860000B4F8C23002950D79BEEB000EA4F8223109
:10861000D4F87C3294F8A11218BF4FF0010E2D1A35
:1086200018BF012513F0020F08BF054681424FF025
:108630000101049294F88422C3F3800AC3F3C009B1
:10864000D4F88832A2F11908C3F3C03318BF01234C
:10865000D8F1000C4CEB080C012A08BF4FF0010CBC
:1086600080468B46C4F80C0105934A1ED2B2531EB5
:10867000152B17D8DFE803F0101010101010101091
:108680000B525446481B4A3B3B3B4C4E501B6346E7
:1086900043B90131C9B2E8E7029B9A42CCBF00233B
:1086A000012323B101200BFA02F248EA020816293D
:1086B000EFD91D4C08B1C4F80C811A2008F072FEE5
:1086C0000023D4F84C22C4F80031C4F85022A26828
:1086D000A4F80431A4F80631A4F80831236084F822
:1086E000483284F8B802C4F8542202234FE7A2F1BA
:1086F0001003039C03EB430323449B78003318BF10
:108700000123CEE7049BC3E73346C1E7059BBFE7E0
:108710003B46BDE72B46BBE77346B9E74B46B7E799
:108720005346B5E7702F0020F41400203082010872
:10873000782F00207C2F00205C1700201C160020C2
:108740006E13002010F8113C0133DBB20A2B00F845
:10875000113C07D9002310F8131C034A22F81130EA
:1087600000F8113C704700BF6021002070B5142450
:10877000474B1A780132B2FBF4F004FB1022586820
:108780001A701A6C81429C680A4404D293F849001A
:1087900008B102F580323F480678B2FBF6F2944207
:1087A00024D293F849501DB14FF4803595FBF6F56E
:1087B000101B451BDD609A6040F68C22002059603A
:1087C000D96883F84900914243D993F8440093F95A
:1087D0004620904231D1021F082A2ED893F8472014
:1087E000182A0BD8013283F8472009E04FF4803073
:1087F00090FBF6F0001B1044D860DCE783F84500DE
:1088000093F9452090420FD193F8481061B10021AF
:10881000214C224D914212DB002420490B2A14DD09
:108820001F490A7801320A70012283F84820002289
:1088300083F8460083F8442070BD0022D3E754F843
:10884000046F25F811600131E4E721F8124001328C
:10885000E4E793F84820CAB140F2DA52A1F2EF20DF
:10886000904208D893F844200B2A04D803EB8200E6
:1088700001610132DEE7002283F8482011461346E9
:108880000848C2180433302BD160FAD170BD00BF44
:10889000F017002026000020FC1700206021002097
:1088A00059210020F417002010B51424094B1A7820
:1088B0000132B2FBF4F004FB10221A701A6C013280
:1088C0000A441A644FF6FF72914204BF012283F8F2
:1088D000492010BDF017002070477047064B10B5B7
:1088E00059681C689B6800F1240204604160836041
:1088F0000C309042F9D110BD88820108034B33F847
:108900000C2F9B7802808370704700BF888201081B
:108910002DE9F047182550264FF028084FF00009A0
:10892000144C154F05FB0045A54201D1BDE8F08769
:10893000237CCBB1D4F804A05046FEF783F8EFF3C4
:10894000128386F31288BAF8242008FB007092B2D2
:1089500001320267BAF81420DBB292B242F001028F
:10896000AAF8142083F3118854F8183BA3F8009058
:10897000DAE700BF6C190020F0170020182370B54B
:108980000E465843074A14181558A16830460AF095
:108990002BF9E1680AF020F80CF0A0FE80B22880E4
:1089A00070BD00BF6C1900202DE9F0412C4B06462C
:1089B0001B782BB92B4A136053609360BDE8F0819C
:1089C000294B2A4C9B79D4F8EC80012BC4F8EC009D
:1089D00009D001D3042B04D90022224B1A605A601B
:1089E0009A60BDE8F081224F224BB7F902200021A6
:1089F0005343B7F9002004F5807093FBF2F3C4F8F9
:108A0000FC3007F0A3FF0AF0F1FA85B240F6E4402B
:108A10006843B7F90250B7F90030C5EB10304FF496
:108A20007A75454395FBF3F5D4F8FC70A6EB080086
:108A3000C4F8F85078430AF083F80F490AF0D4F8E4
:108A4000D4F8F41009F0C8FFC4F8F4000AF0A8FA4A
:108A5000044BC4F8F00083E8A0009860BDE8F08102
:108A6000841C0020BC1500206E130020F01700208D
:108A7000040D002018FCFFFF2FE33E312DE9F041EB
:108A80001B4B1C4D5B79012B2ED11B4E002106F593
:108A9000947007F05BFF194B5A789F781B78C2EBF4
:108AA000023803EB43140AF0A1FA44F6FB7183B2D7
:108AB00003FB0413B3FBF8F3B1FBF8F2B3FBF7F3DA
:108AC000B2FBF7F29BB2A6F82431A6F826212B8040
:108AD0006A800B4B1B78022B04D10A4B6A881A80E0
:108AE0002A885A80BDE8F08100232B806B80F0E754
:108AF0006E130020B4150020F0170020000D002098
:108B00007A1700209815002008B50A4A1378D9076B
:108B10000FD523F001031370074B9B780BB1FFF7C0
:108B2000E5FC0020FEF74FF9BDE80840042006F000
:108B300061BB08BD04130020702F00202DE9F04117
:108B4000654E3378DD0705D5BDE8F04101210020F1
:108B5000FEF75EB9614D2B881C060BD5604B1A6879
:108B6000604B19794FF47A734B43934202D88020BB
:108B700006F01EFC5C4A5D4C137890467BB95C4A5B
:108B800094F84C011778002876D137B108F044FCEE
:108B9000002878D0082006F013FC84F84C711B20C4
:108BA00008F03AFC002872D0102006F009FC08F00A
:108BB00047FC00286FD0202006F002FC4D4B1B78AC
:108BC00018076CD4232008F027FC002867D1402028
:108BD00006F0F6FB484B4FF480601B88642B62D98B
:108BE00006F0EEFB454B1B68590702D5B4F84E2141
:108BF0004AB9B4F850210AB19A0704D4404BB3F8EB
:108C0000B430002B52D04FF4006006F0D9FB242082
:108C100008F0C8FB58B1242008F0FEFB00284AD019
:108C200033785B0747D44FF4807006F0C1FB98F8A7
:108C300000308BB92B88002B42D0324A12781AB1FF
:108C400023F42063002B3BD0002008F0E5FBB8B3F1
:108C50004FF4007006F0B4FB2B8803B1022384F8B4
:108C60005231FDF75FFFD4F85431C01A002831DBD0
:108C7000BDE8F04106F02AB8002F8ED0184608F063
:108C8000CBFB002889D1082006F092FB85E7102055
:108C900006F08EFB8BE7202006F08AFB8EE7402053
:108CA00006F086FB96E706F083FB9BE74FF4006037
:108CB00006F07EFBABE74FF4807006F081FBB6E771
:108CC000002008F0A9FB0028C6D14FF4007006F080
:108CD0006FFBC1E7BDE8F08104130020A41300205E
:108CE000C4130020241C002000000020F0170020E6
:108CF000051300200C1500208A1C0020701700208E
:108D0000FC2200202C0D002070B5344D2B783BB197
:108D1000334C237823B9334801F0CCF80123237076
:108D2000FFF70CFF304B1A883ABB304E3478E3071C
:108D300053D444F003032420337008F033FB10B104
:108D400044F0070434700A22294B4FF47A70B3F9C7
:108D5000043093FBF2F3274A1380274B274A196804
:108D6000AB7800FB0313C2F8583100230520C2F88A
:108D70005C31BDE8704006F03DBA194B1B781BB161
:108D80001F4BB3F8B43043BB92FAA2F3002AB3FAF4
:108D900083F308BF4FF0FF33184A0133D2F85C1158
:108DA0008B421AD0C2F85C31DBB29B00402BA8BFCB
:108DB0004023002214260A2005251249541856542F
:108DC00004326070A5709A4202EB010404F8010CB1
:108DD000F4D3FF230E208B54CBE770BD2C0D002065
:108DE000340D0020B0230020A41300200413002021
:108DF0001C2A0020500C0020C4130020F017002073
:108E0000FC2200204C1F002010B57C4B93F86031F1
:108E1000012B14BF00240324038C002938D123F034
:108E200001031B041B0C0384018B038C89B221F00A
:108E3000F30141F0010141EA0411714C9BB2A042DF
:108E400042F0010212D004F50064A0420ED0B0F14D
:108E5000804F0BD0A4F59834A04207D004F580646D
:108E6000A04203D004F58064A0420ED123F0020397
:108E7000134301830384038B23F00C031B041B0C9B
:108E80000383038B9BB2038310BD23F00A03EFE738
:108E9000042938D123F010031B041B0C0384018B1D
:108EA000038C21F440710905090D41F4807141EAF8
:108EB0000431534C9BB2A04212D004F50064A0428E
:108EC0000ED0B0F1804F0BD0A4F59834A04207D05B
:108ED00004F58064A04203D004F58064A0420CD164
:108EE00023F0200343EA021292B242F010020183FF
:108EF0000284038B23F44063C0E723F0A00342F015
:108F000010021A43F3E708293DD123F480731B04B0
:108F10001B0C0384818B038C89B221F0F30141F097
:108F2000010141EA0411364C9BB2A04212D004F573
:108F30000064A0420ED0B0F1804F0BD0A4F598345D
:108F4000A04207D004F58064A04203D004F58064F9
:108F5000A04212D123F4007343EA022292B242F4F7
:108F6000807281830284838B23F00C031B041B0C0F
:108F70008383838B9BB2838310BD23F4206342F4ED
:108F800080721A43EDE723F480531B041B0C038407
:108F9000818B038C21F440710905090D41F4807126
:108FA00041EA0431164C9BB2A04212D004F5006491
:108FB000A0420ED0B0F1804F0BD0A4F59834A0425F
:108FC00007D004F58064A04203D004F58064A04279
:108FD0000CD123F4005343EA023292B242F480529D
:108FE00081830284838B23F44063BFE723F40073FF
:108FF0005B045B0C42F480521A43F1E7F017002047
:10900000002C014038B510F80E2C044650F8043CF2
:1090100052B9012220F80C1C00F80E2C597918685E
:109020000222BDE83840EFE6002530F80C2C20F88D
:109030000A1C891A89B220F8081C074A10F80F0C7C
:1090400022F8101004F80E5C2A4659791868FFF7C8
:10905000DBFE04F80D5C38BD602100202DE9FF41E6
:109060000C469DF82C80194605462068FDF7CFFC7C
:1090700026686779E379B8F1000F01D083F0020325
:109080000022ADF80220ADF80420ADF80820ADF8BC
:109090000A20ADF80C20ADF80E20602213F0040F6A
:1090A000ADF8002003F0020330D0002B4FF0040293
:1090B00014BF00230823ADF80420ADF80A30BDF832
:1090C00028306A4639463046ADF8063004F056F886
:1090D0003946304605F09CF82268B2F84430114613
:1090E0006FEA43436FEA53439BB2A2F844301388BC
:1090F0009BB243F0010321F8343B6379C81885E83B
:1091000005000022CA5204B0BDE8F0810122ADF88A
:1091100002204FF48072ADF80830ADF80C20CEE795
:10912000022828BF02200C22044B5870044B02FB7B
:109130000030044B186008F0BFB900BF241C0020A9
:10914000080D0020982F002038B5194B187808B367
:1091500018490C89FCB1204609F0EEFC164B054677
:10916000986809F0EDFC0146284609F033FC1349E4
:1091700009F03AFD0546204609F0E2FC0146284682
:1091800009F0E6FD09F00CFF6428A8BF642020EA7E
:10919000E070C0B238BD0A4B4D781B880A7800FBDE
:1091A00015346423521B63435043B3FBF0F0EBE7E9
:1091B000841C00206E130020BC1500200000C84253
:1091C000B41500202DE9F84F0024804625464FF0C5
:1091D0000D0ADFF85090DFF850B00AFB04963768AC
:1091E000414638460EF0C7FD78B13946584607F07B
:1091F00028FF0021304607F0C7FF07F0D0FF3046B8
:1092000008F05FF807F0CBFF01350134BA2CE4D148
:1092100025B9BDE8F84F024808F0BAB8BDE8F88FA4
:10922000C79C01089882010837B301082DE9F74F60
:10923000804608F015FF054628B1012820D198F88E
:1092400000302A2B1CD1774808F0A2F800244FF0F8
:109250000D09DFF8D881744F09FB04863846316860
:1092600007F0EFFE291C18BF01213046013407F03A
:109270008BFF07F094FFBA2CEED103B0BDE8F08F5E
:109280003D2140460EF01BFD002800F0C68006463A
:1092900016F8013C721E202B48D0A6EB08060130C0
:1092A000044623780130202BFAD000270D23DFF865
:1092B0007CA1F6B203FB07A5D5F8009001934846C0
:1092C00008F0CEFE49460246834640460EF005FDB4
:1092D000019B8146002840F09680B34540F0938082
:1092E0002B7903F03003102B22D0202B51D08BBBD5
:1092F00020460CF065F8B5F9053001B28B4229DC47
:10930000B5F907308B4225DB284607F08BFE0D238D
:10931000464A474803FB0727396807F092FE0021B9
:10932000284603B0BDE8F04F07F02EBF1646AFE762
:1093300006468146834695F805803C4B03EBC808FA
:1093400098F878A9564502D2B9F1000F0BD0BBF1BD
:10935000000FDCD1374808F01BF8284603B0BDE801
:10936000F04F07F0AEBFD8F87439214653F8260005
:109370000EF087FC00280CBF4FF001094FF00009E8
:1093800005D131B2284607F04DFE4FF0010B0136F2
:10939000D8E70D268346254B95F8058006FB073652
:1093A000C845D4DD23461C46217801332029FAD054
:1093B0002C2120460EF083FC824618B908F1FF33B9
:1093C0004B4513D1337903F00303022B11D0032B48
:1093D0000FD0284607F019FE834620460BF0F0FF19
:1093E0000BF809004FF0010B0AF1010409F1010922
:1093F000D6E7284607F009FE834620460BF0E0FF3B
:109400002BF81900EEE70137BA2F7FF453AF0A4863
:1094100003B0BDE8F04F07F0BBBF404603B0BDE866
:10942000F04FCFE6D49C010837B3010898820108B9
:10943000E79C0108F29C0108C79C010838B5044666
:109440000B4D204602F0EAF830B10A4B0A48597831
:10945000BDE8384007F028BF20460BF0B1FF0228D6
:1094600004D8C0B2FFF75CFE2C46EAE738BD00BF67
:109470005D9C0108241C0020009D010870B5044675
:109480000A4E0B4D204602F0C9F830B1074B09488F
:109490001978BDE8704007F007BF20460BF090FF39
:1094A000022802D830702C46ECE770BD241C002046
:1094B0005D9C0108049D01082DE9F743054602F073
:1094C000ADF8044620B107F069FF03B0BDE8F083B2
:1094D000284601AA30490BF0CFFF264625462F4FDC
:1094E000DFF8D480DFF8D49078B9022CEBD1A6F560
:1094F0007A73B3F57A7F2ED94FF4FA634FF47A7208
:109500002749284807F0D0FEDFE744B1012C1ED0E0
:1095100001AA2149002001340BF0AEFFE4E70BF073
:109520004FFF051E0DDB3B789D4204DA2946484675
:1095300007F087FBECE7FF2D03D1404607F081FBE6
:10954000E6E739781848013907F07BFBBDE70BF0F7
:1095500037FF0646DCE7FF2D0AD104460F4B134FB9
:109560001D78AC4210DB3146114807F09DFEACE798
:10957000304609F0E1FA0D4B324643F82500294602
:109580000C4807F091FEA0E7304609F0D5FA47F8FD
:1095900024000134E5E700BF319C0108A01500203C
:1095A000FA9C0108609D0108379D010854190020AC
:1095B000869D0108799D0108229D01080F9D0108E3
:1095C00070B5134C0546134807F064FD2069FDF79C
:1095D00090FC606905F098FB0F4B18201978002368
:1095E0001E4618348B420BDB40F2DC50FDF7DEFAEE
:1095F0000A4B0B4A15B10B480B490860DA6070BD85
:1096000000FB03F2125902B116800133EAE700BFF2
:1096100054190020959D0108A015002000ED00E0E0
:109620000400FA05EFBEADDEF04F002038B5054668
:1096300001F0F4FF044628B90622074928460EF037
:109640004CFB40B903F072FD2CB103F073FABDE896
:1096500038400020B4E738BDF0AE010808B503F08B
:1096600069FABDE808400020AAE738B500250A4C91
:109670002069FDF73EFCD4F80031284684F8785084
:10968000C4F8F85084F8FC5023606360A360E36082
:10969000FFF796FF256138BD5419002001208FE7A0
:1096A0002DE9FF41074608F0DBFC08284AD10025D8
:1096B00001AE7C5D0BF08CFE2044437803F0030385
:1096C000022B08BF203CAC550135082DF1D10025F7
:1096D000DFF87C808DF80C507C5D0BF079FE204427
:1096E0004378404603F00303022B08BF203C745527
:1096F000E4B221460EF0E3FA28B101352146701993
:109700000EF0DDFA20B107F049FE04B0BDE8F081AB
:10971000082DE1D10D49304604F018FC00230B4C14
:109720000B481A5D04A90A44195C0133082B02F89E
:109730000C1CF6D1002301A906488DF80C3007F067
:10974000B3FDE2E70028E9D0DDE700BF8017002085
:1097500018940108A19D01082DE9F74F804608F0F3
:109760007FFC454E04463768E8B9444807F069FC79
:109770000C25434EDFF82C81204605F011FD3842C0
:1097800005D005FB04634046996807F05AFC013494
:10979000132CF1D117B93B4807F07CFC03B0BDE8AE
:1097A000F04F07F0FCBC0246374940460EF095FAF0
:1097B000DFF8CC90054670B9344807F06BFC2C46B6
:1097C000334D09EB0403996828460C3407F039FC43
:1097D000FC2CF6D1E2E798F8003000252D2B0CBFC9
:1097E0004FF0010A4FF0000A4FF00C0304BF08F1DC
:1097F000010804F1FF3403FB0592D2F808B040469B
:109800002246594601930EF068FA019B58BBBAF103
:10981000000F17D0132D0BD11E4B33601E4807F0DD
:1098200039FC59461A4803B0BDE8F04F07F03CBD7B
:10983000142D01D17368F0E7284605F0B1FC3843D8
:109840003060EBE7132D03D1C6F800A01348E6E71C
:10985000142D01D17760F9E7284605F0A1FC27EA2D
:1098600000003060F2E70135152DC4D10C4803B07B
:10987000BDE8F04F07F08CBDD01D0020A89D010869
:109880009C920108B29D0108BE9D0108C39D01087C
:10989000BA9D0108FFFF0700CE9D0108D79D010872
:1098A000C79C0108B99D01082DE9F84F054608F04D
:1098B000D7FB364F0446D7F80090B0B9344807F0CC
:1098C000E9FB0126334D344F55F8241049B106FA0F
:1098D00004F313EA090F02D0384607F0B2FB013453
:1098E000F2E7BDE8F84F07F05ABC02462B4928467C
:1098F0000EF0F3F978B92A4807F0CCFB294C2A4D31
:1099000054F8041F0029ECD00B78002BF8D028461F
:1099100007F097FBF4E72B7800262D2B0CBF4FF0B8
:10992000010A4FF0000ADFF86CB004BF013504F102
:10993000FF345BF82680B8F1000F04D11B48BDE866
:10994000F84F07F025BD2246414628460EF0C5F9DE
:10995000D0B90120B040020601D51548EFE78305D4
:10996000FBD4BAF1000F0AD0FDF78EFB114807F0C7
:1099700091FB4146BDE8F84F0B4807F095BC40EA23
:10998000090038600C48F2E70136D2E7C01D00201C
:10999000DF9D010820920108E99D0108BE9D010894
:1099A000C39D01081C920108BA9D0108C79C0108CB
:1099B000ED9D0108CE9D0108D79D010870B50646B2
:1099C00008F04EFB124C054690B1112200212046B2
:1099D0000EF04FF92A460F4930460EF0A5F938B17E
:1099E000102D2A46314628BF102220460EF0AEF92F
:1099F0002378074A002B08BF0121BDE87040054BC2
:109A00001CBF002113460120034A07F0AFBC00BF72
:109A10003B1F0020F99D0108FB9D0108022810B59D
:109A20000C460CD8FFF77CFB0548FFF707FD07F055
:109A3000B6FB2146BDE81040082007F0B5BB10BDBD
:109A40005D9C0108022810B50C460CD803F05CF8A8
:109A50000548FFF713FD07F0A2FB2146BDE81040C3
:109A6000042007F0A1BB10BD5D9C010870B5044641
:109A700008460E4608F0F4FA3146024620460EF03B
:109A80002CF908B1002070BD0BF0A2FC0546304651
:109A900008F0E6FA235C1D446A78120701D4002B13
:109AA000F0D10130204470BD2DE9F04F05468846C5
:109AB00014460027DFF8E0A085B0062300267B438C
:109AC0000393039B334408EB030292F8C0B0002CCD
:109AD0005ED0234493F8C0305246ABEB0300D0F184
:109AE000000949EB0009019300963B464946284688
:109AF00007F026FC8DE840083B465246494628467A
:109B0000013607F033FC062EDBD10137062FD4D106
:109B10000026DFF884B008F1E40A1AF8019B002C53
:109B200038D0A31993F8E4305A46A9EB03014F4209
:109B30004F410193009606233946284607F000FC62
:109B40008DE840020623144A39462846013607F0BC
:109B50000DFC0B2EE1D198F8F0606CB194F8F03068
:109B60002846F21A019300235442544100930A4AB2
:109B70000723214607F0E4FB002301960093064AE1
:109B800007232146284607F0F1FB05B0BDE8F08F1A
:109B9000A146AFE72746D3E7039E01087FB50546F8
:109BA00001F03CFD044630B1002218490120FFF7C6
:109BB0007BFF04B070BD28466A4615490BF05CFC7B
:109BC000134E01AD78B1032C02D107F0E7FBF0E7AB
:109BD0000BF0F6FB6A4645F82400314600200BF0F6
:109BE0004BFC0134EEE7032CEFD101AC70CC3246D4
:109BF0002946E0B2FDF7F0FF0028E6D033462A46BA
:109C00002146044807F050FBD3E700BF8411002031
:109C1000319C0108039E01082DE9FF4781469046CB
:109C20000E4615460027DFF864A0B8F1000F2AD0D1
:109C30002B8832889A4224D174886A88A21A5442A6
:109C40005441EA7821460292AA784846019200934C
:109C500052463B4607F074FBF37852460293B378C2
:109C60002146019336F8043B484600933B460137B2
:109C700007F07CFB102F05F10405D6D104B0BDE838
:109C8000F0870024DDE74446E6E700BF179E0108A1
:109C90002DE9F041064601F0C1FC044628B1BDE8BB
:109CA000F041002223490120B6E730460BF088FB43
:109CB0000F2805462EDC304607F09BF90646DFF8F4
:109CC00084801D4F203530460BF07AFB38F8143075
:109CD000984227DC012C11D0022C13D027F8250044
:109CE00030462C210DF0EBFF064678B101230136FA
:109CF0000134BBB1032CE6D1BDE8F08107EB85034D
:109D00009870EDE707EB8503D870E9E7A21E534290
:109D10005341EDE72246BDE8F0410F2307490848CB
:109D200007F0C2BA002347F82530BDE8F04107F03C
:109D300035BB00BF0412002084110020299E0108B9
:109D4000609D0108B48C010810B510220021044662
:109D50000DF08FFF0A2323800023A381E381E3809A
:109D60002381638110BD03788B4286BF024B33F899
:109D700011000020704700BF581A0020034B187EC6
:109D800010B1002201201A76704700BF581A002037
:109D900070B50546FCF7C6FE354CE369E061C31AB1
:109DA000B3F5FA5F82BF002384F8203084F82130B5
:109DB00094F820303BB9A12D21D1012284F8212033
:109DC0001B2284F8222094F8212032B1E218EDB24F
:109DD000013382F8235084F8203094F8202094F83E
:109DE00022309A420AD194F84630052B0ED0062B29
:109DF0000FD0002384F8213084F8203070BDA22DCC
:109E0000E1D1012284F821202322DAE7002004F0A6
:109E100049F894F824301E2BEBD10025294694F8FC
:109E20002220013AEBB2934208DB224492F823301D
:109E30009942DED1032004F035F8DAE70820234404
:109E400093F82330DBB281EA030616F0010F4FEAE4
:109E5000530300F1FF300CBFDBB283F08C0310F032
:109E6000FF00C1F34701EED101351946DAE700BF23
:109E7000581A00202DE9F041884600240C4B93E845
:109E8000E000054406440744444501DBBDE8F08199
:109E900037F9142036F9143035F91400134402222E
:109EA00093FBF2F3C01A06F071FC0134ECE700BF3B
:109EB00010150020064B1A684FF47A73B3FBF2F3C7
:109EC000C3EB431203EB8203DB000380704700BF48
:109ED0008025002002392DE9F843426804460368D2
:109EE000806806290DD8DFE801F004086A6D7275F4
:109EF000780022605B42636003E05B425242236071
:109F00006260384B1B78002B57D1206808F018FE90
:109F10008046606808F014FE0746A06808F010FE4E
:109F2000314D0646A96C404608F05EFE696D8146DB
:109F3000384608F059FE0146484608F04DFD296EA6
:109F40008146304608F050FE0146484608F044FD80
:109F50000BF0C4FBE96C2060404608F045FEA96D9B
:109F60008146384608F040FE0146484608F034FD78
:109F7000696E8146304608F037FE0146484608F0D3
:109F80002BFD0BF0ABFB296D6060404608F02CFE0A
:109F9000E96D8046384608F027FE0146404608F045
:109FA0001BFDA96E0746304608F01EFE01463846E6
:109FB00008F012FD0BF092FBA060BDE8F88352425E
:109FC000226098E75B4223604042A06099E72260EC
:109FD0006360F9E752426260F6E7524222605B42F8
:109FE000F6E700BF27000020581A0020F8B500242B
:109FF000084D094F05F17006B5F86C0008F09CFD9E
:10A000007A6B01463019243406F058FF6C2CF3D1DA
:10A01000F8BD00BF581A0020401500202DE9F04F70
:10A02000CF4B8BB01978CF4CCB1EDBB2142B00F288
:10A030005F81012202FA03F3CB4A1A40002A00F0A2
:10A04000578184F8DC104FF00008C84D1022002121
:10A05000C7480DF00EFE2320012685F85980C5F86B
:10A060001C80FCF7AEFD68230AAA6B7602F81B8DF4
:10A070002E763346752105F1140001F039F805F10B
:10A080001407C0B1BB4B0DF10E02EB65BA4B414654
:10A090002B663846334601F02BF89DF80E3003F05E
:10A0A0007E038DF80E30002800F02681682B40F0EA
:10A0B000238185F857600026B04B85F856609A7961
:10A0C000984685F8682095F85720022A40F092803B
:10A0D0000120AB4B98F803A02B60AA4B85F85600E3
:10A0E0006B60A94B88F807602B62A84B1A689946E9
:10A0F00002431A60BAF1000F03D0BAF1070F40F023
:10A100007881032398F80200DFF8B4B285F8533061
:10A11000431E85F8543008F013FD594608F064FDDD
:10A1200008F064FF924E85F852A030608F4800F02E
:10A1300013FE98F800300BB185F85630944D04F0BA
:10A14000DBF848220021284636680DF092FD97E89A
:10A15000070005F1080383E807008E4B05F1240E84
:10A1600093E807008EE80700012033F8053C94F8D7
:10A17000E120A5F81F3094F8E230E97FDFF844E2EF
:10A1800085F83030112A134628BF002300FA03F265
:10A1900012EA0E0F40F0328112F04D0F00F02E81C6
:10A1A000022940F02B817C4B79482B607B4B6B6004
:10A1B00095F82030002B0CBF6F236E232B770123E3
:10A1C000AB77D9F8003043F00203C9F800304FF400
:10A1D0008073AB8200F070FD4FF47A736B63B4F858
:10A1E0006C30002B40F0128194F8E030002B40F0EE
:10A1F0000B81012697E807000023694D4FF0000A04
:10A200002F464FF00108EB60664B83E8070094F897
:10A210000B311D46042D84F804A100F2088108FAD0
:10A2200005F313F01A0940F0048113F0050F00F054
:10A23000008194F80C01FCF773FD0AAB03F8189D3C
:10A2400000930123C4F814010A221E211846FBF7CB
:10A2500083FC002800F0ED809DF81030482B40F082
:10A26000E880514B6420C4F8F030504B474AC4F8A2
:10A27000F430032384F80431136843F008031360B7
:10A28000B4F9083193FBF0F500FB153000B208F08B
:10A2900057FC474908F0A8FC8246284608F050FCC5
:10A2A0000146504608F098FB424908F09DFC012108
:10A2B000F8600846FCF7ACFDD4F8F0309847494602
:10A2C0000120FCF7A5FD94F80A3184F81881002BD1
:10A2D00040F0B580384B1A785F79012A194600F0B2
:10A2E000B180022A00F0C68030460BB0BDE8F08F86
:10A2F000002384F8DC30A6E69DF80D3003F07E03E1
:10A30000682B8DF80D306ED1022385F85730062367
:10A3100004AA1946EE6D2948B0479DF815309DF8FE
:10A3200013209B00520002F0020203F004031343C7
:10A330009DF8112002F00102134345D0012B03D1F7
:10A34000002385F85830B6E6022B01D10123F8E747
:10A3500003F00303032BF9D00320FCF7B0FDAAE6BA
:10A360007A170020581A002021001100FC2200203A
:10A3700080250020F1B00008F3AD0008E82200209D
:10A3800059AD0008D3AC000890C1793D701700208A
:10A390004015002058230020B9AC000817AD000874
:10A3A00088150020501B00207DAE0008FFAD00087E
:10A3B0008988883C00002041E214002010230020FE
:10A3C0000000FA42B2FF01000123EE6D0DF10F0211
:10A3D0000C21AC48B0479DF80F3013F00F03BBD0F1
:10A3E000042BB3D1ACE7702B04BF042385F857309E
:10A3F00061E685F85360DFF8B0B289E6012B4FF0D3
:10A4000000023FF6BFAE1346AB77F2E60026DFF858
:10A410009C82B4F86C0008F08FFB6A6B014608EB75
:10A420000600243606F04AFD6C2EF2D1DCE600254B
:10A43000F0E6012D4FF000033FF6EBAE4AE784F85B
:10A44000043147E790490A70DA781B79013A0A71BA
:10A450004B71042F00F2BA8101A353F827F000BF1B
:10A4600099A40008E9A2000899A4000811A6000810
:10A4700041A600085B78844D013B5BB2012BCEBF47
:10A48000002304EB0313D3F81C312A706B60887827
:10A49000FCF746FCA860DCE794F83C81B8F1000FBB
:10A4A00040F0AB804046784DFCF77EFC1420FCF772
:10A4B00088FB2B78012B04D16A7912B97722984650
:10A4C0006A710DF10F07697995F90400012300976E
:10A4D000D022FBF7D9FB002800F0958003229DF8DD
:10A4E0000F30A4F86021552B84F8573140F08B8051
:10A4F000697995F904000123D1220097FBF7C4FB89
:10A500009DF80F30697903F00F021B0984F8593167
:10A5100004AB84F8582195F90400AA22009316236D
:10A52000FBF7B2FB9DF810209DF8113043EA02239F
:10A53000A4F840319DF812209DF8133043EA02231D
:10A54000A4F842319DF814209DF8153043EA022307
:10A55000A4F844319DF816209DF8173043EA0223F1
:10A56000A4F846319DF818209DF8193043EA0223DB
:10A57000A4F848319DF81A209DF81B3043EA0223C5
:10A58000A4F84A319DF81C209DF81D3043EA0223AF
:10A59000A4F84C319DF81E209DF81F3043EA022399
:10A5A000A4F84E319DF820209DF8213043EA022383
:10A5B000A4F850319DF822209DF8233043EA02236D
:10A5C000A4F852319DF824209DF8253043EA022357
:10A5D000A4F8543141F27073AB8146F67813EB81E5
:10A5E0002A4B2B612A4B6B612A4BAB612A4BEB61E7
:10A5F0002A4B2B62012384F83C31294A136843F02B
:10A600000403136070E6B8F1000F01D000236B71F2
:10A610001D4D0A20FCF7D5FA2F78012F2FD16B7929
:10A620006BBB77236B710DF10F030122A02116483C
:10A6300000F090FD814600283AD1002F40F0A6801E
:10A64000114D1420FCF7BDFA2F78012F40F0A180A6
:10A650006B79002B40F09D8076236B71114B0122AA
:10A66000D021094800F076FD94F87431582B00F0A1
:10A670009280002F3FF438AE00236B7134E6002740
:10A68000D1E700BF10230020C8150020E5AD000869
:10A6900089AC0008C5AD000841AC000867AB0008F4
:10A6A00070170020CC1B002000007A44C81A00203C
:10A6B0009DF80F30FF2BC0D04FF0000801221E2163
:10A6C000444800F032FD4FF42F60FCF76FFAC246A9
:10A6D000DFF800B1A8F1600104AB0222C9B258460C
:10A6E0008DF810A08DF811A000F034FD9DF8102019
:10A6F0009DF8113043EA0223374A28F8023008F166
:10A700000208B8F1100FE5D100231946B4F8722100
:10A7100002F00F0E02F47F42A4F8722121F0010032
:10A720002044B0F86401002818BF4FF0000911F070
:10A73000010F1ABFC0B2434083EA1023082013F46C
:10A74000004F18BF83F4C05301384FEA4303F6D1DA
:10A7500001311029E2D142EA0E02A4F87221B9F1C6
:10A76000000F7FF46AAFC3F303339E457FF465AFF8
:10A7700042F21073AB81EB81184B2B61184B6B616C
:10A78000184BAB61184BEB61184B1DE000236B714C
:10A7900056E7002762E7164B182288210D4800F083
:10A7A000D9FC3122F4210B4800F0BFFC0023AB811F
:10A7B000104B6B61104B2B61104BAB61104BEB617D
:10A7C00045F6D813EB810F4B2B6216E7012F7FF470
:10A7D00014AF89E5C8150020BC1B002049B1000852
:10A7E000ADB1000843B100089DB100080BA80008F6
:10A7F000D01B002065AB000829B100084FB100084C
:10A80000BDB10008ADA9000870472DE9F04F002246
:10A810000025634B634EB3F80AC087B034684FEA33
:10A820000C2A05901889B4EB0A0A65EB020BA0FB11
:10A830000A4500FB0B55B3F80480E00940EA456087
:10A840004FEA08440719D8888E464FEAE511A0FB65
:10A850000A4500FB0B5541EB0208CDE90278B3F83D
:10A860000280200A40EA05604FEAC83410EB040871
:10A870004FEA252141EB02099A89B446A2FB0A015D
:10A8800002FB0B11C20D42EA412212F5FA604FEAB7
:10A89000E15343F10001B0F5FA6FCDE9000171F128
:10A8A00000015DDADDE902670524A2FB040104FB77
:10A8B000031100FB03F402FB0144A0FB020121444D
:10A8C0004D104FEA3004361B4FEA900467EB050742
:10A8D00044EA81748D104FF0FF313348B8EB04081F
:10A8E00069EB0509DDE90045844275EB0101CDE91D
:10A8F000026722DA40F6AC50002112184B4102FBED
:10A9000003F1A2FB022303EB4103D900D000101A8C
:10A9100041EA527163EB0101341847EB0105CDE9BF
:10A9200002450B24A2FB040104FB031149104FEA6A
:10A930003000B8EB000869EB01090AFB0BF3DDE915
:10A940000001AAFB0AAB0BEB430B4FEADA7242EAB7
:10A950004B02801A4FEAEB7361EB0301CDE9000172
:10A96000DCF80410A1FB082301FB0933540D44EA71
:10A97000C3245D15DDE90223A21A65EB03031D461E
:10A98000D30B059A43EA454302B11360BEF1000FB1
:10A9900002D0009BCEF8003007B0BDE8F08F00BFBA
:10A9A000BC1B0020081C002024FAFFFF2DE9F74FF4
:10A9B0006A4CDFF8ACE123880091DEF80810B4F9A6
:10A9C0000480C3EB211252435B00C3EBE103B4F9F3
:10A9D000021005465943131308FB03F84FEAA83841
:10A9E00008EBE12101EB8102B1F5FA3802F18002B6
:10A9F0004FEAE1794FEA222349F1FF39B4F90820FF
:10AA0000A8FB08AB019308FB09F3A16102FB09F164
:10AA10000BEB430BD31708FB0311A2FB08230B44DA
:10AA20001F03160347EA1257B4F90A2002FB0BF181
:10AA3000D3170AFB0313A2FB0A011944020A42EAD4
:10AA4000016292194FEA2123E6887B410032A2FB82
:10AA5000060143F5004306FB03114A10CB1752EAE7
:10AA600003016FD0B4F91060B4F90E0006FB0BF1CE
:10AA7000F7170AFB0711A6FB0AAB00FB09F68B448C
:10AA8000C11708FB0161A0FB08898944DEF80C109E
:10AA90004FEA4846C1F5801E1AEB060A76464FEA91
:10AAA000494747EAD8374BEB070BF7170026F9075A
:10AAB00041EA5E014FEACE7040F6354EB4F90C80A3
:10AAC00016EB0A064FEAC80747EB0B07861B61EB3C
:10AAD0000707A6FB0E010EFB071108F0A7FAB4F951
:10AAE00016204E1302FB06FE470B47EAC147D31759
:10AAF00007FB03EEA2FB07235643734407FB0366E1
:10AB0000A2FB07233344560E46EAC3163218B4F9A3
:10AB100014604FEA636747EB01037143F71700FBCB
:10AB20000717A6FB00013944C60C46EA41369219C4
:10AB30004FEAE147B4F912607B41100A40EA036032
:10AB4000320112180DB1120A2A60009B13B11A4685
:10AB5000019B136003B0BDE8F08F00BFD01B002045
:10AB6000081C002070472DE9F041324E324F7489A5
:10AB70003B8AB6F914201B1B34890A255C43E31376
:10AB8000B6F912401A44E40294FBF2F41C44F46156
:10AB90006543A4F57A6404FB04F2B6F90430B6F90F
:10ABA00002E0B6F90E8004FB0EFE5C43B6F90C30F1
:10ABB000121302FB08F85A43121402EB64344CF2ED
:10ABC00050320234F3884FEAEE2EA41004F500440C
:10ABD0000EEBE828B6F900E0B6F920C0634308EBB5
:10ABE0008E0808FA0CF87E6908F10208DC0BA6EB67
:10ABF000A80642FA0CF373434DBFB3FBF4F35B00BA
:10AC0000B3FBF4F35B001A1202FB02F440F6DE32EF
:10AC100062430A4C12145C4302EB2442083502F6EC
:10AC2000CF622D1103EB221300B1036001B10D605F
:10AC3000BDE8F081981B0020081C002043E3FFFFC3
:10AC40001FB503AB4179F62290F90400009303236A
:10AC5000FBF71AF89DF80D309DF80C201B0243EA13
:10AC600002439DF80E201343054AB2F92020C2F199
:10AC70000802D340034A536105B05DF804FB00BFEE
:10AC8000981B0020081C00201FB503AB4179F62259
:10AC900090F9040000930223FAF7F6FF9DF80C20C8
:10ACA0009DF80D3043EA0223024A138205B05DF895
:10ACB00004FB00BF081C002090F8203013B1012BCA
:10ACC00004D070474FF48063838270474FF4006371
:10ACD000FAE737B506230446C56D6A4643211430AA
:10ACE000A847B0B101209DF800209DF8013043EA4B
:10ACF0000223A3879DF802209DF8033043EA022334
:10AD0000E3879DF804209DF8053043EA0223A4F868
:10AD1000403003B030BD37B506230446456A6A4665
:10AD20003B210830A847A8B101209DF800209DF8DC
:10AD3000013043EA0223E3829DF802209DF80330AC
:10AD400043EA022323839DF804209DF8053043EA5B
:10AD50000223638303B030BD70B5044600F11405CF
:10AD6000036E80226B21284698476420FBF729FF59
:10AD7000236E03226B2128469847236E94F85420B3
:10AD80001921284698470F20FBF71BFF236E94F8E4
:10AD900052201A2128469847236E18221B21284644
:10ADA0009847236E18221C2128469847236E0222BA
:10ADB000372128469847236E2846BDE87040012277
:10ADC00038211847064B417993F82030F4229B0133
:10ADD000343303F0FC0390F90400FAF75FBF00BFBF
:10ADE000981B002041792E23F42290F90400FAF7F1
:10ADF00055BF134601200A466821FAF74FBF7FB5B9
:10AE000002AB00930446062303221E210120FAF719
:10AE1000A3FE064668B39DF808309DF80900164D5C
:10AE200040EA032000B207F08BFE296807F0DCFE41
:10AE300008F0B6F89DF80A3020809DF80B0040EA33
:10AE4000032000B207F07CFEA96807F0CDFE08F0F1
:10AE5000A7F89DF80C30A0809DF80D0040EA032073
:10AE600000B207F06DFE696807F0BEFE08F098F8C2
:10AE70006080304604B070BD280000202DE9F0430A
:10AE8000322085B0FBF79DFE112300221E210120F8
:10AE9000FAF704FF0122002460231E211046FAF76E
:10AEA000FDFE6420FBF78DFE02A8FFF7A8FF0A2530
:10AEB00026462746DFF83482012302221E21184647
:10AEC000FAF7ECFE3220FBF77CFE02A8FFF797FFB3
:10AED000BDF90A30BDF90C101E448B42A8BF0B46C9
:10AEE000BDF908200C449342A8BF134643451744BC
:10AEF000C0F2E1800120FBF703FF013DDCD14FF000
:10AF00000108122300221E210120FAF7C7FE0A259C
:10AF1000DFF8D891012302221E211846FAF7BEFE5F
:10AF20003220FBF74EFE02A8FFF769FFBDF90A3099
:10AF3000BDF90C10F61A8B42A8BF0B46BDF90820CC
:10AF4000641A9342A8BF13464B45A7EB0207C0F211
:10AF5000B5800120FBF7D4FE013DDBD1384607F078
:10AF6000EFFD0146574807F0F3FE574D20F0004033
:10AF70002860304607F0E4FD0146524807F0E8FE3D
:10AF800020F000406860204607F0DAFD01464F4897
:10AF900007F0DEFE20F00040A860702300221E2192
:10AFA0000120FAF77BFE012220231E211046FAF72A
:10AFB00075FE002302221E210120FAF76FFE642095
:10AFC000FBF7FFFDB8F1000F04D14FF07E532B606B
:10AFD0006B60AB603E4C2168002968D03D4B3E4A17
:10AFE00093618B88B3FA83F3C3F11F03581C4FD0CE
:10AFF0004FF00F0E394E183246F82320DAB202F025
:10B00000030602F0FC0202F1804202F580329768EA
:10B010000968B6000EFA06FE27EA0E0701F1404164
:10B020009760A1F584319768C1F38721B140394316
:10B0300001272B489160C55C07FA03F3D943294ADD
:10B04000536116680E40166056680E4056601668CA
:10B050001E43166096680E409660D6683140D160F7
:10B0600091680B439360204B5A5DF02A10DDF0226B
:10B070005A5543191B7C01A88DF8043003238DF821
:10B08000053000238DF807708DF8063003F0A2F824
:10B09000236863B19B880122B3FA83F3C3F11F03D2
:10B0A00012FA03F31FBF0F490A6813430B60012014
:10B0B00005B0BDE8F0834FF0000822E74FF000082C
:10B0C0004CE700BF00406F462800002001C05E46EC
:10B0D0006C1B002009A80008081C0020A4100020F8
:10B0E000E08E010800040140E80A002001F0FFFFA3
:10B0F00007B5012000920A466821FAF72DFD03B03A
:10B100005DF804FB0346022210B41C7B1968A240C0
:10B1100040694A605A6810BC136823F001031B049D
:10B120001B0C1360FBF77CBD704713460278012AA5
:10B1300005D10A46417990F90400FAF7AFBD002025
:10B14000704701224821F0E701225821EDE7312222
:10B15000F421EAE713B50C460178012909D14179B8
:10B1600090F90400009313462246FAF78DFD02B0D1
:10B1700010BD0020FBE707B5032201AB0021FFF75C
:10B18000E9FF9DF805309DF804001B0243EA0043E7
:10B190009DF80600184303B05DF804FB08B5FFF7FF
:10B1A000EAFF014B586008BD081C002008B5FFF7F6
:10B1B000E2FF014B186008BD081C002007B50622FD
:10B1C0006B46F721FFF7C6FF9DF801309DF8001090
:10B1D0001B0143EA01339DF80210094A43EA1113A7
:10B1E000D3609DF804309DF803101B0143EA01333E
:10B1F0009DF8051043EA1113936003B05DF804FB5A
:10B20000081C0020C26C70B515880446ADB2A906B2
:10B2100006D5036B23B9C36AA3B1908880B298475F
:10B220002B0620D5636AA26A9A42E36C17D0511CA0
:10B23000A069A162825C9A802369994213D300239A
:10B24000A36270BDE169928840694E1CD2B2E6618A
:10B250004254E169E268914228BFE361E0E7DA68BD
:10B2600022F08002DA6070BD70472DE9F8430D4688
:10B2700016468146002440F634074FF01908484628
:10B2800005F0B7FE814690B10AF09AF8B842A8BF1F
:10B290003846B0F5617FB8BF4FF46170A0F56170BA
:10B2A00090FBF8F04CB928703378013333700134D7
:10B2B000022CE4D14846BDE8F8836870F4E72DE934
:10B2C000F04F07468A46164600248FB0DFF86080AC
:10B2D0000DF124095AF82430494602A8029303F0DC
:10B2E00096F916B356F82430029D0393EB1A5D428B
:10B2F0000DF1100B5D41594603A803F088F9CDF814
:10B3000000B0234642462946384606F019F823463F
:10B31000CDF80090424629463846013406F026F81A
:10B32000202CD7D10FB0BDE8F08F3546EFE700BF36
:10B33000B8A901082DE9F34781460F469046022639
:10B340000024DFF860A0B8F1000F28D037F82420DF
:10B3500038F824309A4238F806201ED1BD5BA91A6D
:10B360004D424D410192009352462346294648469C
:10B3700005F0E6FFBB5B5246019337F824302946BF
:10B38000009348462346013405F0F0FF042C06F1F3
:10B390000406D8D102B0BDE8F0870025E2E74546B3
:10B3A000E8E700BFC2A901082DE9F04F81469046A9
:10B3B0000C46154600261927DFF8B0A087B0B8F173
:10B3C000000F51D023782A7893422B794AD16078A4
:10B3D0006978884246D1A078A978884242D1E0783D
:10B3E000E97888423ED1217999423BD161796879E7
:10B3F000081A414241410593EB7848460493AB78E3
:10B400008B467B4303F5617303936B7801927B4317
:10B4100003F5617302936B7952460093334605F04E
:10B420008FFF237952460593E37859460493A37816
:10B4300048467B4303F561730393637806357B438A
:10B4400003F56173029323780634019314F8013CE9
:10B4500000933346013605F089FF0F2EAFD107B0B8
:10B46000BDE8F08F0021C6E7C346DAE7D3A901089B
:10B470002DE9F04F814690460C46164689B002F100
:10B480001003DFF8D0A0324FDFF8CCB0079394F967
:10B4900002209AF90630934203D09AF90E30934273
:10B4A0004BD1B8F1000F01D145462DE096F902309D
:10B4B00071799A42328849D12088904246D1E57804
:10B4C000F078854242D12579307985423ED1A579FF
:10B4D000B07985423AD16579681A4542454157F8B5
:10B4E000211048460491B17957F821100391317920
:10B4F00057F821100291F178009257F821105A461E
:10B500000191294605F01CFF627994F9023057F841
:10B51000222029460492A279484657F82220039215
:10B52000227957F822200292E27857F822200192DD
:10B53000228800925A4605F019FF079B08369E4262
:10B5400004F10804A3D109B0BDE8F08F0025C6E7D7
:10B550003082010890250020F1A901082DE9F04F63
:10B56000814690460C46154600261927DFF8A8A00C
:10B5700085B0B8F1000F4CD028782378834246D1AB
:10B5800062786B789A4242D1A278AB789A423ED1E7
:10B59000E178EB78CB1A594259418B4606F04BFCC7
:10B5A00098B1EB7852467B4303F561730393AB7814
:10B5B00059467B4303F5617302936B780193037AD9
:10B5C00048460093334605F0BBFE207806F033FC76
:10B5D00098B1E37852467B4303F561730393A378F4
:10B5E00059467B4303F56173029363780193037AB1
:10B5F00048460093334605F0B9FE0136142E04F197
:10B60000040405F10405B4D105B0BDE8F08F0021B4
:10B61000C3E7C346D9E700BF0EAA010820B10078EE
:10B62000B0FA80F040097047012070472DE9F04FD3
:10B6300087B00546FFF7F2FF044638B100225649AD
:10B640000120FFF73CFE07B0BDE8F08F284609F067
:10B65000B7FE1F28074600F39780284605F0C9FC6F
:10B66000A0460646A246A1462546A3464A4B00945C
:10B6700043F827400193494BE1B2E05C00230DF110
:10B680000C0CB64616F8012B1AB190420FD00A2BBB
:10B6900009D106AE33440026904203F80C6C08D062
:10B6A00005F07CFECFE703F80C200133E9E7024602
:10B6B000EFE701390EF10106032932D8DFE801F086
:10B6C0004E1F025B4FF0010EDFF8E4C00DF10B00DE
:10B6D00010F8011F49B30023314AD25C8A4203D0DB
:10B6E0000133072BF8D15346002212F80CA08A45EB
:10B6F0003DD10EFA02F248EA02089A46E8E74FF016
:10B70000010C0DF10B0111F8012F72B10023254836
:10B7100013F800E0964526D10CFA03F349EA030931
:10B72000F1E703A809F04CFE83460134052CA2D1B1
:10B73000009B05F00F0545EA834545EA895949EA2A
:10B740000A2A4FEA0B134AEA0838019ADBB248EAA0
:10B75000030342F8273004F095FD74E703A809F0CD
:10B760002FFE0546E1E70133062BD0D1CBE70132AE
:10B77000062ABAD1C1E703A809F022FE03460F2822
:10B78000C8BF00230093D0E71F232246064907487D
:10B7900005F08AFD57E700BF84110020F88E0108EC
:10B7A0005694010850940108299E0108609D0108E3
:10B7B0005D9401082DE9F0410546FFF72FFF06468D
:10B7C00028B1BDE8F041002227490120B2E5274910
:10B7D00028460CF056FA70B94FF47A714FF4FA62B9
:10B7E000214B19805A809980DA8019815A81998178
:10B7F000DA81BDE8F081284609F0E2FD032804461D
:10B8000029D8284605F0F5FB064658B109F0D8FDC1
:10B8100001270546304605F0ECFB30B9BDE8F041A4
:10B8200005F0BCBD05460746F4E709F0C9FD002F49
:10B83000F4D040F2DC53A5F2EE229A42EED8A0F208
:10B84000EE229A42EAD8084B23F8245003EB8403F3
:10B850005880BDE8F0813246BDE8F0410323044939
:10B86000044805F021BD00BFAA22002012A3010850
:10B8700076A20108609D0108F7B50746FFF7CEFEE6
:10B88000044630B1002236490120FFF78DFD03B098
:10B89000F0BD384609F094FD0E28054659DC062611
:10B8A0004643781C8DF8074005F0A3FB2C4C074657
:10B8B00050B109F085FD032806D8A31958719DF8E9
:10B8C000073001338DF80730384605F092FB074604
:10B8D00058B109F075FD0D2807D806236B43E054D5
:10B8E0009DF8073001338DF80730711C0DF1070208
:10B8F00021443846FFF7B9FC05F07BFB074660B1F1
:10B9000009F05EFD182808D8062303FB0543D8700C
:10B910009DF8073001338DF80730384605F069FB94
:10B9200060B109F04DFD0D2808D8062303FB05453D
:10B930009DF80730287101338DF807309DF80730E6
:10B94000062BA4D00023A219A351938005F026FD55
:10B950009DE70E2322460349034805F0A5FC96E720
:10B960007C1E0020299E0108609D01082DE9F04FF2
:10B9700085B00346FFF752FE054620B105F00EFDE7
:10B9800005B0BDE8F08F03AA5E49184609F074FDC2
:10B990002C460646A8464FF0FF37DFF89491DFF8B3
:10B9A00094A1DFF894B1B6B95748394605F049FB80
:10B9B000564B78B293F90620824200F0898093F9C1
:10B9C0000E20824200F08380B8F1000F33D150483E
:10B9D00005F0DEFCD4E7012D0ED0022D11D01DB9EB
:10B9E000304609F0EDFC074603AA4649002009F05D
:10B9F00043FD01350646D6E7304609F0E1FC8046B6
:10BA0000F2E7494630460CF0B6F920B941493046D4
:10BA10000CF0B1F908B144F00104514630460CF085
:10BA2000AAF928B9594630460CF0A5F90028DBD010
:10BA300044F00204D8E7002C08BF03240022E4B23B
:10BA4000019200944346114603F08EF9054608B969
:10BA50003148BDE74146314805F0F3FA304805F07A
:10BA600097FC304B1C68204603F04EF9284603F043
:10BA70004BF900210846FBF7CBF900210120FBF729
:10BA8000C7F92046FBF717F970B101210020FBF739
:10BA9000BFF92046FBF70CF901462846FBF70EF9E3
:10BAA00000210846FBF7B4F92846FBF704F9002803
:10BAB000E7D001210020FBF7ABF92846FBF7F8F8A7
:10BAC00001462046FBF7FAF800210846D7E708337D
:10BAD0001D68002D3FF478AF134805F059FC54B1B0
:10BAE00069798C4207D01148224605F0AAFAE1B2E2
:10BAF0002846FBF7D7F8EB6A002BAFD00023EB62A8
:10BB0000ACE700BF319C010827AA0108902500205E
:10BB100030AA01086F9F010846AA01085BAA010824
:10BB20009CAA01086819002070AA01087EAA0108D1
:10BB300021AA010824AA0108AEB001082DE9F341A9
:10BB40000346FFF76BFD044630B100220120364961
:10BB500002B0BDE8F0418BE40090019018465E1CF5
:10BB600009F02EFC304D40B295F90230834257D097
:10BB700095F90A30834252D02546304605F039FA0D
:10BB8000074628B109F01CFC0134ADF80000E4B20E
:10BB90000026DFF89880384605F02BFA074600B3F8
:10BBA00009F00EFC002258F82210D3B2884203D0CC
:10BBB0000132102AF7D1002358F82320904210D1E7
:10BBC000022E1AD0032E1DD05A1E012ED2B20FD033
:10BBD0000B2A03D88DF803300134E4B20136042E69
:10BBE000D9D1052C14D802B0BDE8F04105F0D6BB80
:10BBF000042AF3D88DF80430EEE7052BEED88DF843
:10BC00000630E9E79A1E0D2AE8D88DF80530E3E7FB
:10BC10006B4603CB2860696002B0BDE8F08108354F
:10BC20008DF802000124A8E7A22500203082010837
:10BC3000F7B50746FFF7F2FC044630B100222C4965
:10BC40000120FFF78BFC03B0F0BD384609F0B8FBCC
:10BC5000132805463ADC8600781C8DF8074005F06D
:10BC6000C8F9074690B109F0ABFB4FF00C0E214B21
:10BC7000C0B203F108010EFB04F201EB020C9CF8C8
:10BC800008C0844529D00134252CF4D1384605F06C
:10BC9000B0F9174C074650B109F092FB0D2806D8B1
:10BCA000A31958709DF8073001338DF80730B11C87
:10BCB0000DF1070221443846FFF7D7FA9DF8073007
:10BCC000042BC0D0002344F82530BCE713232246C0
:10BCD00009490A4805F0E8FAB5E713441A7A044B13
:10BCE00003F825209DF8073001338DF80730CDE7A4
:10BCF000DC1D0020F88E0108299E0108609D0108C6
:10BD0000F7B50646FFF78AFC054678B100242546BC
:10BD10000A2201A92046FBF7F5F90134057001A8B4
:10BD2000FFF7EEFF122CF3D103B0F0BD304609F05F
:10BD300047FBC4B2112C5DD8701C05F05AF9304D88
:10BD40000746B8B92F4B13F814108A1E51425141BF
:10BD50002C4B13F81420AA5C002946D003EB4403B3
:10BD6000597819234B432146274803F2EE2305F067
:10BD70009BFAD9E7017828460BF0A1FF60B1032CAC
:10BD80008CBF03220022214B401BC0B21344184435
:10BD900090F8C461032E02D105F000FBC4E73846D9
:10BDA00005F027F9F0B1022EF6D109F009FB40F6B3
:10BDB000CA0280B29042A8BF104640F2EE229042E2
:10BDC000B8BF10461922A0F2EE2090FBF2F00D4B06
:10BDD00003EB44035870B31E59425941094B03F811
:10BDE0001460B5E7022EF6D1D6E72146084805F0E3
:10BDF0005BFA99E711232A4606490748B7E700BFCF
:10BE0000989301085D220020BDAA0108F88E010860
:10BE1000CDAA010876A20108609D01087FB5094BF3
:10BE2000094A0493094B0A4903930A4B0A480293AF
:10BE30000A4B01930A4B00930A4B05F035FA07B001
:10BE40005DF804FB65AC01084497010850970108B0
:10BE5000199701085A9701083AAC0108639701083D
:10BE600013970108291C002038B50A4B0D4603EB37
:10BE7000C00494F8C020084853F8221005F0E1F8F7
:10BE800094F8C6302BB1691C0448BDE8384005F071
:10BE9000D8B838BDC4900108BB9D010850B3010853
:10BEA0002DE9F04F00252F46AA465D4E8BB05D4B25
:10BEB0005D49DA680023934222DB0135102D06F13B
:10BEC0003406F4D15749CB78BBB14FF47A73486D3F
:10BED0008A6DB0FBF3F35209C96D544805F0E4F9DB
:10BEE0000A2297FBF2F39AFBF2F102FB1377504818
:10BEF000009702FB11A205F0D7F90BB0BDE8F08F57
:10BF000051F82300864222D00133D4E74346079AF2
:10BF10000121484805F095F84C463AE038B106F062
:10BF20000FFE0146444806F013FF07F039F80446B7
:10BF300042462946414805F084F84FF0000928E0C0
:10BF4000584631E021463E4805F0AEF95AE07368A4
:10BF5000012D0793336BD6F800800893B36AD6F8A7
:10BF60002CB00993F069D9D138B106F0E9FD01464A
:10BF7000314806F0EDFE07F013F8324B81461B788E
:10BF8000012B90FBF3F4C1D9424601212B4805F067
:10BF900058F8BBF1000FD3D041F288314FF47A70DA
:10BFA0000BFB0411B1FBF0F0099B5B091DBF41F2D3
:10BFB00088324FF47A7103FB04221A4618BFB2FB91
:10BFC000F1F21849052DC9781CBF8244BF18002919
:10BFD000B8D04FF47A7E0899B1FBFEF104910A21A2
:10BFE00092FBF1FE01FB1E22039290FBF1F201FB9A
:10BFF000120100920191CDF808E05A4621461248FC
:10C0000005F052F9012D7FF458AF0E4B1B78012B30
:10C010007FF653AF4A4607990C4805F045F94CE7BF
:10C0200034000020241C0020341C0020C0AC010877
:10C03000E0AC010879AC0108002474496AAC01083D
:10C04000BCAC0108892200208CAC0108B0AC01080E
:10C05000374B2DE9F34119684FF47A733548B1FB3A
:10C06000F3F105F021F9344B344F1A78344B35494C
:10C07000354C03EB8203D3F8483197F860200988E8
:10C08000324805F011F9324BD4F840133148B1FB76
:10C09000F3F104F0D6FF05F082F8B7F862602E4A9B
:10C0A0002E492F4805F000F92E4A2F4BB6B2D31A6D
:10C0B0003146B7F864202D4805F0F6F8266D254680
:10C0C000002E33D0304606F03BFD0146284806F0EE
:10C0D0003FFE06F065FF8046D5F8EC0038B106F06B
:10C0E0002FFD0146224806F033FE06F059FF0446B4
:10C0F000E86938B106F024FD01461D4806F028FE27
:10C1000006F04EFFB7F86610434664290190A8BFB9
:10C11000642100943246174805F0C6F8164B1748BC
:10C12000198802B0BDE8F04105F0BEB8B046D3E7CB
:10C13000C41300200EAD010869130020241C002048
:10C14000C4900108B41500203400002028AD010877
:10C1500040420F004EAD01080050002000080000D2
:10C160005EAD01080000020800F8010882AD010878
:10C1700000247449BCAD0108A413002002AE0108DC
:10C180002DE9F04F0746304C87B023782F4A60885E
:10C1900052F82380FAF766FF2D4BD0F804A093F8ED
:10C1A000683082689BB1D3469246012607F040036F
:10C1B0000593A379721E002B08BF0123934208DC6C
:10C1C000244B08349C42E0D107B0BDE8F08F9B4679
:10C1D000EBE7A38813441AF803501BF80330EA1A5C
:10C1E000D2F1000949EB020993B9009643461A4A75
:10C1F0004946384605F0A4F8C5B9059B33B9009601
:10C200004346154A4946384605F0B0F80136D0E7AE
:10C2100003F00F021B09403302920193009643463C
:10C220000E4A4946384605F08BF8E5E705F00F035E
:10C230002D0940350293019500964346074A494629
:10C24000384605F093F8E1E784910108C4900108AD
:10C25000241C00200C9201081DAE010831AE01081B
:10C260002DE9F04F89B0074605F0FAFE044628B9DB
:10C270004120FFF785FF09B0BDE8F08F02469249E3
:10C2800038460BF02AFD914D0646002849D19048CA
:10C2900005F07EF88F4CDFF87482DFF8749204F5B5
:10C2A0008C77A2882168B2FA82F201F14041A37929
:10C2B000A1F58431890A413155F82330C2F11F02BA
:10C2C000404604F0BEFEE17911B1484604F0B9FEE3
:10C2D000083404F064FFA742E3D104F060FF7E4815
:10C2E00005F056F87D4CDFF82C82DFF82C92DFF851
:10C2F0002CA2237E013632460121404655F8237098
:10C3000004F09FFE627E39463AB1504604F0CCFFFD
:10C31000072E04F11C04ECD1ADE7484604F0C4FF3D
:10C32000F6E7384607AA6E4909F0A6F805F1C007F6
:10C3300082460026B84617F83630224655F82310B4
:10C3400050464FEAC6090BF0C8FC30B10136112E39
:10C35000F1D1644805F01CF88DE707AA604909F09F
:10C360008BF8044609F02CF84D4495F8C630074682
:10C37000EBB9002829DCC844B8F80200FAF772FECD
:10C38000FBB20193019AB8F8043027781344029362
:10C3900043680393002F00F09380534920460BF02D
:10C3A00070FCE0B9039B029A98545048D2E70028E9
:10C3B00005DD1A46BA420ADA002B08BF0123012222
:10C3C0004B494C4804F070FF55E70122F2E707AAF9
:10C3D0004349002009F050F8013F0446CBE7A7F19C
:10C3E0004105EDB2072D04D9A7F16105EDB2072D86
:10C3F00066D8601C08F0E4FFC3B20F2B82465FD8FA
:10C400006C1C40EA0414E4B22046FAF789FC0028C8
:10C4100056D0002C49D04FF0000823094033049334
:10C42000DFF8FC9004F00F03059300272FE0B9F824
:10C430000200FAF717FEB9F8043042683B44D15CB9
:10C44000A14223D1464504D101998F421ED000213B
:10C45000D154059A0499284804F0F3FD5FFA87FB4C
:10C460005FFA88F3594618460093FFF7FDFC4645EE
:10C4700009D1224804F0E5FD00985946FFF7F4FC85
:10C480001F4804F0DEFD1F4804F082FF013799F8D1
:10C490000630002B08BF01239F42C8DB08F10108CA
:10C4A000B8F1110F09F10809BFD15FFA8AF205F15D
:10C4B0004101154804F0F8FE039B029A9C54DAE609
:10C4C00004F06CFFD7E600BFBE9D0108C4900108D0
:10C4D00047AE0108901C002055AE010878030020EB
:10C4E000319C010873AE01082CAE01087BAE010837
:10C4F000299E0108609D010881AE0108A5AE0108D2
:10C50000A8AE010859AA0108B2AE01084AAE010856
:10C5100050B301085AAE0108BA9D01086CAE01087B
:10C52000849101082DE9F04F0D468DB0CB490446AA
:10C53000FDF79CFA0646002840F08281C849204653
:10C54000FDF794FA0646002840F07C81C549204654
:10C55000FDF78CFA0646002840F076812046C24955
:10C56000FDF784FA0028064612BF08242646012457
:10C570000DB144F01004BD4DBD4FBD42C0F0668109
:10C580000123BC4D85F8683000F0D0FDBA49304633
:10C59000FDF76CFA08B144F0200414F0090F00F024
:10C5A00036810020FFF73AFC04F01803182B04D161
:10C5B000B24804F06FFD04F0F2FD4FF0000995F869
:10C5C0008431AF4A002B08BF0121AE4B1CBF0021B4
:10C5D00013462046AC4A04F0C9FE2046FFF7D0FDC2
:10C5E000DFF8ECB2D5F89871D5F89C81A74B53F8D9
:10C5F0002960002E40F07E8168EA0703DFF8D4B29C
:10C600000293A24B53F826A0BAF1000F40F0938199
:10C61000D5F8A071D5F8AC3156467B40DB43DFF846
:10C62000B892DFF8B8A20393304602F0B9FD039B3D
:10C63000974A034214BF4FF001084FF0000817EA71
:10C64000000302934FF00C0303FB0623D3F808B05A
:10C6500014BF4A4652465B464146204604F070FEEF
:10C66000029A5B46002A14BF52464A46414620467B
:10C67000013604F07BFE132ED6D101270023854E10
:10C68000DFF85CE2DFF85CC29A5D13F80E100CA8CC
:10C69000104400F8201C13F80C000DF13008804401
:10C6A00008F8101C2FB1A2EB0008D8F1000747EBE7
:10C6B00008070133082BE7D1002608AB764A394634
:10C6C00020468DF8186004F03BFE04AB724A3946F0
:10C6D000204604F04BFE714A71492046FEF7C8FE21
:10C6E000704A71492046FEF7EAFD704A70492046BB
:10C6F000FDF792FA6B4A6C492046FDF7D5F96D4A71
:10C70000204602F15001FEF729FF6B4A204602F154
:10C710005A01FEF749FE694A69492046FEF70AFEBA
:10C720004FF00108DFF8C0A1DFF8C0B17300029339
:10C730001AF816201BF816309A4240F0238118F898
:10C740000A7018F80B10781A47424741022ADFF89E
:10C75000A09140F0198119211BF808204B444A434D
:10C7600093F8D43202F2EE2201920093554A3346F6
:10C770003946204604F0E4FD192218F80A303946FB
:10C78000534303F2EE230193730013F80A304D4A2A
:10C79000994499F8D43220460093334604F0E6FDDC
:10C7A0000136122E08F10208C0D12146002004F003
:10C7B000FBFC210740F100812146002095F80C6325
:10C7C000FDF740F921460120FDF73CF92146022002
:10C7D000FDF738F9304600F097F93B48FCF74EFE7C
:10C7E0002146002095F80D63FDF718F92146012038
:10C7F000FDF714F921460220FDF710F93046FCF749
:10C800008FFC3148FCF71AFE304804F043FCA207C5
:10C8100004D5214695F80C03FDF714F9630704D5F8
:10C82000214695F80D03FDF7F9F8104C104B9C428A
:10C83000C0F0CD80002385F868300DB0BDE8F08FE2
:10C84000012495E6022493E6042491E66A88696847
:10C85000A86808F0DDFD14358FE600BFD3AE0108EF
:10C86000E3B20108BA980108DAAE0108B8B80108C5
:10C8700000BC0108241C0020DEAE0108E7AE010860
:10C88000A81D0020F99D0108FB9D010820920108C8
:10C890009C920108B0170020A19D0108A22500204C
:10C8A000E225002084110020E01300200412002063
:10C8B00060140020DC1D00207C1E0020AA22002025
:10C8C0009A220020BDAA01085D9C0108F2AE010871
:10C8D000F7AE010803AF0108BEAE0108C8AE0108FB
:10C8E0001894010880170020BA2200205D22002041
:10C8F000C49001083378DBB14FF0010A68EA0703FE
:10C900000AFA09FA13EA0A0F14BF0121002133467B
:10C910005A46204604F014FD67EA080313EA0A0F9A
:10C920005A46334614BF01210021204604F01EFD63
:10C9300009F101095AE69AF800300BB34FF00109EA
:10C9400009FA06F918EA090F0BD067EA080313EA97
:10C95000090F5A46534614BF01210021204604F016
:10C96000EFFC17EA090F0BD0029B5A4613EA090F96
:10C9700018BF0121534608BF0021204604F0F6FCF1
:10C9800001363EE60027E1E64B4493F8D4323946BF
:10C990000093124A3346204604F0D2FC104B72003A
:10C9A0009B5C3946994499F8D4320C4A009320464E
:10C9B000334604F0DBFCF3E6214695F80C03FDF763
:10C9C00041F8214695F80D03FDF728F81FE7628826
:10C9D000A168606808F01CFD143427E7CDAA01089F
:10C9E000BA22002038B50546064C206800B938BD8B
:10C9F0004368EB1A002BFADB8368236003689847CF
:10CA0000F3E700BFFC21002000231A4630B5084C94
:10CA1000037219198D79AD0742BF0979815401322A
:10CA2000D02B03D0072A03F11003F2DD30BD00BF85
:10CA300014960108002210B5064C04EB02118B7904
:10CA400013F0010302D00B79037010BD01320E2ADE
:10CA5000F3D1F9E71496010808B50B4B18201978A3
:10CA600000231D46094C8B4207DB40F2DC50FAF7ED
:10CA70009DF8074A074BDA60FEE700FB03F2125904
:10CA800002B115800133EEE7A01500206C190020DB
:10CA90000400FA0500ED00E080B501210220FAF75C
:10CAA000B7F9144B1B7803F00503052B12D1124B79
:10CAB0000024186806F074FA104B114F1D7806B266
:10CAC000AC4210DB0F4B1B780BB102F087FE32201B
:10CAD000FAF777F800210120FAF79AF900210846C1
:10CAE000FAF796F9FEE7304606F02AF847F82400F0
:10CAF0000134E5E7941F0020541A0020A0150020FF
:10CB0000A4150020D80D0020022828BF0220064BC3
:10CB1000064A18704E2303FB0023054A0130C0B2B9
:10CB2000136002F00FBC00BF241C0020422B002029
:10CB3000741700202DE9F04F8BB001F093FA032613
:10CB4000DFF840914A4FA7EB09071822002104A8FB
:10CB50000BF08FF8474B484ACDF8109005975A6074
:10CB600002F188325A6001228DF824203422DA60E2
:10CB7000424B02221B88694604A8ADF80030FAF740
:10CB800033FA022269464FF6FF7004F0D0F94FF0F5
:10CB9000000B80463A4CDFF8F0A0544536D3002510
:10CBA0000AAC24F8245D0222214604A8FAF71CFAF4
:10CBB00002222146404604F0BAF940BAC04302229C
:10CBC000ADF8080002A904A8FAF70EFA079860B1B8
:10CBD00006ABC0F10402294618440BF04AF8069946
:10CBE00004A8FAF792F9079508909DF82430089A5E
:10CBF00023B120490B6943F080030B61013E2DD026
:10CC0000002AA2D1FAF748FA50B32CE0658802A9AD
:10CC1000C5F30B05AB1DADF80830238804A8C3F39A
:10CC20000B02ADF80A201B0B06228DF80C308DF894
:10CC30000DB0FAF7D9F9062202A9404604F077F9B7
:10CC4000804661682A4604A8FAF7CEF96168404632
:10CC50002A4604F06CF9143480469EE7002AD1D0AD
:10CC60000520FAF72CF901F0E5F90BB0BDE8F08FDB
:10CC700000000208002002402301674508940108D3
:10CC8000B8B8010800F8010800BC0108F8B53D4B30
:10CC90005A899989914228BF0022198A28BF5A814E
:10CCA000DA89914228BF0022D97828BFDA8139B1C8
:10CCB000072905D0012234489A7002700022DA71E7
:10CCC000D8799A78002830D0102AB8BF10229A70EC
:10CCD0002E4A92F857200A2A2BD00C2A0CBF2C4C33
:10CCE0002C4C29B1072903D00A2A14BF2A4C2B4CFB
:10CCF00000B12B4C2B4DAA78022A97BF2A49284E07
:10CD000001EB82014E682979A9B1013A032A37D88B
:10CD100031464FF07E5006F01BF808F0DFFC2B8800
:10CD2000984228BF18462880F8BD032AB8BF0322BE
:10CD3000CDE71E4CD5E7987805F002FF214605F0B7
:10CD400053FF0746104D2C78204605F0F9FE394672
:10CD500005F04AFF0146304606F002F980B1394637
:10CD6000304605F0F5FF06F01BF91028A8BF10208B
:10CD70000128B8BF0120C3B29C4298BF04462C7062
:10CD8000F8BD00BFE822002089220020FC220020FC
:10CD90000AD7A3396F1203396F12833A0F506E3AD4
:10CDA0006F12033804160020089401085304E93870
:10CDB0002DE9F04701F056F9B34CB44FDFF8548336
:10CDC000BC422DD2B24D00E015462E88002E00F058
:10CDD0005281AA19424580F04E81052E40F24B81C6
:10CDE00023886988C3F30B039942EDD16B799B07C4
:10CDF000EAD16168204695F80490FAF70EF9238885
:10CE0000B9EB133F0AD16388B21FC3F30B039A42F5
:10CE1000A8BF1A46A91D606808F0FAFA1434CFE7D3
:10CE20009C4C6378022B84BF002363702378022B11
:10CE300084BF00232370984B9A78042A40F0108115
:10CE40001A8AB2F57A7F02D24FF47A721A82934D1F
:10CE5000934A2B681A4012B943F008032B602B68E1
:10CE6000D80702D58F48FAF70FF92B68590402D575
:10CE70008D48FAF709F92B681A0702D58B48FAF79B
:10CE800003F92B689B040FD58948FAF7FDF84FF496
:10CE90000040FAF7F9F8874B40209A79012A04BF3D
:10CEA00000229A71FAF7F0F8834E00273368DFF812
:10CEB00060825A8C998C3D46914224BF00225A844C
:10CEC000FFF7E4FEC2464FF0FF0937F80820530889
:10CED00003F07733900800F03330D31A1B1AD008D0
:10CEE00000F011301B1A03EB231303F00F3393FBF5
:10CEF000F9F012F00101C0EB002018BF0135A3EBDF
:10CF0000000318BFEDB2012B0DDD022B40F0B880FD
:10CF100011B112F42F7F06D10AEB0700FAF74EFD8C
:10CF2000002800F0AD800837102FCED1013D022D32
:10CF300000F2A6804020FAF7A7F88020FAF7A4F8BC
:10CF40004FF40070FAF7A0F84FF48040FAF79CF81D
:10CF50004FF40030FAF798F84FF48020FAF794F87D
:10CF60005648FAF791F84FF40010FAF78DF84FF0A1
:10CF70000070FAF789F84FF08060FAF785F84FF003
:10CF80000060FAF781F84FF00050FAF77DF8637807
:10CF9000022B05D80C214A4A01FB0323494A13609E
:10CFA0002378022B9FBF4E21474A01FB03233360A6
:10CFB00004F082FA3022002144480AF05AFE306818
:10CFC00001F068F8002004F0EDF9414A414B117975
:10CFD000642280F001004A43187034683E4BC83226
:10CFE0001C603E4B5A6000229A60DA601A615A61F6
:10CFF0009A61DA6183F8202083F82120384B394A7E
:10D00000136033F8062C384B1A80384B5B6B0BB12E
:10D01000FCF7ECFF364D374B68881E8805F090FD15
:10D02000354905F0E1FD354C6060A88805F088FDC4
:10D03000314905F0D9FDEB79314A2372AB79206093
:10D040006372304B30461A6005F07AFD01462E4877
:10D0500005F07EFEBDE8F0472C4B186000F0EABFFB
:10D06000002A7FF4F4AE1A88B2F5F07F84BF4FF443
:10D07000F0721A80EBE661682046F9F7CEFFCDE644
:10D08000234801F08EFD55E7B8B8010800BC01083F
:10D0900002F80108241C002004160020C01D0020F6
:10D0A000096000020860000209200002016000021D
:10D0B000094000026E1300207417002020001000A9
:10D0C000080D0020982F0020422B0020680F002020
:10D0D000482A0020000000209C0F00208013002020
:10D0E0003C1B0020E0300020C41A00204015002026
:10D0F000941F0020800C002017B7D138042A00208C
:10D100003661023D302A0020C0C9FB48840C002053
:10D11000A22500200000020808B5FFF70BFDFFF76D
:10D1200047FEBDE80840012002F00CB938B50C4CB0
:10D130000C4DAC420DD300220B4B0C481A705A70A8
:10D140000B4B0C4A0C491A60BDE83840086003F0EC
:10D1500099B861682046F9F760FF1434E9E700BF29
:10D16000B8B8010800BC0108241C0020422B002094
:10D17000982F0020080D00207417002070B50C298E
:10D1800048D8DFE801F00747474748474747844703
:10D190004747BE00038C158823F001031B041B0CBA
:10D1A0000384038C8488018B23F0020321F0730134
:10D1B0000904090C2943568815891B0435431B0CA7
:10D1C0002B43674DA4B2A8429BB20FD005F5006572
:10D1D000A8420BD005F54065A84207D005F580654B
:10D1E000A84203D005F58065A8420ED1558923F0E9
:10D1F00008032B43958823F004032B43D689958994
:10D2000024F4407435432C43A4B2D2888480018333
:10D210008286038470BD038C148823F010031B04E2
:10D220001B0C0384038C8588018B23F0200321F4DD
:10D23000E6410904090C41EA0421568814891B04BB
:10D2400034431B0C43EA0413454CADB2A04289B2EF
:10D250009BB203D004F50064A04213D1548923F09B
:10D26000800343EA04134FF6BF741C409388D689A9
:10D2700044EA0313948925F44065344345EA840560
:10D280009BB2ADB2D288858001830287C1E7038C4F
:10D29000148823F480731B041B0C0384038C85887F
:10D2A000818B23F4007321F073010904090C2143DD
:10D2B000568814891B0434431B0C43EA0423284C6E
:10D2C000ADB2A0429BB203D004F50064A04213D1DA
:10D2D000548923F4006343EA04234FF6FF341C40CF
:10D2E0009388D68944EA0323948925F4405534432E
:10D2F00045EA04159BB2ADB2D288858081838287CE
:10D3000087E7038C158823F480531B041B0C0384CC
:10D31000038C8488818B23F4005321F4E6410904B3
:10D32000090C41EA0521568815891B0435431B0C5D
:10D3300043EA05330A4DA4B2A84289B29BB203D096
:10D3400005F50065A84205D1958924F4804444EA96
:10D350008514A4B2D28884808183A0F8402058E745
:10D36000002C014030B598B10A4B00221C461D79B3
:10D37000854207D19D79294202D004EB021030BDCD
:10D380000029FAD001320E2A03F11003EFD1002058
:10D3900030BD00BF1496010801490248F9F7EDBA03
:10D3A000B41800200008004001490248F9F7E5BA26
:10D3B0008C1800200004004002494FF08040F9F72B
:10D3C000DCBA00BF6418002001490248F9F7D5BA59
:10D3D0003C180020002C0140FFF7F6BF07298EBF44
:10D3E0000020024B53F8210080B27047BC1F002080
:10D3F0002DE9F041164D95F8203013B90020BDE815
:10D40000F081002385F8203095F82130A82BF5D144
:10D4100095F83440002CF1D10E4F0F4E05F1210844
:10D4200008EB0403D8781B7903EB002005F084FB9C
:10D43000394605F0D9FB314605F0CCFA05F0D6FDAA
:10D4400045F814000234102CEAD10120BDE8F08127
:10D45000BC1F00200000203E0080BB43024B03EBBA
:10D460004101C88EC0087047BC1F00201F4BF0B59B
:10D4700093F8562019460AB90020F0BD002093F811
:10D480005740B3F8586003EB440595F85D7095F884
:10D490005E2083F8560042EA07229642ECD193F8C8
:10D4A0005B30012B02D0812B14D0F0BD1846102C1C
:10D4B00088BF10234FF0000288BF81F857300C4B13
:10D4C00091F85740A3F12705D1B28C4203F1020332
:10D4D00002D8F0BD0320EAE713F8026C13F8011C30
:10D4E00041EA062125F812100132EDE7BC1F0020A9
:10D4F0001920002003788B420CD9074B890093F840
:10D500007F200B44D3F8800002B1400800F577700B
:10D5100080B2704700207047BC1F0020054B03EB12
:10D520008101D1F8B00000EB8000C00800F55C700C
:10D5300080B27047BC1F00205E4B10B593F8F80016
:10D54000002800F0B680002293F8FB4093F8FC001E
:10D5500083F8F82093F8FA2004F0070142EA012248
:10D5600000F03F01490141EAD401C3F8B02093F82B
:10D57000FD20C3F8B41093F8FE10920093F8FF401A
:10D5800042EA901201F0010042EA8022C3F8B8207A
:10D5900093F8000104F00F02D20142EA510200F0B8
:10D5A0007F01C3F8BC20090193F8012141EA14115D
:10D5B00093F802415200C3F8C01042EAD01204F0BE
:10D5C000030193F8030142EA4122C3F8C42093F80F
:10D5D000042100F01F018901D20041EA940142EACE
:10D5E000501293F8064193F80701C3F8CC2093F842
:10D5F0000521C3F8C81004F0070142EA012200F037
:10D600003F01490141EAD401C3F8D02093F8082131
:10D61000C3F8D41093F80911920093F80A4142EA32
:10D62000901201F0010042EA8022C3F8D82093F85A
:10D630000B0104F00F02D20142EA510200F07F0117
:10D64000090141EA1411C3F8E010C3F8DC2093F893
:10D650000C2193F80D41520004F0030142EAD0126C
:10D6600042EA4122C3F8E42093F80F2193F80E0117
:10D67000D20042EA501200F01F01C3F8EC2093F8E8
:10D680001021890141EA9401D407C3F8E8104CBF86
:10D6900040F21471AD21C3F8F01091074CBF40F275
:10D6A0001471AD2112F0080F14BF03200120C3F83C
:10D6B000F41010BDBC1F002008B5084B03EB81011E
:10D6C000D1F8140105F038FA054905F08DFA05493D
:10D6D00005F082F905F08AFC80B208BDBC1F00206D
:10D6E00001F11F3F00405C446E4B30B593F854216C
:10D6F0000AB9002030BD002293F8570183F8542165
:10D70000162840F0C980082210F0800F4FEA400030
:10D7100018BF80F0D500013AC0B2F5D193F8561188
:10D72000614D02398A42C0F2A78093F86E2182428D
:10D73000DFD1182293F8594193F85A0183F8562102
:10D7400093F8582104F0070142EA012200F03F015A
:10D750004901C3F8142141EAD40193F85B21C3F8CD
:10D76000181193F85C11920093F85D4142EA90120F
:10D7700001F0010042EA8022C3F81C2193F85E0107
:10D7800004F00F02D20142EA510200F07F01C3F817
:10D790002021090193F85F2141EA141193F86041B7
:10D7A0005200C3F8241142EAD01204F0030193F8A6
:10D7B000610142EA4122C3F8282193F8622100F076
:10D7C0001F018901D20041EA940142EA501293F804
:10D7D000644193F86501C3F8302193F86321C3F8DD
:10D7E0002C1104F0070142EA012200F03F01490137
:10D7F000C3F8342141EAD40193F86621C3F8381103
:10D8000093F86711920093F8684142EA901201F090
:10D81000010042EA8022C3F83C2193F8690104F038
:10D820000F02D20142EA510200F07F01090141EAF0
:10D830001411C3F84411C3F8402193F86A2193F8F6
:10D840006B41520004F0030142EAD01242EA412245
:10D8500093F86C01C3F8482193F86D2100F01F0183
:10D860008901D20042EA501241EA9401C3F84C11F6
:10D87000C3F85021012030BDAC18E4786040082482
:10D8800010F0800F4FEA400018BF80F0D500013C37
:10D89000C0B2F5D1013245E7A0F128035842584102
:10D8A00030BD00BFBC1F00201121002070B5304EDC
:10D8B000054633782F4C3BB1D4F8983183429EBF54
:10D8C0000023337084F89C312B4B1B6813F001024A
:10D8D0001CD094F89D2194F89E3193420CD00123E2
:10D8E000002184F89C31254B84F89E211970D4F8CE
:10D8F000A0312B44C4F8983194F8BC3173BBD4F8F0
:10D90000CC01854234BF0020012070BD13F40053C8
:10D9100008D013461A4A32F8131009BB01330C2BF6
:10D92000F9D1E9E784F8BC31D4F8C8319847C30786
:10D93000E2D5012300F00200002814BF1A4600229D
:10D9400084F8BC310D4B5A700CBF01230023337097
:10D95000D4F8A0312B44C4F89831CDE7012070BD34
:10D960000123002284F89C31044B1A70F0E700BFB9
:10D9700005130020BC1F00207C1700203C04002061
:10D980006021002000207047002070470023032BF7
:10D99000CCBF012200220CBF05211E2100F813205C
:10D9A00000EB43020133122B5170F0D1704710B5D8
:10D9B00000234FF47A744FF4FA61C452C21804334E
:10D9C000102B5180F9D110BD024B03EB4101B1F88E
:10D9D000A4017047BC1F0020024B03EB4101B1F8CA
:10D9E000A4017047BC1F0020024B03EB8101B1F87A
:10D9F000D0017047BC1F00202F4BF0B593F80822D0
:10DA00000AB90020F0BD002093F8092283F808022B
:10DA1000012A93F80C1232D1194491F80C2291F892
:10DA20000B12B3F80A4201EB022193F82D2289B2BE
:10DA300002F11C05EDB29E1896F80E7296F80D02D2
:10DA4000023200EB0720D2B22044AA4284B2F2D1C3
:10DA5000A142D6D1002193F82D52184805EB41027E
:10DA6000D2B21A4492F80E4292F80D2202EB04222E
:10DA700040F8212001310E29F0D10120F0BD4FF6F0
:10DA8000FF728C1E03F20D25A0420FD3194491F8AA
:10DA90000C12B1EB122FB4D11C4494F80D12D2B277
:10DAA0009142AED193F82E22202AD2E7465D013072
:10DAB000921B92B2E8E700BFBC1F00208C2100201F
:10DAC00010B50446F9F72EF841F288310D4BD3F822
:10DAD0003022C3F83002821A8A4284BF002283F8BF
:10DAE000342293F83422142A03EB02010CBF0122E2
:10DAF000013281F8214014BF83F8342283F82020BA
:10DB000010BD00BFBC1F002010B50446F9F70AF88D
:10DB1000254BD3F83822C3F83802821AB2F57A6F4F
:10DB200084BF002283F83C2293F83C224AB9A82CF7
:10DB300038D183F85620A3F85820991881F85A4014
:10DB400006E0022A02D183F85740F6E7242AF4D9E6
:10DB500093F8571001320231D2B249008A4283F859
:10DB60003C2216DA082241F22101B3F85800E4B24F
:10DB700080EA042010F4004F02F1FF324FEA400027
:10DB800018BF484012F0FF0280B2F3D1A3F858004A
:10DB900010BD01318A4201BF002283F83C220122DC
:10DBA00083F8562010BD00BFBC1F0020F8B5434CC1
:10DBB00094F84402002859D0002384F8443294F8A1
:10DBC000453294F8465205EB0325F8F7ABFF3C4B82
:10DBD000ADB2B0FBF3F0D4F85832002B47D1A4F823
:10DBE0005C52C4F858020322D4F8603294F85F52B1
:10DBF0001E7894F85E0294F86472511E631893F8CC
:10DC000045322B4103F00F03B34212D20B2B10D835
:10DC100008B183420DD0214491F845E2A11891F852
:10DC200045120EEA070E04EB830301EB0E21C3F845
:10DC300080100232112AE0D194F86532ABB194F829
:10DC4000663293B194F847321B060ED5F8F76AFF97
:10DC5000D4F840321B4964301BB15A68121A002AAA
:10DC600028DB194AD36004320A600120F8BD9842CB
:10DC7000B9D0C31A012BB2D194F85E22002AAED0DB
:10DC8000B4F85C3294F87F1092002244EB1A49B148
:10DC90006FF01301DB0293FBF1F303F50063C2F8AD
:10DCA00080309CE76FF013019B0293FBF1F303F5C7
:10DCB0008063F4E703F108019B68CDE7BC1F0020F7
:10DCC00020A10700FC2100203C04002010B50446E0
:10DCD000F8F728FF41F288310E4BD3F86822C3F8D9
:10DCE0006802821A8A4284BF002283F86C2293F869
:10DCF0006C220F2A0DD8511CC9B21A441029E4B263
:10DD000082F8454214BF0022012283F86C1283F886
:10DD1000442210BDBC1F002010B50446F8F702FFD6
:10DD200040F6AC51104BD3F87022821A8A42C4BF1D
:10DD3000002283F8742293F874228AB90F2C11D12F
:10DD4000C3F87002511CC9B21A44192982F8F9406B
:10DD500014BF0022012283F8741283F8F82001E036
:10DD6000182AEFD910BD00BFBC1F002010B5044613
:10DD7000F8F7D8FE154BD3F8782202F57A72904264
:10DD800084BF002283F87C2293F87C221AB9C3F85E
:10DD90007802052104E0022AFBD993F856110231DA
:10DDA000914211DD501CC0B21A44814282F85541A3
:10DDB000D4BF0122002283F85421D8BF002283F867
:10DDC0007C02D8BF83F87C2210BD00BFBC1F00209E
:10DDD00010B50446F8F7A6FE284AD2F88032C31AD6
:10DDE000B3F5FA7F134628D9002283F8842283F8FA
:10DDF000852293F88422C3F8800292B9E1B2042903
:10DE000001D0202921D183F82E1283F80C1202218F
:10DE1000002083F82D124FF6FF7183F80902A3F852
:10DE20000A12991881F80D4293F80C1201398A42AE
:10DE300020D1012283F8082210BD92F88512002912
:10DE4000D7D0013982F8851210BD93F82E1271B91E
:10DE5000552C0CD101211F2083F8091283F82E4282
:10DE600083F80C02A3F80A2283F82D12D9E78C421A
:10DE7000D7D010BD013283F88422FAE7BC1F0020FE
:10DE800010B5074C94F8662242B104F28621D4F80A
:10DE90009C02F8F716FF002384F8663210BD00BF1D
:10DEA000BC1F0020F0B50025234B41F221071A7852
:10DEB0002B462249961EECB2B44218DB0244941E53
:10DEC000013A0C5D8A5C02EB042292B293420DD1BE
:10DED00000244FF4AF671A4B1A4E93F8A05201304A
:10DEE000E3B29D4216D80122174B1A70F0BD0444CC
:10DEF0000C5D83EA0423082413F4004F04F1FF347B
:10DF00004FEA430318BF7B4014F0FF049BB2F3D1E8
:10DF10000135D0E700EB4303DAB211F802E0013239
:10DF20008B5C03EB0E239BB27B431B1303F54873FF
:10DF300026F814300134D3E77A1A00207B1A002027
:10DF4000BC1F0020581A0020701A00202DE9F04153
:10DF500005460F460446094E06F10808217809B91E
:10DF6000BDE8F081054809F0AAFE20B140453EBF5A
:10DF7000801B631B3B540134F0E700BF1894010879
:10DF800010B500212C22044609F073FE01236372B0
:10DF900023752923A37540F2DC53238340F21A43EF
:10DFA000638340F26C73A3830223A377132384F863
:10DFB000203040F24653638440F27533A38440F628
:10DFC0004303E3840623214684F828300148BDE852
:10DFD0001040BBE783B20108124B03EB400393F8F8
:10DFE000A1222AB1022A12D00F4B33F81000704739
:10DFF000022809D90328F7D10C4B1B6813F4805F62
:10E000000B4B02D1988C7047094B188B704793F8D3
:10E01000A20200EB800000EB800000F2EE2080B254
:10E02000704700BFBC1F00203C1300207C1700205D
:10E030008017002008B5F8F775FD0222064B83F81B
:10E04000CC22C3F8C802054B1A68054B9A6001221E
:10E0500083F8212008BD00BFBC1F0020C41300208E
:10E060008013002008B5F8F75DFD0222074B00F58C
:10E07000B71083F8CC22064A00F55870C3F8C802DE
:10E08000936803F2DC53936008BD00BFBC1F0020FF
:10E090008013002038B5134A134C054694F8CD324E
:10E0A00010685843114B186004F046FD104904F005
:10E0B0009BFDC4F8D002284601F0A8FA284601F0DA
:10E0C000D5F9288D04F03CFD0A4904F08DFDC4F813
:10E0D000D402688D04F034FD064904F085FDC4F8CF
:10E0E000D80238BD80250020BC1F00205817002012
:10E0F000BD3786356F12833A084BDA68D10709D4E9
:10E10000DA68520708D4DB6813F0100F14BF03203D
:10E110000420704701207047022070470020024011
:10E120000EB40FB5074A06AB0190074901A8039347
:10E1300002F09EFC0022019B1A7004B05DF804EB13
:10E1400003B070478CB201088B080108A0F17D0371
:10E15000012B70B504460D460A4E11D87D2130685A
:10E16000F8F7ACFD84F020013068F8F7A7FD35B171
:10E170002888204400EB102000F0FF00288070BDAC
:10E180000146F1E7E0220020024B01465868F8F70B
:10E1900095BD00BFE0220020012300F01F024009CE
:10E1A000022803FA02F308D003280BD001280DD16E
:10E1B000074A51690B4353617047054A91690B4304
:10E1C00093617047024AD1690B43D361704700BF26
:10E1D000001002400C4B0D49DB68DB43C3F3022304
:10E1E000C3F104024378934002781B018818DBB224
:10E1F00080F800330123500902F01F0203FA02F2F3
:10E2000041F82020704700BF00ED00E000E100E091
:10E210000C2921D8DFE801F0072020201020202041
:10E22000182020202100038B23F008031B041B0C63
:10E2300043F0080303837047038B23F400631B043C
:10E240001B0C43F40063F5E7838B23F008031B04E6
:10E250001B0C43F0080383837047838B23F4006314
:10E260001B041B0C43F40063F5E7214A038890422A
:10E270009BB212D002F5006290420ED0B0F1804FF6
:10E280000BD0A2F59832904207D002F580629042FE
:10E2900003D002F58062904202D123F070039BB25A
:10E2A000144A904206D002F5806290421CBF23F4CB
:10E2B00040739BB203808B8883850B8803850C4B4E
:10E2C00098420FD003F5006398420BD003F54063EA
:10E2D000984207D003F58063984203D003F580632A
:10E2E000984201D10B7A038601238382704700BFD5
:10E2F000002C0140001000402DE9F347774C784E88
:10E30000657BC4F8D4607DB9D4F8A022754B658ACA
:10E31000B3FBF2F3AB42A18AC4F85061C0F087802E
:10E32000002D40F0968084E0D4F8A0826D4BB3FBC2
:10E33000F8F3AB42E8D3237B04F1D80713B3012BE6
:10E3400057D1694BC4F84471C4F8D430284604F05E
:10E35000F3FB054642460146384602F0AFFD04F1A4
:10E36000FC00D4F8A0222946C4F8480102F0A6FD1A
:10E3700004F59070D4F8A0222946C4F84C0102F0AC
:10E380009DFDC1E7594B4046C4F8D43004F0D4FB9E
:10E39000574904F029FC8046284604F0D1FB014689
:10E3A000544804F0D5FC05460146404604F014FBF1
:10E3B0000146404604F0CCFC04F1E803C4F84831BF
:10E3C00004F1F803C4F84471C4F8E050C4F8E480E0
:10E3D000C4F8DC00C4F8F050C4F8F480C4F8EC00D1
:10E3E000C4F84C31C4F80051C4F80481C4F8FC00EE
:10E3F0008AE7414B1FFA88F229463846C4F8D430E0
:10E40000C4F8447102F0B0FC04F1EC00B4F8A022AE
:10E410002946C4F8480102F0A7FC04F58070B4F85E
:10E42000A0222946C4F84C0102F09EFC6CE78B4206
:10E430000ED8D4F8A0222B4BE58AB3FBF2F3AB4203
:10E44000218BC4F8C06125D33DBB02B0BDE8F08785
:10E450009DB20029EDD0244B2846C4F8503102F07B
:10E4600039FD002781464FF0010ADFF890802846E9
:10E4700004F062FB07F59C7E0146CDF800A04B46F8
:10E48000D4F8A02208EB0E00243702F076FC6C2FA3
:10E49000EDD1CEE78B42D8D99DB20029D5D0124B11
:10E4A0002846C4F8C03102F015FD002681464FF021
:10E4B000010ADFF84880284604F03EFB06F5D477D1
:10E4C0000146CDF800A04B46D4F8A02208EB070087
:10E4D000243602F052FC6C2EEDD1B6E7E02200208B
:10E4E000C309010820A107004D090108A509010879
:10E4F000BD37863583F9223EE9080108FC22002059
:10E5000073B504461A4A00210068F8F780FA2168BA
:10E51000184A0B889BB243F001030B80002352F88A
:10E520003340D800A1421ED102445579012400266F
:10E5300001A88DF804508DF805408DF806608DF81F
:10E540000740FFF747FE1B2D0BD1192301A88DF8BB
:10E5500004308DF805408DF806608DF80740FFF710
:10E5600039FE02B070BD0133042BD8D10025DDE7A0
:10E5700040420F003094010870B50024164B93F808
:10E58000C02293F9B65203EBC20193F9BE6201F5C2
:10E590003171012A04D90CB183F8C022002070BD6A
:10E5A00031F8024C013214F0010FD2B20BD02042EC
:10E5B00009D091F90040AC4203D183F8C022074B47
:10E5C00007E0B44202D008310124E2E783F8C02218
:10E5D000034B186870BD00BFE0220020902500208A
:10E5E000982500200022024B83F8C022C4E700BF18
:10E5F000E022002010B50446006802F0C7F8606809
:10E6000002F0C4F8A068BDE8104002F0BFB8F0B551
:10E610000C46054689B014220021204609F029FB4A
:10E6200004A92A6800230D461D4EC2F3855040FA06
:10E6300003F7FF0748BF9F5D03F1010344BF0F705D
:10E640000131062BF3D1002316480B70C2F30321CE
:10E65000014491F82610C2F305368DF818102D30BC
:10E660000DF1190146FA03F7FF0748BF1F5C03F1DC
:10E67000010344BF0F700131062BF3D100230B704F
:10E68000C2F38343029306AB0193009502F00F039C
:10E690000549C2F303122046FFF742FD09B0F0BD61
:10E6A00050940108309401088CB201088B6810B5B1
:10E6B0000C6A026823430C6922F4FF4223434C692D
:10E6C00022F0700223438C692343CC6923434C6AB4
:10E6D00023438C6A234313430360CB6843600B6876
:10E6E00083604B68C36010BD036823F001031B0403
:10E6F0001B0C03600023036043608360C360294BED
:10E70000984204D1284A536843F00F0326E0274B70
:10E71000984204D1244A536843F0F0031EE0244B8E
:10E72000984204D1204A536843F4706316E0214BA9
:10E73000984204D11C4A536843F470430EE01E4BC8
:10E74000984204D1184A536843F4702306E01B4BE7
:10E75000984205D1144A536843F4700353607047DC
:10E76000174B984204D1104A536843F07063F5E7A1
:10E77000144B984201D1144AC5E7144B984201D179
:10E78000114AC8E7124B984201D10F4ACBE7114B0F
:10E79000984201D10C4ACEE70F4B9842DFD10A4A8A
:10E7A000D1E700BF08000240000002401C00024008
:10E7B0003000024044000240580002406C00024019
:10E7C0008000024008040240000402401C04024091
:10E7D000300402404404024058040240224A10B56A
:10E7E000536803F00C03042B28D0082B29D01F4BAF
:10E7F000036053681E49C3F303130B4493F833407B
:10E800000368E34043605468C4F302240C4494F862
:10E81000334023FA04F484605468C4F3C2240C44E3
:10E8200094F83340E340C3605268C2F3813211442C
:10E8300091F84320B3FBF2F3036110BD0D4B1B684D
:10E84000D6E753685168C3F38343C90303F1020356
:10E8500002D409494B43CBE7516811F4003F054905
:10E86000096818BF4908F5E70010024000127A0055
:10E87000309401084C04002000093D0010B5044606
:10E88000FFF73AFC012806D10CB9052010BDFFF7AF
:10E8900033FC013CF6E7002C08BF052010BD2DE934
:10E8A000F041CB780E88DA0648BF8A7803F00F056E
:10E8B00048BF154316F0FF0F1AD000214FF0010E8C
:10E8C0004FF00F0C02680EFA01F737EA06040BD17D
:10E8D0008C000CFA04F822EA080205FA04F4282B4A
:10E8E00042EA040225D1476101310829EBD10260D7
:10E8F000FF2E1CD900214FF0010E4FF00F0C426883
:10E9000001F108040EFA04F434EA06070BD18F0073
:10E910000CFA07F822EA080205FA07F7282B42EA60
:10E9200007020AD1446101310829E9D14260BDE8FA
:10E93000F081482B08BF0761D6E7482B08BF046168
:10E94000F1E70F4B1A6842F001021A6059680D4A4C
:10E950000A405A601A6822F0847222F480321A60E7
:10E960001A6822F480221A605A6822F4FE025A6061
:10E970004FF41F029A604FF00062034B9A60704799
:10E98000001002400000FFF800ED00E080F308886E
:10E990007047034B93F8D612D3F8D802F8F78EB924
:10E9A000E022002038B50446054D0146D5F8D802CE
:10E9B000F8F784F995F8D6325C4085F8D64238BD30
:10E9C000E022002008B50020FFF7ECFF0020FFF751
:10E9D000E9FF0020FFF7E6FFBDE808400020E1E77F
:10E9E00010B50446C0B2FFF7DDFF200ABDE81040B5
:10E9F000D8E738B500230546094C2421D4F8D802BD
:10EA000084F8D632F8F75AF9D4F8D8025421F8F736
:10EA100055F92946D4F8D802BDE83840F8F74EB980
:10EA2000E02200207FB500240B0A04AD8DF8080019
:10EA30008DF80A10000A8DF80B3025F80A4D0B0CE2
:10EA4000090E8DF809008DF80D10102029468DF85B
:10EA50000C30FFF77BFB02AE305D29460134FFF737
:10EA600075FB062CF8D19DF806000021C043C0B20A
:10EA7000FFF76CFB04B070BD73B50F4C0646D4F8BD
:10EA8000DC020D4600F04BF994F8E53294F8E622EA
:10EA9000003318BF01230AB143F00803019396F92C
:10EAA000000000954FF496430022082100F05CF925
:10EAB000C4F8DC0202B070BDE022002010B5064CA4
:10EAC000D4F8DC02F8F7F7F800B910BDD4F8DC028E
:10EAD000F8F7EEF8F4E700BFE022002008B50B4B92
:10EAE000D3F8F02292781E3A012A08D9D3F8DC0232
:10EAF00001210430FFF7C0FFBDE80840DEE7012137
:10EB0000D3F8DC02F8F7CEF8F6E700BFE0220020E9
:10EB10000028114AB8BF404290FBF2F330B50F4CC9
:10EB200004FB03053C2068430D4D90FBF2F295F881
:10EB3000E75275B903EB830303EB830302EB830313
:10EB40000B804FF47A7304FB020292FBF3F24A80CB
:10EB500030BDC3EB0313F1E780969800806967FF2F
:10EB6000E022002010B50446C0B2F8F7F5FEC4F369
:10EB70000720BDE81040F8F7EFBE00BF064A116855
:10EB800049B1642350684343B3FBF1F303490B805D
:10EB90000023136053607047082600208A1C002061
:10EBA000704710B514220021044609F062F80523CD
:10EBB000002201210420E3706371E37263730C4B44
:10EBC000A270A271A27393F9022020718A42A172ED
:10EBD0002073218009D093F90A208A4204D052235D
:10EBE000A3746423238210BD083340221A80F6E701
:10EBF000A2250020194B2DE9F0411C6807460F2C77
:10EC0000984607DC0023164A9C4206DC0025144E79
:10EC1000A54208DD0020BDE8F08152F823108F42A4
:10EC2000F8D00133F0E756F82530681C7BB9800036
:10EC3000621B011F920031443044013408F0FFFF91
:10EC400046F82570C8F800400120BDE8F0811A7D23
:10EC50003B7D9A42EBD30546DAE700BF301C00202B
:10EC6000341C00201128F8B50FD00F280CD83422FE
:10EC7000124B02FB003009B1C3684BB90022104DA2
:10EC800010492C68A24206DBF8BD0F4B1868F2E76A
:10EC9000BDE8F840AEE751F822709300B84203EBAC
:10ECA000010609D1A21A0433920019443046013CEE
:10ECB00008F0C5FF2C60F8BD0132E3E73400002006
:10ECC000301C0020341C0020901F002008B50C4B85
:10ECD000197801290CD00AD302290DD0F7F722FFA9
:10ECE000084B00F5F42000F59070186008BD002175
:10ECF0000020F8F78DF8F1E70020F8F701F8EDE7CC
:10ED0000421900204419002010B504462046F7F7A8
:10ED1000CCFF00B110BD0A20F7F753FFF6E7064B12
:10ED20001A68904203D09A68904204D108330022B6
:10ED3000C2629A801A6070479025002070B505461F
:10ED40000024084EA359AB4207D12846FFF7E7FF3E
:10ED5000CC220021301908F08CFFCC34B4F5197F97
:10ED6000F0D170BD102600202DE9F04F264D9B46B6
:10ED700095F9063093B08342039104929DF8708018
:10ED80009DF8747043D095F90E3083423ED0002038
:10ED900013B0BDE8F08F0130072867D100206CE088
:10EDA0000132072A40F0858000228AE0019B53B19E
:10EDB000711CC9B220B14FF00B0EC17180F806E092
:10EDC0001A21F7F7CFFF029B002B00F0C980711CBE
:10EDD000C9B2B9F1000F04D00C2089F8071089F8E6
:10EDE00006004A214846B9E04FF6DF72E36C1A800C
:10EDF000DA6842F02002DA600BE1E26CD36843F09B
:10EE00008003D36031E100BF902500200835B5F8BC
:10EE10000490B9F1000FBAD10128B8D8994BC6B205
:10EE200003EB8000D0F86C42002C00F02981964B57
:10EE3000D4F854A0236004F15A03636104F5AD7360
:10EE4000A3614FF48073DAF80420C4F808B0E264D8
:10EE5000E36023619AF81600FFF79EF9DAF80C20B8
:10EE6000F2B18A4B48464FF01C0C19460CFB003996
:10EE7000D9F804904A458ED1C0B24FF01C0909FB65
:10EE80000010834B0169D3F814E04EEA0101596187
:10EE90000C210176711C41762263E26C0432A2647B
:10EEA000DAF8081000293BD0784800224FF01C0CFB
:10EEB00086460CFB0209D9F8043099427FF470AF02
:10EEC000D2B21C2101FB02EE714ADEF8101050692B
:10EED000084350610B208EF81800701C8EF8190042
:10EEE00053699AF81900194351616A4ACEF81440DF
:10EEF000CEF808209EF80D208DF81C2082098DF890
:10EF00001D2000228DF81E20012207A88DF81F2049
:10EF1000FFF760F9DAF808206263E26C0432626499
:10EF200094F85800F7F7FCFE814694F85900F7F77B
:10EF3000F7FE08F00203019317F0080F08F0010331
:10EF400002933FF433AF721CD2B210B10B21C271E5
:10EF5000817117F0100F14BF1A211E21F7F702FF5D
:10EF6000DAF80C2012B1DAF808208AB99AF81820D9
:10EF700007A88DF81C209AF81A309B098DF81D30CF
:10EF800000238DF81E3001238DF81F30FFF722F982
:10EF9000012384F8503000232362E361A36263629B
:10EFA0000593049B84F80580E362C4F808B0A77158
:10EFB0002046F6F7C7FB029A059B002A29D0206B52
:10EFC00000283FF411AF09930B930D930E93119307
:10EFD000A36C07934FF48053109380230C93E36842
:10EFE0000A9320230F9363690893FFF77DFB07A91A
:10EFF000206BFFF75BFB226BE16C136843F00103AE
:10F0000013608B8A9BB243F040038B8253689BB2A0
:10F010002364019B002B28D0606B00283FF4EDAEE9
:10F02000636C002707934FF48053109380230C9355
:10F03000236908970A9310230B9709930D970E974E
:10F040000F971197FFF750FB07A9606BFFF72EFB97
:10F05000636B1A6842F002021A60E26C5F605F60E4
:10F06000938A9BB243F080039382E26C93899BB2B4
:10F0700043F400539381BDF80C302671AB802C60B3
:10F08000204685E6082600207894010878030020B1
:10F090000010024005B1000838B1038813EA0100EE
:10F0A00003D08B420CBF0120022070470023F0B533
:10F0B0001D460E490E4E81F87832DAB2012A04D983
:10F0C0000DB181F878220020F0BD5F1C06EBC3046F
:10F0D00036F8333001321842D2B24FF0010503D076
:10F0E00081F878222046F0BD3B46E6E7082600205E
:10F0F000A22500202DE9F74F0120FFF7D7FF0024BC
:10F10000234D244E78B3022C2DD84FF0CC0A0AFBA5
:10F1100004F905EB0908D8F8087017B10134E4B216
:10F12000F0E70322C378012190F9020056F823305A
:10F13000009201973A46FFF717FE834648B11648FA
:10F14000524639464844013408F093FDE4B2C8F809
:10F1500008B0002195F87822104FD3B2012B05D9C1
:10F1600009B185F8783203B0BDE8F08F02F1010EE5
:10F1700007EBC20037F832200133D207DBB24FF081
:10F18000010102D585F87832BCE77246E5E700BF99
:10F19000082600203082010810260020A225002029
:10F1A000142809D80C235843044B185C28B10123B8
:10F1B000013803FA00F07047002070479C92010864
:10F1C00010B500240020F7F7FEFD074B1C70FFF779
:10F1D0007DFD064B1C70064BC3F87C42A3F88042B1
:10F1E000C3F8844210BD00BF421900201F13002045
:10F1F00008260020F0B440B1154B1B6813F400330F
:10F2000006D0144B1B78032B01D1F0BCD8E70023A8
:10F21000114C0C26224606FB03F10F5D0D198742A7
:10F2200004D00133152BF6D1F0BC70470B4BD3F84B
:10F23000840218B16C7840788442F5D20A44C3F84D
:10F2400084220022A3F88022C3F87C22ECE700BFCE
:10F25000D01D0020691300209C9201080826002080
:10F26000F8B506460D2002F0D7F810B10A20FFF7D6
:10F27000C1FF2F4CD4F88422002A57D0D4F87C3216
:10F28000B34253D82B4BB4F880121878576860BB40
:10F29000012018707B5C002B38D01378264A013B84
:10F2A000126800FA03F3134201D1F7F78CFD012233
:10F2B000224B1A70FFF70AFDB4F880324BB9D4F82C
:10F2C00084321B78053B012B03D8F7F72BFC1C4B32
:10F2D0001860D4F88432B4F880225B689B5CFE2B03
:10F2E0000FD10023A4F88032F8BD00251D707B5C8F
:10F2F00063B12846F7F767FD104B1D70FFF7E6FC7A
:10F30000E7E7FF2B08D1BDE8F84059E7D4F884328D
:10F31000B4F880225B689B5C42F2107101FB0363CE
:10F320000132C4F87C32A4F88022F8BDF8BD00BFD9
:10F33000082600201F130020D01D002042190020A5
:10F34000401700204000402830B4A8BF40200023D0
:10F3500002251424064A9D5402339918984201F854
:10F36000014CF8D8FF21D1540E2030BC42E700BF39
:10F370004C1F002010B5064C228822EA0000824271
:10F38000208002D00120FFF7DDFF208810BD00BFE4
:10F390006613002010B5054C22881043824220805D
:10F3A00002D00120FFF7CEFF208810BD6613002099
:10F3B000024A138823EA000010807047A41300203B
:10F3C000024A138818431080704700BFA41300201E
:10F3D00038B50346064D00F1EA0418464E22294688
:10F3E00006F016F803464E33A342F6D138BD00BFEF
:10F3F000A49401084FF47A524FF47A7302800422E5
:10F4000083818270038201224FF4E1730271438190
:10F410004FF4FA620023C2811A4630B5074C19191D
:10F420008D796D0741BF0D7981184D710132D02B57
:10F4300003D0032A03F11003F1DD30BD1496010857
:10F4400038B50024054D55F83400013401F022FE92
:10F4500001F0A5FE1E2CF6D138BD00BFF4940108C2
:10F460000121FDF75FB80021FDF75CB82DE9F74FEA
:10F470000546074600265B4CDFF884B1DFF884A11F
:10F48000DFF8848104F10C0904F118033878019342
:10F4900003F056FB594603F0A7FB44F826007878A2
:10F4A00003F04EFB514603F09FFB49F82600B87865
:10F4B00003F046FB414603F097FB019B033743F8FB
:10F4C00026000136032EE1D195F8370003F038FB12
:10F4D000454903F089FB606295F8360003F030FB84
:10F4E0000146424803F034FCA062687D03F028FB2B
:10F4F0003F4903F079FBE062A87D03F021FB3C4922
:10F5000003F072FB2063E87D03F016FB95F83030C2
:10F5100095F82F6084F838306063C6F1AF0003F0CF
:10F520000FFB344903F060FBE063C6F1640003F0B5
:10F5300007FB314903F058FB6427304B2064688F88
:10F540001E68784303F0FCFA314603F04DFBA064DB
:10F550006064288F784303F0F3FA314603F044FBEC
:10F56000E06495F8270003F0E7FA234903F03CFB39
:10F5700001464FF07E5003F02DFA01464FF07E50C9
:10F5800003F0E6FB4FF47A732065B5F8422095F856
:10F5900047005A436265B5F844205343A3650A23E4
:10F5A00095F846205343E36503F0C6FA2066E88FDA
:10F5B00003F0C2FA6066A88F03F0BEFAA066B5F841
:10F5C000400003F0B9FAE066B5F84A0003F0B4FA77
:10F5D0002067B5F84C0003F0AFFA606703B0BDE8F0
:10F5E000F08F00BF902800200402013C0000C842B8
:10F5F000CDCCCC3D6666E63F0AD7233C8C2200206A
:10F60000D730033D033F7A3E97AC0A3A2DE9F04FDD
:10F61000674E85B0336805460393664C3BB9664B2D
:10F62000A367E367C4F8803005B0BDE8F08F634F8F
:10F630004FF07C50396803F08BFB03F0D7FCB5F832
:10F64000229080464845BB4633D2AB8C984233D992
:10F650001FFA80F9A98C00292ED0594B4846A36780
:10F6600001F038FC574F8246C4F88470484603F0D6
:10F6700063FA0123014681460093039A53463846B4
:10F6800001F07BFB0123009307F12400534632680D
:10F690004946C4F8880001F070FB288C08B1804509
:10F6A0000DD2454BE367E88B08B1804561D2424BF0
:10F6B000B8E7B9F1000FCDD13F4BA367EDE795F85F
:10F6C0002630012B3DD015D3022BEAD13E4F3F4BC4
:10F6D0003288C1B23846E367C4F8D47001F044FB05
:10F6E00007F11400328895F82010C4F8D80001F012
:10F6F0003BFBD8E7364BC0B2E36703F021FA014683
:10F70000344803F025FBDBF800600746014630462D
:10F7100003F062F90146304603F01AFB2A4BC4F8A5
:10F72000E470C4F8D4301033C4F8E860C4F8E000E2
:10F73000C4F8D830C4F8F470C4F8F860C4F8F00025
:10F74000B1E71F4B204FE367C4F8D47003F0F4F91E
:10F75000326801463846243701F0B0FBC4F8D8704F
:10F76000288C03F0E9F932680146384601F0A6FB1F
:10F7700099E7174BC0B2C4F88030174BDBF8005044
:10F78000C4F8243103F0DCF90146124803F0E0FA32
:10F79000C4F834510146C4F83001284603F01CF97E
:10F7A0000146284603F0D4FAC4F82C013CE700BF18
:10F7B0005817002090280020C30901088C2200203F
:10F7C0004D0901081C2900206C290020E9080108C6
:10F7D000A509010883F9223EB82900202DE9F0414E
:10F7E0000024094E094D0A4F3078844204DBD5F8D5
:10F7F0003C31BDE8F041184757F82410E0B2D5F885
:10F80000383198470134EFE7A015002090280020F8
:10F81000A41500202DE9F74F4C4B4D4CD3F8009028
:10F82000D4F840514946284603F0DEF9D4F8447133
:10F8300080464946384603F0D7F9D4F8486100902D
:10F840004946304603F0D0F939468246284603F04F
:10F85000CBF931468346284603F0C6F93146814646
:10F86000384603F0C1F939460190384603F0BCF937
:10F87000014603F0B1F831460746304603F0B4F9CB
:10F88000014603F0A9F806460146384603F0A4F8FD
:10F8900001464FF07E5003F09DF85146C4F84C01EC
:10F8A000584603F097F8014603F096F84946C4F825
:10F8B0005001009803F090F8014603F08DF8594686
:10F8C000C4F85401504603F087F8014603F084F869
:10F8D0002946C4F85801284603F086F9014603F08A
:10F8E0007BF800F100453146284603F073F84FF0ED
:10F8F0007E5103F071F84146C4F85C01019803F0B1
:10F9000069F8014603F068F80099C4F860014846B8
:10F9100003F060F8014603F05FF80199C4F8640150
:10F92000404603F059F8014603F056F83946C4F84A
:10F930006801284603F04EF84FF07E5103F04CF872
:10F94000C4F86C0103B0BDE8F08F00BF5004002084
:10F95000902800202DE9F04FAD4B89B01B68AD4ACF
:10F9600013F0020F00F0038492F84410002900F015
:10F97000FE83A949D2F83890D1F87041C1F87001DE
:10F9800009FB09F1D2F83CB0D2F840A00BFB0B11F7
:10F99000041B0AFB0A106421928A4143524391FBE3
:10F9A000F2F213F00803A2F152020494069208D076
:10F9B0009A4A13682BB153681BB19368003318BF80
:10F9C000012304981C4603F0B7F8954903F00CF99D
:10F9D000944D00909449686803F006F992490190AB
:10F9E000A86803F001F990490290E86803F0FCF878
:10F9F00000250390002C00F0A783884C206803F0BA
:10FA00009FF80746606803F09BF80646A06803F07D
:10FA100097F831460446304603F0E6F82146804622
:10FA2000204603F0E1F80146404602F0D5FF394692
:10FA30008046384603F0D8F80146404602F0CCFF35
:10FA40007A49804603F08CFA002800F07D83404616
:10FA500006F004F901464FF07E5003F079F9804634
:10FA60000146384603F0C0F841460590304603F0A1
:10FA7000BBF841460746204603F0B6F8664C0646FA
:10FA8000D4F84C11059803F0AFF8D4F85011079052
:10FA9000384603F0A9F8079B0146184602F09CFF80
:10FAA000D4F854110790304603F09EF8079B0146A6
:10FAB000184602F091FFD4F858110790059803F00A
:10FAC00093F8D4F85C118046384603F08DF801466F
:10FAD000404602F081FFD4F860110746304603F03B
:10FAE00083F80146384602F077FF079B0646194621
:10FAF000184603F079F831460746304603F074F8AB
:10FB00000146384602F068FF06F0A8F80146304684
:10FB100003F06AF800F10046D4F86411304603F0AF
:10FB200063F8D4F868118046304603F05DF8D4F8E5
:10FB30006C110746304603F057F80646069B262B05
:10FB400000F29180484602F0FBFF8146584602F0E1
:10FB5000F7FF0446504602F0F3FF21468246204656
:10FB600003F042F851468346504603F03DF8014603
:10FB7000584602F031FF49468346484603F034F8C0
:10FB80000146584602F028FF2849834603F0E8F969
:10FB9000002868D0584606F061F801464FF07E50C4
:10FBA00003F0D6F883460146484603F01DF859464F
:10FBB0008146204603F018F859460446504603F0A3
:10FBC00013F8154B8346D3F86C2120461146D3F821
:10FBD00068A10692059303F007F8414602F0FCFE87
:10FBE00051468046584602F0FFFF0146404602F06B
:10FBF000F1FE059B8046D3F86431584619460593BB
:10FC000002F0F2FF394602F0E7FE069A07460FE0DF
:10FC10007017002040150020902800208815002033
:10FC2000BD3786358025002035FA8E3C0AD7233C27
:10FC30001146484602F0D8FF0146384602F0CAFE97
:10FC400051460746484602F0CFFF314602F0C4FE57
:10FC5000059B06461946204602F0C6FF014630467F
:10FC600002F0B8FE0646AE4C0021D4F87491484626
:10FC700003F076F9002800F06B820299084602F042
:10FC8000B3FF03990546084602F0AEFF0146284639
:10FC900002F0A2FE01990546084602F0A5FF0146C2
:10FCA000284602F099FE9F4903F03CF908B3494603
:10FCB000009802F099FF4146054602F095FFD4F8FE
:10FCC000801102F089FE3946C4F88001284602F00E
:10FCD0008BFFD4F8841102F07FFE3146C4F8840112
:10FCE000284602F081FFD4F8881102F075FEC4F8AE
:10FCF00088018D4BD4F878011B78DA0700F12F8248
:10FD00008A4B1A6844F61F639A4200F22882884997
:10FD100002F06AFFD4F880110546019802F05CFEFB
:10FD200029468146404602F05FFF0146484602F000
:10FD300053FED4F884118046029802F04DFE294605
:10FD40008146384602F050FF0146484602F044FE24
:10FD5000D4F888110746039802F03EFE29468146F2
:10FD6000304602F041FF0146484602F035FE4FF0B2
:10FD70007C518146009802F037FF4146064602F06A
:10FD800033FF39460546304602F02EFF494680468D
:10FD9000304602F029FFD4F84091664B824629464E
:10FDA00009F10040D3F800B0059302F01DFFD4F82C
:10FDB000446101903146404602F016FF019A014627
:10FDC000104602F007FED4F84871019039465046BB
:10FDD00002F00AFF019A0146104602F0FBFD594667
:10FDE00002F0FAFD59460190284602F0FDFE314628
:10FDF0000290504602F0F8FE029A0146104602F0C8
:10FE0000EBFD494602F0E8FD39460290404602F01B
:10FE1000EBFE029A0146104602F0DCFD59460390C3
:10FE2000404602F0E1FE39460290284602F0DCFE30
:10FE30000146029802F0D0FD314602F0CDFD494660
:10FE40000290504602F0D0FE0146029802F0C2FD38
:10FE500059460290504602F0C7FE49468246404647
:10FE600002F0C2FE0146504602F0B6FD394602F0ED
:10FE7000B3FD31460746284602F0B6FE0146384635
:10FE800002F0A8FD01990646084602F0ADFE039A6D
:10FE900005461146104602F0A7FE0146284602F02C
:10FEA0009BFD02990546084602F09EFE0146284643
:10FEB00002F092FD31460546304602F095FE0146BD
:10FEC000284602F089FD05F0C9FE01464FF07E503C
:10FED00002F03EFF05460146019802F085FE039AB6
:10FEE000059B29461860104602F07EFE2946C4F89C
:10FEF0004001029802F078FE2946C4F844013046D9
:10FF000002F072FEC4F84801FFF784FCD4F86831AF
:10FF1000D4F86C9118464946019305F0A7FC0BE014
:10FF200090280020E68AF93D04130020C413002025
:10FF300000002041500400208F4902F055FE05F0DA
:10FF4000CDFBD4F864A1A4F88C010AF1004005F0BF
:10FF50003DFC0146894802F03DFD874902F044FE20
:10FF600005F0BCFBD4F85831D4F84CB1A4F88E019C
:10FF700059461846029305F079FC7F4900F100408C
:10FF800002F032FE05F0AAFB03B2002BA8BFA4F8D2
:10FF900090317B4BBCBF00F56160A4F89001D3F8B1
:10FFA0009411484602F0DCFF764B1A78002800F0E6
:10FFB000D98042F00802744D1A70A86B02F0C0FD9F
:10FFC0000746E86B02F0BCFD8046286C02F0B8FDE5
:10FFD0006B4C0646D4F85011404602F005FE5946D7
:10FFE0000390384602F000FE039B0146184602F0DB
:10FFF000F3FCD4F854118346304602F0F5FD014677
:020000040801F1
:10000000584602F0E9FC51468346384602F0ECFDC2
:1000100001998246404602F0E7FD0146504602F053
:10002000DBFC49468246304602F0DEFD0146504682
:1000300002F0D2FCD4F85C118146404602F0D4FDB7
:1000400002998046384602F0CFFD0146404602F054
:10005000C3FCD4F860110746304602F0C5FD0146E6
:10006000384602F0B9FC94F87C3100F10046012BCF
:100070007BD1464B1B78DB070ED44023D4F8980184
:1000800090FBF3F3C01A02F05BFD494602F0A4FCBA
:1000900002F086FFC4F898014023D4F8980190FB41
:1000A000F3F002F04DFD0146484602F093FCD4F80F
:1000B000A0110746009802F08FFC0146009802F05C
:1000C00047FED4F89C5180462946384602F082FC0F
:1000D0000146404602F088FD294602F07DFC0546B7
:1000E000C4F89C01584605F0F9FA94F87E71394637
:1000F00000F0C4FDD4F8A4311844C4F8A40130467B
:1001000005F0ECFA394600F0B9FDD4F8A8311844EE
:10011000C4F8A801284605F0E1FA94F87F1100F030
:10012000ADFDD4F8AC31049A1844D4F8B031C4F819
:10013000AC011344C4F8B031D4F8B4310133C4F87D
:10014000B43109B0BDE8F08F2F46A8462E46F5E43D
:10015000C4F88051C4F88451C4F88851C9E54FF0FF
:100160007E51D5E522F0080225E7A88A99E7002309
:100170009363D3631364E4E74C3D0F44DB0FC93F43
:10018000902800200C1500204015002004130020AA
:10019000012310B50A4C4FF48060E370022384F809
:1001A0002030FFF7F7F86421064B1A68064B93F8E6
:1001B000BD3101FB0323636123880133238010BD1C
:1001C00080130020C41300209028002038B5044676
:1001D0008022002107F04DFD3822002104F180002B
:1001E00007F047FD00231748E218C1580433382BA5
:1001F000C2F88010F8D12422134904F1C00005F0A0
:1002000007F90B22114904F1E40005F001F900237C
:1002100003220D4984F8EF3084F8F02001F1300515
:1002200018012A18927912F0100205D0014491F8B1
:10023000343084F8F13038BD01330E2BF0D184F81E
:10024000F12038BDC4810108E49501080896010831
:10025000002370B5084C094D094E2278934200DB0B
:1002600070BD55F8232030EA020204BF0A6846F840
:1002700023200133F1E700BFF81200208411002091
:10028000781200200023F0B5304C1A461846A646D6
:1002900054F8201059B1C1F30325062D00F10100D7
:1002A00008BF0132890448BF01332028F0D100245F
:1002B0000F2527492F464A708B7022462346087027
:1002C000844225D1BA42234E234C35DD3A445010A6
:1002D0000130013A30705210AB4222701F48204C5E
:1002E0002EDD2B445A100132013B22705B1003704B
:1002F00006234A78B2FBF3F003FB102010F0FF0F47
:1003000004D01346062B01DDDA071DD5CB70F0BDF6
:100310005EF824600134C6F3031C624506F00F0644
:10032000B8BF62466745A8BF6746B342B8BF334609
:10033000B542A8BF3546C3E7072232700622CBE795
:10034000072323700623D2E75B10DBE7841100202C
:10035000F81200201B1300201C130020191300208A
:100360001A1300202DE9F04F844B87B01B7803F05F
:10037000FF04002B41D14FF03C0B814927460A89ED
:10038000A44603924A89A64602925846224691F80C
:1003900004904D798B790C804C800194059121B2A9
:1003A00020292DD17649BCF1000F01D0A1F800E041
:1003B0000FB181F80490019800B14D7102B18B71B9
:1003C000BCF1000F01D020234B8001226B4B1A702F
:1003D00091F836338BB140F22A33D1F83823D1F873
:1003E0003C13536000238B840B889BB243F00103C2
:1003F0000B80136843F00103136007B0BDE8F08F72
:10040000604901EB840C9CF803109CF802C0CCF10D
:10041000FF0C1FFA8CFCBCF1000F00F0AA80594EB3
:10042000CCF1FF0C36F8248001FB0CFCB8FBFBFA86
:100430004FEA2C2CBAF1050F00F29E80DFE80AF09B
:10044000033A4F617586A1EB0C0508FB05F5B5FB7A
:10045000F0F55FFA8CF31D44EDB2012217460192CC
:100460004FF0170C4FEA012949EA05490EEB0C063B
:1004700049EA03090496049EA6EB0C08012606FA35
:100480000CFA039E1AEA090FB246029E1FFA88F878
:1004900018BFB246059E1CF1FF3CB04488F80CA082
:1004A000E9D20EF1180E1FFA8EFE01344FF0010C46
:1004B000894674E7B8FBF0F200FB12881FFA88F84F
:1004C0005FFA8CF3C8F13C08A1EB0C0C0CFB08FCA8
:1004D000BCFBF0FC0D469C445FFA8CF1BDE7B8FB19
:1004E000F0F300FB13835FFA8CF29BB2A1EB0C0CD0
:1004F00003FB0CF3B3FBF0F30D461344DBB21146E0
:10050000ABE7B8FBF0F500FB15881FFA88F5C5F1DD
:100510003C08A1EB0C0505FB08F5B5FBF0F55FFA0F
:100520008CF21544EDB20B46E9E7A1EB0C035FFA40
:100530008CF5B8FBF0FC00FB1C8C1FFA8CFC0CFB50
:1005400003FCBCFBF0FC0B46AC44C5E7B8FBF0F386
:1005500000FB13881FFA88F3C3F13C08A1EB0C03DE
:1005600003FB08F3B3FBF0F35FFA8CF52B44DBB22B
:1005700073E70B460D4670E7494671E71E130020EE
:100580002C2C0020781200200B4BD3F84023824201
:100590000CDA93F84623032A0AD1D3F84C331B69AB
:1005A00043B19842B4BF0120022070470020704739
:1005B00002207047012070472C2C002010B50E4CF3
:1005C00094F84633032B15D1D4F84C0303689B6889
:1005D0009847D4F8402394F850331344B3F5807F00
:1005E000A8BF4FF480738342D4BFC4F84033C4F82B
:1005F000400310BD0020ECE72C2C0020054B93F8A5
:100600004623032A03D1D3F84C03F6F74EBB002050
:10061000704700BF2C2C002070B50546064E0446DE
:1006200014F8011B09B9401B70BDD6F84C03F6F74E
:1006300045FB2046F3E700BF2C2C0020024B01466F
:10064000D3F84C03F6F73ABB2C2C00200846F5E70C
:10065000F8B500230646011F083051F8042F02F1B7
:1006600020043F2C3AD802F108040F2C1BD8023288
:10067000032A02D9002B08BF01238142EDD1012BAF
:10068000306812D0022B1ED0736800019B0000F06E
:10069000300003F00C030343B06800F0030018437C
:1006A000BDE8F840CAE70223E7E700F00F0040F09A
:1006B0004000FFF7C3FFB068736800F00F0040EA26
:1006C0000310C0B2ECE700F03F0040F08000FFF7FD
:1006D000B5FF3079FFF7B2FF307AE1E706F10C079A
:1006E0003C46002554F8043DAD0003F18002FF2A8A
:1006F00006D903F50042B2F5803F19D245F0010555
:10070000B442EFD165F03F00C0B2FFF797FF05F0AC
:100710000303022B207819D0032B1ED0012B11D0FC
:100720000434FFF78BFFA7424FEAA505EFD1F8BDD0
:1007300003F50003B3F1807F34BF45F0020545F0B7
:100740000305DDE7FFF77AFF6078E9E7FFF776FF5B
:100750006078FFF773FFA078E2E7FFF76FFF60783C
:10076000FFF76CFFA078FFF769FFE078D8E710B5D6
:1007700004467F2C03D8E0B2BDE810405EE764F089
:100780007F00C0B2FFF75AFFE409F2E7C31783EA1C
:100790004000ECE770B506460D460024AC4200DB95
:1007A00070BD36F91400FFF7F1FF0134F6E70EB41F
:1007B00077B5064607AC482054F8045BFFF73EFFC8
:1007C0002020FFF73BFF3046FFF726FF3A20FFF7D8
:1007D00035FF23462A460A490020019400F048F9D3
:1007E00004460A20FFF72AFF064A0334D2F84033B2
:1007F0001B1BC2F8403303B0BDE8704003B0704724
:100800004D0601082C2C00200FB407B504AB53F89B
:10081000042B05490020019300F02AF903B05DF88C
:1008200004EB04B0704700BF4D060108074BB3F955
:100830005203B3F9543333B190FBF3F203FB1202CA
:1008400018461346F7E7C0B2704700BF2C2C0020B3
:1008500070B50124B0FBF4F58D4202D21CB91C70B6
:1008600070BD4C43F6E7B0FBF4F6092E0BDD002A11
:1008700014BF37255725354404FB160003F8015BE8
:10088000B4FBF1F4EAE73025F5E703685A1C02608F
:1008900019707047002B2DE9F04106460F461446AB
:1008A00014BF4FF030084FF02008069B13F8012BBF
:1008B0003AB92546002D0FDC24EAE47404E0013C3B
:1008C000F4E7002CFBDC0024069D641B281915F8B6
:1008D000011B31B9BDE8F08141463046B847013DC2
:1008E000E8E73046B847F1E770B50446A568084622
:1008F0002B1D013544F82310E168A56002F06CF867
:100900006668E060B54204BF0023A360A3680433B7
:1009100054F8231002F05EF80546E0602068864235
:1009200007DB304602F00CF90146284602F010FAC7
:1009300070BD0130206002F003F90146284602F044
:1009400007FA4FF07E5102F047F870BDF8B50E4639
:1009500004460168304602F047F9616902F03CF84C
:1009600061680546304602F03FF9A16902F034F8AB
:10097000E1680746284602F037F90146384602F09A
:1009800029F8A1686061304602F02EF92169064617
:10099000284602F029F90146304602F01BF8A06112
:1009A0002846F8BD38B5044625680846294602F0B1
:1009B00011F8616802F018F9294602F00DF820607C
:1009C00038BD08467047024B1868F6F777B900BF84
:1009D000140E0020026810B51146531C036011F874
:1009E000024BD31C01605178036093781B0443EAE7
:1009F0000123111D0160D078234343EA006010BD3C
:100A000003685A1C02601A4612F8021B02605878EA
:100A100041EA0020704703685A1C0260187870474A
:100A200038B504461546006804F0F2FC22682A44F2
:100A3000226038BD03685A1C0260197003685A1C92
:100A400002600A0A1A7003685A1C02600A0C1A70C3
:100A50000368090E5A1C02601970704703685A1C1B
:100A6000026019700368090A5A1C02601970704705
:100A70002DE9F04F82468B4615461C46002789B06B
:100A80000DF114082978002930D0252904D05046CA
:100A90000135D8470137F5E76A784FF00009302A69
:100AA00012BF00230123AA780293A2F1300314BFDE
:100AB000AE1CEE1C092B0CD8A2F13003D9B20929C7
:100AC00018D9A2F16103052B1AD8A2F157030A2BFA
:100AD00010DD6C2A74D13278751C642A00F0AB806A
:100AE00022D8252A66D012D8002ACBD1384609B0A0
:100AF000BDE8F08F0A2202FB093916F8012BDBE76B
:100B0000A2F14103052BE4D8A2F13703DFE7582A0D
:100B100018D0632AB6D12E4621785046D847251DD5
:100B200001372C463546ADE7732A37D006D86E2AF2
:100B3000A8D12E46236804341F60F3E7752A65D0D8
:100B4000782A9FD143461021A2F15800424204F175
:100B500004064241206807E02D2340428DF81430FE
:100B60000DF1150300220A21FFF772FE3446CDF87D
:100B70000080029B4A4659465046FFF78BFE0744C9
:100B800080E72D2340428DF814300DF1150300222B
:100B90000A21FFF75DFE3546039CE8E72E462368F1
:100BA0004A460093594600235046FFF773FE251D21
:100BB0000744B6E72E4625215046D8470137B1E70E
:100BC000642A31D00AD8252AF5D002D8002A8DD03F
:100BD000A8E7582A0CD0632A9ED0A3E7732ADED058
:100BE00002D86E2AA6D09DE7752A14D0782A99D10A
:100BF000A2F158014A4204F104054A4120684346E3
:100C000010212C46FFF724FE3546B0E7261D43464B
:100C100000220A219EE7231D0393002243460A2156
:100C20002068FFF715FEB6E72068231D0028039310
:100C3000A7DB4346ABE72068261D00288CDB434634
:100C400090E70FB437B50B4806AB53F8042B016897
:100C500040680193FFF70CFF0446074D2868F6F73C
:100C600024F80028FAD0204603B0BDE8304004B094
:100C7000704700BF882F0020140E002080EAE07328
:100C8000A3EBE0738B4206DB002801DD401A7047BE
:100C900002D0084470470020704770B5044602F047
:100CA0007FF9203040284DD8274D284E2946204630
:100CB00002F056F9002830D1254D244E2946204611
:100CC00002F030F900282ED12249204602F048F9DE
:100CD00000282ED021461C4801F07CFE0446214607
:100CE000204601F081FF05461B4901F07DFF1B49AD
:100CF00001F072FE294601F077FF194901F06AFE02
:100D000029460646204601F06FFF0146304601F0B5
:100D10006BFF214601F060FE70BD2046314601F0B8
:100D200059FE0446C2E72046314601F055FE04460E
:100D3000C4E70C49204602F0F5F80028CFD0214640
:100D40000348C9E7002070BDDB0F4940DB0FC940F5
:100D5000DB0F49C0DB0FC93F92E741B99730083C30
:100D600015A82A3EDB0FC9BF10B514220021044686
:100D700006F07FFF0123636010BD2DE9F74F0546A4
:100D800010461F46884601F0D7FE4B4904464046B0
:100D900001F02AFF0146204601F026FF804604F0BC
:100DA000D7FC0446404604F053FC39468346384697
:100DB00001F012FE0146204601F0CAFF9DF83060A6
:100DC0000746012E4FF0000449D008D3022E5DD013
:100DD0002346A3462646A046A146A2461DE0594604
:100DE0004FF07E5001F0F6FD4FF07C51814601F04E
:100DF000FBFE4FF07E518246384601F0EDFD4FF08C
:100E000040410646584601F0EFFE394683464FF012
:100E10007E5001F0DFFDD046034631465046019337
:100E200001F096FF31462860484601F091FF3146B7
:100E30006860404601F08CFF3146A860584601F0DA
:100E400087FF019BE8603146184601F081FFAC61E5
:100E500028616C612C62EC6103B0BDE8F08F4FF04B
:100E60004041584601F0C0FE4FF07E518146384661
:100E700001F0B2FD394606464FF07E5001F0AAFD62
:100E80004FF07E580346CB46C246C6E74FF07E5130
:100E900000F1004801F0A0FD4FF0404106465846E1
:100EA00001F0A2FE394683464FF07E5001F092FDDC
:100EB000BA460346A146B0E727D4D236002307B589
:100EC0000093034BFFF759FF03B05DF804FB00BF2D
:100ED000F304353F70B50D4601F02EFE044628465A
:100EE00001F02AFE0146204601F032FF04F0ECFB3F
:100EF000014601F071FD4FF0804405460146204651
:100F000004F02CFD4FF07C510646284601F06CFEA3
:100F10000146204604F022FD4FF07E510446304643
:100F200001F058FD0146204601F012FF70BD10B5DA
:100F300041F221040A44914200D110BD11F8013B55
:100F400080EA0320082310F4004F4FEA400018BF46
:100F50006040013B80B2F6D1EDE701234A0901F080
:100F60001F0103FA01F150F822300B4340F8223000
:100F7000704701234A0901F01F0103FA01F150F8FB
:100F80002230194214BF012000207047037903F07A
:100F90000C03042B05D0082B0FD0BBB9B0F80B0005
:100FA00070470B4BB0F80B001B7803EB8302C3EBCD
:100FB000C20300EB430080B27047054BB0F80B0052
:100FC0005B7803EB430300EB8300F4E700207047FA
:100FD000241C002010B4447A631CDBB20444437226
:100FE000A172027A9A4202D810BCF5F782BF10BCF7
:100FF000704708B5202106F062FE034618461BB173
:1010000002780133202AF9D008BD10B50446B0F8A3
:101010000900F6F727F801462046FFF7B7FF4B68AF
:10102000184410BD38B505460C46FFF7EEFF2B7986
:1010300003F00303012B00D001D2047038BD0480FB
:1010400038BD0FB413B5084C04AB53F8042B074953
:1010500020680193FFF70CFD2068F5F74AFF02B006
:10106000BDE8104004B0704764190020D50F010896
:10107000074B1B68597A4A1CD2B219445A728872BB
:10108000197A914202D81846F5F733BF704700BF6E
:101090006419002038B50B4C451E15F8011F206857
:1010A00019B9BDE83840F5F724BF427A531CDBB2CA
:1010B000024443729172027A9A42EED8F5F719FF10
:1010C000EBE700BF641900202DE9F04103790546E4
:1010D00003F0300020280E46144625D10024264F68
:1010E000DFF8A0806B799C4201DBBDE8F0812B79B1
:1010F00003F00303022B11D0032B12D0012B14BFDA
:10110000315D31573846FFF79CFF6B79013B9C42BC
:1011100002DA4046FFF7BEFF0134E3E736F8141069
:10112000F0E736F91410EDE703F00303012B06D0C6
:1011300008D2097848B1102813D0BDE8F08191F9A0
:101140000010F7E7B1F90010F4E70B48FFF779FF5B
:1011500084B1B5F90720B5F905100848BDE8F0419C
:101160006FE76A79064BBDE8F04153F8323053F827
:1011700021008FE7BDE8F08151B301082BB30108CE
:101180000C8C010829B3010838B50D460446FFF759
:101190003CFF2A4601462046BDE8384094E7014816
:1011A00078E700BF6DAA01082DE9F74F314C814661
:1011B00088460025274601F0100300932E4B18683F
:1011C000F5F797FE94F804B00BF00C034B453FD1B4
:1011D0000D2303FB0573B3F80900F5F743FF06463B
:1011E0002046FFF7D3FE0BF00302012A8246716806
:1011F000B06835D039D210F80A0011F80A20831AE5
:101200005A425A41009B03B112BB18F0200F10D074
:101210007AB90D2101FB0571184809680192FFF7A1
:1012200010FF7168019A51442046FFF74DFFFFF708
:10123000B6FF0D2202FB057211481168FFF701FF8E
:10124000B168002251442046FFF73EFFFFF7A7FF99
:101250000135BA2D04F10D04B0D103B0BDE8F08F13
:1012600010F90A0011F90A20C9E730F90A0031F92A
:101270000A20C4E7988201086419002032B30108EB
:1012800033B3010810B5064C0B46024605492068E9
:10129000FFF7EEFB2068F5F72CFEBDE810407EE777
:1012A00064190020D50F01080FB407B504A951F83F
:1012B000040B0191FFF7E6FF03B05DF804EB04B007
:1012C0007047F8B5037903F03003102B0AD0202BB8
:1012D00023D03BBBBDE8F840B0F90720B0F90510BA
:1012E0001148E1E700244579104E1148FFF7D2FE7E
:1012F00006EBC5031F79BC4202D3BDE8F8404EE7B8
:1013000014B10C48FFF7C6FE56F835300A4853F8BA
:101310002410FFF796FE0134EDE74179BDE8F8406F
:101320000648C1E7F8BD00BF3DB301080C8C0108B9
:1013300054B3010829B30108BA9D010864B3010838
:101340000CB407B510F0200009D069B92320FFF7CD
:101350008FFE05A904980191FFF794FF012003B0C7
:101360005DF804EB02B070470020F8E70CB4C30648
:1013700007B500D551B905A904980191FFF782FF7F
:10138000012003B05DF804EB02B070470020F8E7DD
:1013900008B5FFF77FFEBDE8084000E70048F7E723
:1013A00075B30108002310B5074A9C5C9918844264
:1013B00003D18C78C9788C4204D30433502BF4D1F8
:1013C000002010BD012010BDDC1D002010B50C78E0
:1013D00049788C421CD20F4B043033F9102040F670
:1013E00033039A42A8BF1A461923B2F5617FB8BFEA
:1013F0004FF461725C4304F28334944208DA03FBD5
:1014000001F000F283309042B4BF0020012010BDF3
:10141000002010BD3C13002001460148FFF7A9BD84
:10142000FC14002008B51C20FFF7F6FF20B9034B81
:101430001868C0F3805008BD012008BD7C1700204B
:1014400038B50F4B0F4D1B680F4C13F4805F11D054
:101450001D20FFF7E1FF68B90C4A238BD288B5F94C
:101460000600991A884209DD13449842B4BF00204F
:10147000012038BDB5F90600638BF6E7012038BDC1
:101480007C1700203C13002080170020902F0020A4
:101490001FB5084B9B784BB100238DF80C000191D0
:1014A0000D2001A98DF80D30F6F7BCFC05B05DF8F4
:1014B00004FB00BF702F0020F0B500210A2515485D
:1014C00084680A30E27897B2CB1B1BB2002B1EDD7A
:1014D000C2F16402D2B203FB03F694F804E0524373
:1014E0000EFB06F696FBF2F2CEF1640E7244534305
:1014F00093FBF5F307EB87070A3103EB470389B248
:1015000003F57A73782920F8023FDBD1F0BD08BFDC
:101510000122E0E7902F0020F8B52D4B1B685B07F8
:1015200015D52C4E2C4D37783446012F10D06B69D1
:1015300028469847AB692846984701233370EB89C2
:101540002BB1642BB8BF6423244A12681361F8BD21
:10155000EB69284698472B6928469847311D06F1C4
:1015600008002B6A9847B3683169F2681C4E481C22
:10157000B679B042A66908BF277506F1010708BF12
:101580000020032F02BF01272777002704EB8606E0
:101590003362267FA7616EB1266A636AA76A9E429C
:1015A000DEBF9E4633467646BE42A8BF3E46B342A5
:1015B000B8BF334604EB8101CB6204EB8001C96AFA
:1015C0002061521A1344E36000232370AB89B7E70C
:1015D00070170020BC2F0020C8150020901F00208D
:1015E000E21400202DE9F04FAC4B85B01A68994603
:1015F00012F0040F00F03282A94C237D002B00F082
:101600002D82D4F8EC30C31A009346F2A713009A47
:101610009A4240F22382A34DC4F8EC00B5F8008052
:10162000A14FB8F1000F00F0618108209F49BB79FC
:101630000A685E1EE368B3FBF6F392FBF0F6921BBA
:101640009E180E6096FBF0F001F07AFA984901F0CE
:10165000CBFA984904F082F901464FF07E5001F030
:10166000B9F9954901F0C0FA01F09AFCD4F8F430C8
:10167000C4F8F0009E420ABF002308F1FF382B8017
:101680004FF0000318BFA5F800804FF0000818BF06
:10169000C4F8F460C4F8F830C4F8FC30D9F800306D
:1016A00001939B0740F16D81844B186801F044FA67
:1016B0008349814601F098FA824B02901E68002E01
:1016C00000F05D81804B986801F03AFA824630461E
:1016D00001F036FA0146504601F03AFB0646D4F8CE
:1016E0000011484601F080FA314601F07DFA81464A
:1016F000B88901F025FA754901F076FA8346D4F8E5
:10170000F8A04FF07C51484601F06EFA514601F0C6
:1017100063F9029901F068FAD4F8FC1001F05CF961
:10172000594601F061FA6A4A0390506A01F008FADA
:10173000594602904FF07E5001F04CF9029A014652
:10174000104601F051FA039B0146184601F044F996
:1017500051468346C4F8FC00484601F03DF9C4F800
:10176000F800584601F01CFC5A4B18605A4BDFF841
:1017700054B11B78DFF85091122B15D1DBF8002003
:10178000D9F80830DFF860A193FBF2F3D4F8F80041
:10179000AAF8003001F004FCAAF80200D4F8FC001A
:1017A00001F0FEFBAAF804000023444AC9F8003007
:1017B000C9F80430C9F80830CBF800301360019B39
:1017C00013F0040300F0DF802B88002B40F04681EB
:1017D000D4F80401A8EB000001F0B2F93F4901F090
:1017E00003FA0546009801F0A7F90146284601F0E2
:1017F000AFFA01F0D5FB40F2DC539842A8BF18467F
:10180000A3F6B83398424FF00A01B8BF1846C4F89F
:101810000481FFF733FA0546788901F091F92B49E5
:10182000074601F0E1F901464FF07E5001F0D2F891
:101830008046284601F084F90146404601F0D4F97B
:1018400022490546D4F8F80001F0CEF9394601F0F6
:10185000CBF90146284601F0BFF8C4F8F80003F0C0
:101860003DFF05210546FFF709FA1D4A1D4BB2F958
:101870000010186081EAE173A3EBE173B3F5487FD0
:1018800009DAB2F9022082EAE273A3EBE273B3F55C
:10189000487FC0F2E6800020DCE000BF7017002027
:1018A000BC2F00203E190020E21400205404002028
:1018B00008942537B1DC423ED048874A402A0020B0
:1018C000BD378635442A0020342A00206F12833A1F
:1018D000C8150020680C00207A17002000247449E5
:1018E0001C2A00203410002098150020BB79E068E5
:1018F000013BB0FBF3F001F01FF95E4901F074F910
:101900005D4904F02BF801464FF07E5001F062F87B
:101910005A4901F069F903F0E1FE0646388901F001
:101920000FF9D4F8F0305649F61A804601F05CF908
:101930008346304601F004F9594606464FF07E5082
:1019400001F048F80146304601F04EF9DFF858A1A1
:101950000646DAF8240001F0F3F8494901F044F9A9
:10196000414601F041F90146304601F035F803F0F7
:10197000B5FE444B8046CAF8240018608EE6002667
:10198000ADE60026F2E61D4646E73E4A3E4B1068AD
:101990001B680A211B1AB3F5FA7FA8BF4FF4FA732C
:1019A0003A489842B8BF1846FFF768F9D8F80030AF
:1019B0005B7A5843802390FBF3F0B0F5967FA8BF85
:1019C0004FF49670A3F5D6739842B8BF18462023FB
:1019D000D8F80020401BD57E2D49454395FBF3F5F3
:1019E00092F81CE00B68B5F5967F00FB0E30A8BF9F
:1019F0004FF49675B0F5C81FA8BF4FF4C810254B1B
:101A0000D4F808719842B8BF18464FF400530860E4
:101A100090FBF3F0204B9D42ACBF4519C518507F99
:101A200001F08EF84FF06C5101F0DEF8314680463F
:101A3000384600F0D1FF0146404601F0D5F801F0EC
:101A4000AFFA9628A8BF96206FF095039842ACBFD6
:101A5000281AE81A114BC4F80861186005B0BDE8EF
:101A6000F08F0F4BDFF844801B78002B8DD00D4B8F
:101A70001868ACE708942537B1DC423ED048874A65
:101A80006F12833A680C0020640C00200CFEFFFFEC
:101A90005C0C00200000E7FFD4FEFFFF540C002088
:101AA000700C00206C0C0020C8150020741700205A
:101AB000414B2DE9F0411B6806461B077AD53F4C88
:101AC0003F4F04F586707B6898473E4DB4F90C3162
:101AD000397D2B60B4F90E3128466B60B4F91031B2
:101AE000AB60F8F7F7F938492246087810F0040F90
:101AF00016D000239846354FC4F8146104F58C7C49
:101B000004F58F7E35F9234027F8028F2CF8134017
:101B10002EF813400133032BF4D120F00400087099
:101B20002B4B1B787BB12B4B2968B3F90600091AA4
:101B30002960B3F908006968091A6960B3F90A10E5
:101B4000AB685B1AAB60D2F814319BB3F61A224B28
:101B500000249E42214E06F1060716D82046F5F7CE
:101B6000CFF8204655F8203036F9101042008B424D
:101B7000B95EB8BF26F810308B4200F10100C8BF33
:101B8000BB520328EED1BDE8F08120460221C2F805
:101B900014410E4A36F9103037F910400130234411
:101BA00093FBF1F3032822F8023FF3D1BDE8F041A3
:101BB000FBF7B2BABDE8F08170170020BC2F0020FF
:101BC000481B0020881500200C150020641B0020F5
:101BD000701B0020601B00207FC3C901D43000208F
:101BE00003680A7A591C01601A7070472DE9F8439E
:101BF000794D6B6828469847002800F0EA80012359
